:020000041000EA
:1004000000940008910400100D0000007DCB021044
:1004100000000000000000000000000000000000DC
:1004200000000000000000000000000065CB02108A
:10043000000000000000000029CB02101105001090
:1004400011050010D1CB021011050010110500108C
:1004500011050010110500101105001025CA021029
:1004600011050010110500101105001011050010F4
:1004700011050010110500101105001011050010E4
:100480007047EFF3108072B6704780F310887047A2
:10049000FFF7F6FF72B6174C174DAC4209DA216828
:1004A0006268A368043B02DBC858D050FAE70C34FA
:1004B000F3E7124B124CA34208DA19685A6800207D
:1004C000043A01DB8850FBE70833F4E70D480E4996
:1004D0000860BFF34F8F2CF083FBEFF314800221F1
:1004E000084380F31488094880F3098823F0FCFC52
:1004F000FEE70000300500109C0500109C05001070
:10050000F405001000AF010808ED00E0009C0008B1
:10051000FEE7FEE700B504207146084202D0EFF383
:10052000098001E0EFF30880043026F0AFFFFEE71A
:100530000004001000AF010830010000A00C0310FF
:1005400080AF010878020000000C031000180008BA
:1005500000000000000C0310009C000800000000D8
:10056000000C031000C2000860000000600C0310C3
:1005700080CD000840000000A00C0310809B010803
:1005800000000000A00C031000A001080000000003
:0C059000180F031000F80208C00400005F
:10059C00F8B10108A4360000009C000820180000E7
:1005AC0080B40008800D000060C2000880040000C8
:1005BC0000C7000880060000C0CD0008A0AD0000F8
:1005CC00807B010800200000809B010820000000B7
:1005DC00009C01080004000000A00108600200005B
:0805EC0080A20108000C0000D0
:0805F4000000000000000000FF
:1005FC0000000000000000000000000000000000EF
:10060C0000000000000000000000000000000000DE
:1006200010B50A22002100F0ADFA10BD10B50A2263
:10063000002100F067FB10BD10B5034B0A0001005C
:10064000186800F084F810BD20B00108084B10B500
:100650000400002B02D0002100E000BF054B186809
:10066000836A002B00D0984720002FF0C3F8C046C3
:1006700000000000CC190010EC300068704700004A
:10068000044B1B681B6A002B00D1034BEC3318682A
:100690007047C04620B0010884B0010810B5034B74
:1006A0000100186800F0ACF810BDC04620B0010889
:1006B00010B5034B0100186800F058F810BDC04693
:1006C00020B0010882B0002900D101A9101E06D077
:1006D000002B06D013780B601078431E984102B0AF
:1006E000704702204042FAE730B50024A24201D10F
:1006F000002005E0035D651C0C5DA34201D0181BC2
:1007000030BD2C00F2E7002310B59A4200D110BD95
:10071000CC5CC4540133F8E710B5884202D98B1879
:10072000984203D3002307E08B5C8354013AFBD249
:1007300010BDCC5CC45401339A42FAD1F8E70300EF
:100740001218934200D1704719700133F9E74A43F8
:1007500070B51100140000F053F8051E03D02200FC
:100760000021FFF7ECFF280070BD000070B5050008
:10077000002910D00C1F2368002B00DAE418280091
:1007800000F0A4FD1D4A1368002B05D163601460BE
:10079000280000F09CFD70BDA34209D921686018B3
:1007A0008342F3D118685B6841182160EEE71300BB
:1007B0005A68002A01D0A242F9D919685818A042F3
:1007C0000BD120680918581819608242E0D11068CE
:1007D0005268411819605A60DAE7A04202D90C2326
:1007E0002B60D5E721686018824203D110685268F7
:1007F0004118216062605C60CAE7C04608E80108F1
:10080000032370B5CD1C9D43083506000C2D1ED268
:100810000C25A9421DD8300000F058FD254A146867
:100820002100002919D1244C2368002B03D130006A
:1008300000F0C8F820602900300000F0C3F8431C25
:100840002BD10C233000336000F041FD03E0002D7C
:10085000DFDA0C233360002070BD0B685B1B19D4FA
:100860000B2B03D90B60CC18256003E04B688C423E
:100870000DD11360300000F02AFD200007220B305C
:10088000231D9043C31AE7D05A42E250E4E7636065
:100890000C00EFE70C004968C3E70323C41C9C432A
:1008A000A042E1D0211A300000F08CF8431CDBD1CB
:1008B000C7E7C04608E801080CE801080FB40B4B75
:1008C00013B51C68002C05D0A369002B02D12000B1
:1008D00000F0FCFB05AB049AA1682000019300F036
:1008E0001FFD16BC08BC04B01847C04620B0010864
:1008F00070B505000E00002804D08369002B01D1DB
:1009000000F0E4FBAB69AC68002B02D1280000F0DA
:10091000DDFB244B9C420FD16C68A3891B0702D5D9
:100920002369002B1FD12100280000F061FA002864
:1009300019D00120404270BD1B4B9C4201D1AC68D4
:10094000EBE71A4B9C42E8D1EC68E6E70136A3607E
:10095000002B04DAA2699A4216DC0A2914D0236813
:100960005A1C22601970A3683178013B0029EDD12F
:10097000A360002B0FDA22000A31280000F0D6F91C
:10098000431CD6D00A20D6E72200280000F0CEF97A
:10099000431CE8D1CDE70A2023685A1C2260187056
:1009A000C9E7C046FC1A00101C1B0010DC1A00101E
:1009B00010B5034B01001868FFF79AFF10BDC04641
:1009C00020B00108002370B5064C05000800236024
:1009D0002EF002FF431C03D12368002B00D02B60B4
:1009E00070BDC04698E80108C9B20378002B04D056
:1009F0008B4200D170470130F7E74B4259414942E1
:100A00000840F7E702780B78002A03D00130013163
:100A10009A42F7D0D01A70470023C25C0133002AF3
:100A2000FBD1581E704730B50500002A00D130BDFB
:100A30000C78013A6B1C2C700131002C05D19A18EE
:100A40009A42F4D01C700133FAE71D00EDE710B5AF
:100A50000378002B0FD10B785A4253415B42184068
:100A600010BD0023CA5C002AFAD0C45C944201D1B4
:100A70000133F7E701300378002BF2D11800EFE7DC
:100A8000F0B51F000E0087B00590019102920C98FE
:100A90003478FFF7F1FD082200194378751C1340E4
:100AA00036D12D2C36D1B51C74780126002F62D09A
:100AB000102F09D1302C07D120222B789343582BAB
:100AC00054D110276C7802352D4B3900F3181800DB
:100AD000039302F0AFFB049101210023494202007D
:100AE0008C4618002100303909291AD80C00A74279
:100AF00023DD591C09D06346824206D302D10499F2
:100B0000A14202DB0123784320182C780135E9E764
:100B10002E00BCE72B2C01D01E00C7E7B51C747853
:100B2000FAE721004139192901D8373CDFE72100D4
:100B30006139192901D8573CD9E75A1C08D1059ABF
:100B400023331360029B0398002B09D107B0F0BD3B
:100B5000002E00D04042029A002AF7D0002B01D08C
:100B60006B1E0193029B019A1A60EFE73024002F5D
:100B7000AAD10827A8E7302C9ED00A27A4E7C046B0
:100B8000FFFFFF7F37B51300064A05001068046AAF
:100B9000002C00D1044C0A0000942900FFF770FFDC
:100BA0003EBDC04620B0010884B00108F0B51F006A
:100BB0000E008DB00B900291039212983478FFF7DB
:100BC0005BFD082200194378751C134053D12D2C6E
:100BD00053D17478B51C01330193002F00D18AE002
:100BE000102F0AD1302C08D120222B789343582B78
:100BF00000D07AE010276C780235019B002B41D1A0
:100C0000013B04933E4B05933A00FB17049805996A
:100C1000089302F015FB002309900E00002000212C
:100C20000A922200303A092A31D81400A7423DDD49
:100C30005A1C1DD0B14236D802D1099B984232D8F5
:100C4000099B834206D18E4204D101230A9A5B425A
:100C5000A2420DDB0B0002000899380002F010FBE5
:100C6000E31706940793069B079CC0186141012374
:100C70002C780135D5E72E009FE72B2CACD1B51C85
:100C80007478A9E70023049380231B06BBE72200A6
:100C9000413A192A01D8373CC8E72200613A192A9B
:100CA00004D8573CC2E701235B42E1E75A1C09D153
:100CB0000B9A23331360039B04980599002B0ED1E4
:100CC0000DB0F0BD019A002A04D006000F000021EB
:100CD0007042B941039A002AF2D0002B01D06B1E5A
:100CE0000293039B029A1A60EAE73024002F00D097
:100CF00083E7082781E7302C00D175E70A277CE7D6
:100D0000FFFFFF7F37B51300064A05001068046A2D
:100D1000002C00D1044C0A0000942900FFF746FF84
:100D200003B030BD20B0010884B00108F8B505005B
:100D30000E001400002804D08369002B01D100F0BC
:100D4000C5F9224B9C422DD16C68A369A360A3898D
:100D50001B0731D52369002B2ED023682269F7B2F7
:100D6000981A6369F6B2834205DC2100280000F07E
:100D70003FF9002826D1A3680130013BA360236816
:100D80005A1C22601F706369834204D0A389DB0769
:100D90001AD50A2E18D12100280000F029F90028C0
:100DA00012D00FE00A4B9C4201D1AC68CDE7094B51
:100DB0009C42CAD1EC68C8E72100280000F018F86E
:100DC0000028CAD0012676423000F8BDFC1A001077
:100DD0001C1B0010DC1A00100B1E04D0FF2A04D9C3
:100DE0008A2303608B3B180070470A700123FAE7DF
:100DF000364B70B51D6806000C00002D05D0AB69A0
:100E0000002B02D1280000F061F9314B9C420FD138
:100E10006C680C23E25E93B219072DD4D90611D465
:100E200009230120336037331343A381404270BD4F
:100E3000284B9C4201D1AC68EBE7274B9C42E8D1A0
:100E4000EC68E6E75B0713D5616B002908D0230047
:100E50004433994202D03000FFF788FC00236363DB
:100E60002422A3899343A381002363602369236021
:100E70000823A2891343A3812369002B0BD1A0214E
:100E80008022A389890092000B40934203D0210065
:100E9000300000F0D7F90123A289134011D00023BC
:100EA000A36063695B42A361002023698342BED1D2
:100EB0000C23E25E1306BAD540231343A381013805
:100EC000B5E7920700D46369A360EDE720B001089D
:100ED000FC1A00101C1B0010DC1A0010F7B58A89E0
:100EE00005000C00130760D44B68002B04DC0B6C6E
:100EF000002B01DC0020FEBDE76A002FFAD00023A2
:100F00002E682B6080235B01216A1A4034D0606D0B
:100F1000A3895B0706D56368C01A636B002B01D0F9
:100F2000236CC01A0200216A00232800E76AB84730
:100F3000A189431C06D12B681D2B30D82B4ADA40DF
:100F4000D3072CD50023636023692360CB0405D528
:100F5000431C02D12B68002B00D16065616B2E60B1
:100F60000029C7D023004433994202D02800FFF75C
:100F7000FDFB00206063BEE701232800B847431C47
:100F8000C6D12B68002BC3D01D2B01D0162B01D14D
:100F90002E60AFE74023A2891343A381ABE7402330
:100FA0000B430120A3814042A5E70F69002FA1D088
:100FB0000B680F60DB1B01930023920700D14B6984
:100FC000A360019B002B00DC94E7019B3A00216A9F
:100FD0002800A66AB047002803DC4023A2891343F7
:100FE000DFE7019B3F181B1A0193EAE7010040204D
:100FF0000B6970B505000C00002B01D1002070BDFD
:10100000002804D08369002B01D100F05FF80B4B5E
:101010009C4209D16C680C22A35E002BEED021000B
:101020002800FFF75BFFEAE7054B9C4201D1AC6863
:10103000F1E7044B9C42EED1EC68ECE7FC1A00109F
:101040001C1B0010DC1A0010002310B50400036004
:101050004360836081814366C28103614361836130
:10106000190008225C30FFF76AFB054B24626362BB
:10107000044BA362044BE362044B236310BDC046E0
:10108000391800106118001099180010C5180010C8
:1010900010B5024900F08CF810BDC046F10F0010E9
:1010A00070B568254A1E55430E0029007431FFF7BC
:1010B000A7FB041E08D000212A00016046600C3006
:1010C000A0606832FFF73BFB200070BD836913B559
:1010D0000400002B28D18364C3640365134B144AB6
:1010E0001B6882620193984201D101238361200031
:1010F00000F020F86060200000F01CF8A0602000E4
:1011000000F018F80022E06004216068FFF79CFFFF
:1011100001220921A068FFF797FF02221221E0684F
:10112000FFF792FF0123A36113BDC046CC19001045
:1011300091100010F8B51C4B07001E68B369002B16
:1011400002D13000FFF7C2FF4836B4687368013B34
:1011500004D53368002B07D03668F6E70C22A55E6D
:10116000002D0DD06834F2E704213800FFF798FF16
:1011700030600028F0D10C2304003B602000F8BD53
:1011800020000A4B656625606560A560E360256107
:101190006561A561082229005C30FFF7D0FA65631C
:1011A000A563A564E564E9E7CC1900100100FFFF21
:1011B000F7B504000700002601914834002C01D146
:1011C0003000FEBD6368A5680093009B013B00935F
:1011D00001D52468F2E7AB89012B08D90E22AB5E5A
:1011E000013304D029003800019B98470643683535
:1011F000EBE7000070B50E001D000E23C95E96B02F
:101200001400002907DA00232B60B3891B0611D4D0
:101210008023DB000FE06A4600F080FB0028F2DB51
:10122000F022019B12021340054A9B185A42534177
:101230002B60EDE740230020236016B070BDC04650
:1012400000E0FFFFF7B502268B8905000C00334252
:1012500006D0230047332360236101236361F7BD78
:1012600001AB6A46FFF7C6FF009907002800FFF7A9
:10127000C7FA002808D10C22A35E9A05EFD40322F6
:1012800093431E43A681E4E70F4BAB628023A28900
:1012900020601343A381009B20616361019B002BAD
:1012A0000DD00E23E15E280000F04AFB002806D096
:1012B0000322A38993431A0001231343A381A08926
:1012C0003843A081CBE7C0469110001070477047AB
:1012D000936810B5013B9360002B04DA9469A34234
:1012E00007DB0A2905D01368581C10601970080024
:1012F00010BDFFF71BFD0100F9E7F8B506000F0070
:101300001400D518AC4201D1002007E021783A0042
:101310003000FFF7DDFF0134431CF3D1F8BD0000BE
:10132000F0B5A1B003900F0016001D00002805D0F5
:1013300083690593002B01D1FFF7C8FE7B4B9F42C9
:101340005CD1039B5F68BB891B0763D53B69002B9E
:1013500060D0002308AC6361203363761033A3763A
:10136000079535002B78002B01D0252B5CD1AB1BCA
:1013700005930CD0320039000398FFF7BEFF431CE1
:1013800000D1C4E06269059B9446634463612B7895
:10139000002B00D1BBE0012200235242626004A96D
:1013A000543252186E1C2360E360A3601370A3656F
:1013B000317805225E4800F0E9FA751C002835D125
:1013C0002268D30604D5532304A95B182021197081
:1013D000130704D5532304A95B182B211970337804
:1013E0002A2B2CD0350000210A20E3682A786E1CB5
:1013F000303A092A64D900292ED026E04D4B9F426D
:1014000002D1039B9F689EE74B4B9F429BD1039B5E
:10141000DF6898E739000398FFF7EAFC002898D0C6
:101420000120404221B0F0BD01359BE7404B2268CE
:10143000C01A01238340134323602E00B8E7079BA3
:10144000191D1B680791002B01DB0B9304E05B4225
:10145000E3600223134323602B782E2B0AD16B7891
:101460002A2B35D1079B02351A1D1B680792002BCA
:101470002BDB0993314E29780322300000F086FAE5
:10148000002806D04023801B834022680135134387
:101490002360297806222A486E1C217600F076FA0D
:1014A00000283AD0274B002B25D10722079B073372
:1014B0009343083307936369049A9B18636150E769
:1014C000434301219B18350090E701235B42D0E79D
:1014D00000230A201A000135636029786E1C303918
:1014E000092903D9002BC5D00992C3E74243012340
:1014F00052183500F1E707AB00933A00124B210078
:10150000039800E000BF0490049B0133D3D1BB8952
:101510005B0600D584E70D9884E707AB00933A009B
:10152000094B2100039800F07FF8ECE7FC1A00104B
:101530003C1B00101C1B0010DC1A0010421B00108A
:10154000461B001000000000FB120010F7B515004C
:1015500001938A680B6900900C00934200DA130033
:1015600022002B6043321278002A01D001332B6015
:1015700023689B0602D52B6802332B60062723685D
:101580001F4027D0230043331B785A1E9341226803
:10159000920630D42200019943320098089EB04749
:1015A000431C25D0062320682A68E16803400025F3
:1015B000042B03D18D1AEB43DB171D40A36822696E
:1015C000934201DD9B1AED180027BD4220D1002077
:1015D00010E00137E3682A689B1ABB42D2DD220083
:1015E0000123193201990098089EB047431CF0D19D
:1015F00001204042FEBD3020E11843310870210037
:101600005A1C45310978A218433202331170C1E7E0
:10161000220001231A3201990098089EB047431C0A
:10162000E6D00137D1E70000F0B589B004920A0096
:1016300043320593039002920A7E0C000E9B6E2AA1
:1016400000D186E01FD8632A33D008D8002A00D101
:101650008CE0582A4DD0250042352A7030E0642AAB
:1016600001D0692AF7D1196825680A1D280629D5ED
:1016700008681A60002803DA2D23029A404213708A
:101680006B4E0A274FE0732A74D008D86F2A1FD0F8
:10169000702AE0D1202209680A43226003E0752AFB
:1016A00016D0782AD7D12200782145321170614EA8
:1016B00022E025001A684235111D196013682B704D
:1016C000012365E008681A606906D3D500B2D1E746
:1016D00019682568081D186008682E0605D5544E3F
:1016E00008276F2A1BD00A2719E06D06F7D580B2AC
:1016F000F5E745314E4E0A7018682268011D0068F2
:101700001960150621D5D30702D520231A4322607C
:101710001027002803D1202322689A432260230047
:10172000002243331A706368A360002B58DB042245
:10173000216891432160002854D1029D002B5AD08A
:101740002500337842352B7055E05506DBD580B245
:10175000D9E71A680D68101D4969186013682E06CC
:1017600001D5196002E06D06FBD519800023029DAA
:1017700023614FE01A68111D196015680021626825
:10178000280000F003F9002801D0401B6060636866
:1017900023610023029A13703CE023692A00049914
:1017A0000398059DA847431C3ED023689B0715D48A
:1017B000079BE068984239DA180037E022000123DD
:1017C000193204990398059EB047431C2CD001356B
:1017D000E368079A9B1AAB42F0DCE9E70025F7E7DC
:1017E0000028ADD0029D390001F024FD735C013D5D
:1017F0002B700028F7D1082F09D12368DB0706D505
:1018000063682269934202DC3023013D2B70029B06
:101810005B1B2361059B07AA00932100049B03988F
:10182000FFF794FE431CB8D10120404209B0F0BD3F
:101830004D1B00105E1B001070B50C000E25495F9B
:1018400000F0B0F8002803DB636D1B18636570BD02
:10185000A389024A1340A381F9E7C046FFEFFFFFC7
:10186000F8B51F008B8905000C001600DB0505D5B7
:101870000E23C95E0022022300F074F8A389054AF2
:1018800028001340A38132000E23E15E3B0000F0EC
:101890001FF8F8BDFFEFFFFF70B50C000E25495F84
:1018A00000F060F8A389421C03D1054A1340A381CC
:1018B00070BD802252011343A3816065F8E7C046E2
:1018C000FFEFFFFF10B50E23C95E00F015F810BD45
:1018D00070B50500080011000022064C22601A00B5
:1018E00023F0E6F8431C03D12368002B00D02B60C3
:1018F00070BDC04698E80108002370B5064C05008D
:10190000080023602DF040FF431C03D12368002B07
:1019100000D02B6070BDC04698E80108002370B568
:10192000064C05000800110023602DF035FF431C14
:1019300003D12368002B00D02B6070BD98E801080C
:10194000002370B5064C0500080023602DF02CFF25
:10195000431C03D12368002B00D02B6070BDC04610
:1019600098E8010870B50500080011000022064C37
:1019700022601A002DF020FF431C03D12368002BA6
:1019800000D02B6070BDC04698E80108C9B282182B
:10199000904201D10020704703788B42FBD0013088
:1019A000F6E7000070B50500080011000022064CA3
:1019B00022601A002DF008FF431C03D12368002B7E
:1019C00000D02B6070BDC04698E8010824B0010823
:1019D0004300504F534958002E0000202020202063
:1019E00020202020282828282820202020202020CF
:1019F00020202020202020202020208810101010BF
:101A00001010101010101010101010040404040412
:101A1000040404040410101010101010414141413E
:101A20004141010101010101010101010101010126
:101A30000101010101011010101010104242424238
:101A400042420202020202020202020202020202F6
:101A5000020202020202101010102000000000001A
:101A60000000000000000000000000000000000076
:101A70000000000000000000000000000000000066
:101A80000000000000000000000000000000000056
:101A90000000000000000000000000000000000046
:101AA0000000000000000000000000000000000036
:101AB0000000000000000000000000000000000026
:101AC0000000000000000000000000000000000016
:101AD0000000000000000000000000000000000006
:101AE00000000000000000000000000000000000F6
:101AF00000000000000000000000000000000000E6
:101B000000000000000000000000000000000000D5
:101B100000000000000000000000000000000000C5
:101B200000000000000000000000000000000000B5
:101B3000000000000000000000000000232D302BFA
:101B40002000686C4C0065666745464700303132BE
:101B50003334353637383941424344454600303115
:101B60003233343536373839616263646566000074
:101B700005DF70470020FBE706DF7047000000002C
:101B80000800000008000000000200000000000043
:101B90000000000000000000000000000000000045
:101BA00000000000000000000B0000003F000000EB
:101BB000000000003F00000000000000EFF314836D
:101BC0000138421E9041012210409343184380F394
:101BD0001488704730B58BB00290039102A904912C
:101BE000069308210EAB0893042305917020073952
:101BF0000792099302F0FEFB041E10DD002304AAE5
:101C0000019300930021033302F0F6FB050020004E
:101C100002F0FEFB032D05D028000BB030BD84255B
:101C20006D42F9E787256D42F6E7C04670B58CB086
:101C3000039204AA08920822099203AA0A92042293
:101C4000119E0B92109A0490059106920793002E14
:101C500019D00121712002F0CDFB041E16DD0123F5
:101C6000019306AB009308AA0223002102F0C4FBF3
:101C70000500200002F0CCFB032D04D0079B33604D
:101C800028000CB070BD87256D42F9E784256D42B0
:101C9000F6E7C04630B589B002AB04930823029042
:101CA000039105930121043372200692079302F0F9
:101CB000A1FB041E11DD0123019306AB009304AACE
:101CC0000123002102F098FB0500200002F0A0FB98
:101CD000032D05D0280009B030BD84256D42F9E7F9
:101CE00087256D42F6E7C04630B587B002AB049356
:101CF00008230290039101217320059302F07AFBDF
:101D0000041E0EDD002304AA019300930021013379
:101D100002F072FB0500200002F07AFB280007B0F9
:101D200030BD84256D42F9E70020704730B595B08D
:101D30000C000390242200210BA8FEF700FD0AAA44
:101D400006922822079203AA022308920422012164
:101D5000802004940A930992059302F04BFB041E21
:101D60000FDD0123019304AB009306AA0223002197
:101D700002F042FB0500200002F04AFB280015B0EB
:101D800030BD84256D42F9E7862040427047C04649
:101D900030B58FB005002422002105A8FEF7CFFC46
:101DA000032304AC0493012125338020E5800294B1
:101DB000039302F01FFB041E0EDD002302AA019311
:101DC00000930021013302F017FB0500200002F010
:101DD0001FFB28000FB030BD84256D42F9E7C046D7
:101DE000F0B595B007000E001500002124220BA8C5
:101DF0001C00FEF7A4FC04230A930AAB04932823D7
:101E00000593043B07930121223B8020029406970F
:101E100008960995039302F0EDFA041E0FDD0123E5
:101E2000019302AB009304AA0323002102F0E4FA19
:101E30000500200002F0ECFA280015B0F0BD842562
:101E40006D42F9E730B58FB005002422002105A8C6
:101E5000FEF775FC052304AC049301212333802095
:101E6000E5800294039302F0C5FA041E0EDD002300
:101E700002AA019300930021013302F0BDFA05008C
:101E8000200002F0C5FA28000FB030BD84256D4255
:101E9000F9E7C04670B590B006AC06000D002822E8
:101EA00000212000FEF74BFC282301210393802012
:101EB000043BE68002940495059302F09BFA041E0D
:101EC0000FDD0123019304AB009302AA012300213B
:101ED00002F092FA0500200002F09AFA280010B0F1
:101EE00070BD84256D42F9E7F0B5C64600B590B0E7
:101EF00007000E0015000021242207A89846FEF7CF
:101F00001EFC062306AC0693012122338020E780C5
:101F1000029403930496059502F06CFA041E14DDF6
:101F20000123019304AB009302AA0123002102F0D4
:101F300063FA4346059A05001A60200002F068FA29
:101F4000280010B004BC9046F0BD84256D42F7E730
:101F5000F0B5C64600B590B007000E001500002190
:101F6000242207A89846FEF7EAFB072306AC06934F
:101F7000012121338020E780029403930496059584
:101F800002F038FA041E14DD0123019304AB009320
:101F900002AA0123002102F02FFA4346059A050008
:101FA0001A60200002F034FA280010B004BC9046F9
:101FB000F0BD84256D42F7E7F0B593B007000E0041
:101FC00015000021242209A8FEF7B9FB0823089375
:101FD00020330593043B08AC07930121223B80206A
:101FE000E780049406960295039302F003FA041E18
:101FF0000FDD0123019302AB009304AA0223002109
:1020000002F0FAF90500200002F002FA280013B0ED
:10201000F0BD84256D42F9E7F0B5C64600B592B033
:1020200004000F0016000021242209A89846FEF79C
:1020300086FB1D230893236808ADEB60282301214C
:1020400003938020243B04940295059306970796FA
:1020500002F0D0F9041E14DD0223019304AB0093B7
:1020600002AA0123002102F0C7F94346079A05009E
:102070001A60200002F0CCF9280012B004BC90468F
:10208000F0BD84256D42F7E7F0B593B004000F0072
:1020900016000021242209A8FEF751FB1E230893F5
:1020A000236808ADEB602823012105938020243BA1
:1020B0000294049506970796039302F09BF9041E79
:1020C0000FDD0123019302AB009304AA0223002138
:1020D00002F092F90500200002F09AF9280013B0EE
:1020E000F0BD84256D42F9E7F0B591B005000F0011
:1020F00016000021242207A8FEF721FB1B230693CC
:102100002B6806ACE3602823012103938020243B45
:10211000E780A66002940495059302F06BF9041E13
:102120000FDD0123019304AB009302AA01230021D8
:1021300002F062F90500200002F06AF9280011B0EF
:10214000F0BD84256D42F9E7F0B591B005000F00B0
:1021500016000021242207A8FEF7F1FA1C2306939B
:102160002B6806ACE3602823012103938020243BE5
:10217000E780A66002940495059302F03BF9041EE3
:102180000FDD0123019304AB009302AA0123002178
:1021900002F032F90500200002F03AF9280011B0EF
:1021A000F0BD84256D42F9E7F0B5C64600B594B0A0
:1021B000040088461700002124220BA81E00FEF709
:1021C000BEFA1F230A9323680AADEB60282303930A
:1021D00043460493042307931A9B0121802006940D
:1021E000029505970896099302F004F9041E14DD80
:1021F0000223019306AB009302AA0223002102F0FE
:10220000FBF8099A1B9B05001A60200002F000F9F8
:10221000280014B004BC9046F0BD84256D42F7E759
:1022200030B591B004002422002107A8FEF787FAF8
:1022300021230693236806ADEB6028230121039335
:102240008020243B04940295059302F0D3F8041EE9
:102250000FDD0123019304AB009302AA01230021A7
:1022600002F0CAF80500200002F0D2F8280011B0F0
:1022700030BD84256D42F9E7F0B5C64600B592B091
:1022800004000F0016000021242209A89846FEF73A
:1022900056FA20230893236808ADEB602823012118
:1022A00003938020243B0494029505930697079698
:1022B00002F0A0F8041E14DD0223019304AB009386
:1022C00002AA0123002102F097F84346079A05006D
:1022D0001A60200002F09CF8280012B004BC90465E
:1022E000F0BD84256D42F7E770B590B005000E0093
:1022F0002422002107A8FEF722FA0B2306932B685D
:1023000006ACE3602823012103938020243BA660D0
:1023100002940495059302F06DF8041E0FDD01236D
:10232000019304AB009302AA0123002102F064F898
:102330000500200002F06CF8280010B070BD842564
:102340006D42F9E7F0B593B004000F0016000021CC
:10235000242209A8FEF7F3F90C230893236808AD9B
:10236000EB602823012105938020243B02940495EF
:1023700006970796039302F03DF8041E0FDD012334
:10238000019302AB009304AA0223002102F034F867
:102390000500200002F03CF8280013B0F0BD8425B1
:1023A0006D42F9E7F0B5C64600B592B004000F00E3
:1023B00016000021242209A89846FEF7C0F90D2333
:1023C0000893236808ADEB60282301210393802044
:1023D000243B0494029505930697079602F00AF8A9
:1023E000041E14DD0223019304AB009302AA01230F
:1023F000002102F001F84346079A05001A60200008
:1024000002F006F8280012B004BC9046F0BD842506
:102410006D42F7E7F0B593B004000F0016000021FD
:10242000242209A8FEF78BF90E230893236808AD30
:10243000EB602823012105938020243B029404951E
:1024400006970796039301F0D5FF041E0FDD0123C5
:10245000019302AB009304AA0223002101F0CCFFF8
:102460000500200001F0D4FF280013B0F0BD842542
:102470006D42F9E730B591B004002422002107A88D
:10248000FEF75DF90F230693236806ADEB60282362
:10249000012103938020243B04940295059301F0CD
:1024A000A9FF041E0FDD0123019304AB009302AAD0
:1024B0000123002101F0A0FF0500200001F0A8FF8A
:1024C000280011B030BD84256D42F9E770B590B099
:1024D00006000C002422002107A8FEF730F9102383
:1024E0000693336806ADEB6028230393243B0295E3
:1024F00004940593002C02D02368002B18D10121ED
:10250000802001F077FF041E0FDD0123019304AB4F
:10251000009302AA0123002101F06EFF05002000B4
:1025200001F076FF280010B070BD84256D42F9E7F8
:1025300089256D42F6E7C046F0B591B005000F0061
:1025400016000021242207A8FEF7F9F813230693AA
:102550002B6806ACE3602823012103938020243BF1
:10256000E780A66002940495059301F043FF041EE2
:102570000FDD0123019304AB009302AA0123002184
:1025800001F03AFF0500200001F042FF280011B0E1
:10259000F0BD84256D42F9E7F0B591B005000F005C
:1025A00016000021242207A8FEF7C9F81423069379
:1025B0002B6806ACE3602823012103938020243B91
:1025C000E780A66002940495059301F013FF041EB2
:1025D0000FDD0123019304AB009302AA0123002124
:1025E00001F00AFF0500200001F012FF280011B0E1
:1025F000F0BD84256D42F9E7F0B593B004000F00FB
:1026000016000021242209A8FEF799F81523089343
:10261000236808ADEB602823012105938020243B2B
:102620000294049506970796039301F0E3FE041EB7
:102630000FDD0123019302AB009304AA02230021C2
:1026400001F0DAFE0500200001F0E2FE280013B0E0
:10265000F0BD84256D42F9E7F0B5C64600B592B0ED
:1026600004000F0016000021242209A89846FEF756
:1026700066F816230893236808ADEB602823012130
:1026800003938020243B04940295059306970796B4
:1026900001F0B0FE041E14DD0223019304AB00938D
:1026A00002AA0123002101F0A7FE4346079A050074
:1026B0001A60200001F0ACFE280012B004BC904665
:1026C000F0BD84256D42F7E7F0B593B004000F002C
:1026D00016000021242209A8FEF731F817230893D9
:1026E000236808ADEB602823012105938020243B5B
:1026F0000294049506970796039301F07BFE041E4F
:102700000FDD0123019302AB009304AA02230021F1
:1027100001F072FE0500200001F07AFE280013B0DF
:10272000F0BD84256D42F9E730B591B00400242254
:10273000002107A8FEF703F818230693236806ADC7
:10274000EB602823012103938020243B049402950D
:10275000059301F04FFE041E0FDD0123019304AB2E
:10276000009302AA0123002101F046FE050020008B
:1027700001F04EFE280011B030BD84256D42F9E70E
:10278000F0B595B004000F001600002120220BA820
:102790001D00FDF7D4FF22230A936B46DC851A9BAC
:1027A0000C971395002B36D00AAB0493282305937E
:1027B0001C9B06931D9B07931A9B08931B9B0993D5
:1027C0001E9B02931F9B0393102D27D8002E06D02B
:1027D000002D04D02A0031000FA8FDF794FF01213D
:1027E000802001F007FE051E1BDD1A9B01225C1EE6
:1027F000A341019202AA02330092002104AA01F02F
:10280000FBFD039A209B04001A60280001F000FEE3
:10281000200015B0F0BD1B9B002BC5D0872464425F
:10282000F6E784246442F3E7F0B595B004000F00A6
:102830001600002120220BA81D00FDF780FF232396
:102840000A936B46DC851A9B0C971395002B36D0A8
:102850000AAB0493282305931C9B06931D9B0793A7
:102860001A9B08931B9B09931E9B02931F9B039328
:10287000102D27D8002E06D0002D04D02A003100BC
:102880000FA8FDF740FF0121802001F0B3FD051ED8
:102890001BDD1A9B01225C1EA341019202AA023396
:1028A0000092002104AA01F0A7FD039A209B0400D6
:1028B0001A60280001F0ACFD200015B0F0BD1B9B94
:1028C000002BC5D087246442F6E784246442F3E7F2
:1028D000F0B5C64600B592B080460F001600002144
:1028E000242209A81D00FDF72AFF2E230893434642
:1028F00008ACE38028230593189B01210293199BC0
:102900008020A760049406960795039301F072FD5A
:10291000041E14DD0123019302AB009304AA0223D9
:10292000002101F069FD039A1A9B05001A6020003E
:1029300001F06EFD280012B004BC9046F0BD842565
:102940006D42F7E7F0B5C64600B592B080460F007D
:1029500016000021242209A81D00FDF7F0FE2E23F9
:102960000893434608ACE38028230593189B012174
:102970000293199B8020A760049406960795039301
:1029800001F038FD041E14DD0123019302AB009316
:1029900004AA0223002101F02FFD039A1A9B0500CF
:1029A0001A60200001F034FD280012B004BC9046EB
:1029B000F0BD84256D42F7E7F0B5C64600B592B08C
:1029C00080460F0016000021242209A81D00FDF7F3
:1029D000B6FE2F230893434608ACE38028230393D5
:1029E000189B01210693199B8020A76002940496EE
:1029F0000595079301F0FEFC041E10DD002302AADA
:102A0000019300930021033301F0F6FC0500200040
:102A100001F0FEFC280012B004BC9046F0BD8425F5
:102A20006D42F7E7F0B5C64600B592B080460F009C
:102A300016000021242209A81D00FDF780FE2F2387
:102A40000893434608ACE38028230393189B012195
:102A50000693199B8020A76002940496059507931E
:102A600001F0C8FC041E10DD002302AA01930093AC
:102A70000021033301F0C0FC0500200001F0C8FC78
:102A8000280012B004BC9046F0BD84256D42F7E7E3
:102A9000F0B595B005000C001700002124220BA80A
:102AA0001E00FDF74CFE30230A936B46DD851A9B12
:102AB0000C94002B28D00AAB0493282304AC636049
:102AC0001A9BE66023611B9B02AE63611C9BA7609F
:102AD00002931D9B01217360802001F08BFC032376
:102AE000051E2BDD01220096019200212200280004
:102AF00001F082FC72681E9B04001A60280001F03D
:102B000087FC200015B0F0BD1B9B002B19D10AAB30
:102B10000493282304AC63601B9BE660236163611C
:102B20001C9B02AE02931D9BA76073600121802055
:102B300001F060FC051E01DD0223D3E7842464421A
:102B4000DFE787246442DCE7F0B595B005000C00B0
:102B50001700002124220BA81E00FDF7F0FD3123F1
:102B60000A936B46DD851A9B0C94002B28D00AAB88
:102B70000493282304AC63601A9BE66023611B9BCB
:102B800002AE63611C9BA76002931D9B01217360D1
:102B9000802001F02FFC0323051E2BDD012200966F
:102BA000019200212200280001F026FC72681E9B81
:102BB00004001A60280001F02BFC200015B0F0BDC5
:102BC0001B9B002B19D10AAB0493282304AC636030
:102BD0001B9BE660236163611C9B02AE02931D9BFD
:102BE000A76073600121802001F004FC051E01DD57
:102BF0000223D3E784246442DFE787246442DCE7CE
:102C000070B590B006000D002422002107A8FDF742
:102C100096FD33230693336806ACE3602823012135
:102C200003938020243B02940495059301F0E2FB7A
:102C3000041E0FDD0123019304AB009302AA0123BC
:102C4000002101F0D9FB0500200001F0E1FB280084
:102C500010B070BD84256D42F9E7C046F0B591B063
:102C600007000E0015000021242207A8FDF767FDCC
:102C7000382306933B6806ACE360282301218020BB
:102C8000029403930496059501F0B4FB041E0FDD36
:102C90000123019304AB009302AA0123002101F058
:102CA000ABFB0500200001F0B3FB280011B0F0BD24
:102CB00084256D42F9E7C046F0B58FB005000F00DE
:102CC00016000021202206A8FDF739FD36230493C3
:102CD0002B6804ACE360282301218020A780E680D4
:102CE0000294039301F086FB041E0EDD002302AA6A
:102CF000019300930021013301F07EFB05002000C9
:102D000001F086FB28000FB0F0BD84256D42F9E785
:102D100030B591B004002422002107A8FDF70FFD73
:102D20003A230693236806ADEB6028230121039321
:102D30008020243B04940295059301F05BFB041E64
:102D40000FDD0123019304AB009302AA01230021AC
:102D500001F052FB0500200001F05AFB280011B0E1
:102D600030BD84256D42F9E7F0B5C64600B592B096
:102D7000050088461700002120220AA81E00FDF742
:102D8000DEFC37230893434608ACA3802B6801215F
:102D9000E36028230593189B802007930423E78092
:102DA000049406960295039301F024FB041E11DDA2
:102DB0000123019302AB009304AA0223002101F036
:102DC0001BFB0500200001F023FB280012B004BC0F
:102DD0009046F0BD84256D42F7E7C04630B591B00E
:102DE00005000C002422002107A8FDF7A8FC3C23C5
:102DF000069306AB029328230495039305940025BC
:102E0000002C02D1280011B030BD0121802001F03A
:102E1000F1FA041E0DDD0123019304AB009302AA15
:102E20000123002101F0E8FA0500200001F0F0FA8A
:102E3000E8E784256D42E5E730B593B00C00050066
:102E40002422002109A8FDF77AFC3D23089308AB52
:102E5000049328230593043B07930121223B802000
:102E600002940695039301F0C5FA041E0FDD0123B9
:102E7000019302AB009304AA0223002101F0BCFAE3
:102E80000500200001F0C4FA280013B030BD8425ED
:102E90006D42F9E7862040427047C0468620404296
:102EA0007047C046862040427047C0468620404258
:102EB0007047C046862040427047C0468620404248
:102EC0007047C046862040427047C0468620404238
:102ED0007047C046862040427047C0468620404228
:102EE0007047C046862040427047C046F0B5C6468F
:102EF00000B592B00700884616000021242209A8D8
:102F00001D00FDF71CFC3B230893434608ACE380FF
:102F100028230593189B01210293199B8020A76009
:102F2000049406960795039301F064FA041E14DDD9
:102F30000123019302AB009304AA0223002101F0B4
:102F40005BFA039A1A9B05001A60200001F060FAF0
:102F5000280012B004BC9046F0BD84256D42F7E70E
:102F600070B590B005000E002422002107A8FDF7DF
:102F7000E6FB322306932B6806ACE360282301218D
:102F800003938020243BA66002940495059301F0EE
:102F900031FA041E0FDD0123019304AB009302AA52
:102FA0000123002101F028FA0500200001F030FA89
:102FB000280010B070BD84256D42F9E770B58EB061
:102FC00006000D002422002105A8FDF7B8FB3423DC
:102FD0000493336804ACE360282301218020256139
:102FE0000294039301F006FA041E0EDD002302AAE8
:102FF000019300930021013301F0FEF90500200048
:1030000001F006FA28000EB070BD84256D42F9E784
:10301000F0B5C64607001E2000B590B088461600E1
:103020000021222268441D00FDF789FB3523069309
:10303000434606ACA3803B680121E360282380203F
:10304000029403930496059501F0D4F9041E10DD53
:10305000002302AA019300930021023301F0CCF96E
:103060000500200001F0D4F9280010B004BC9046FF
:10307000F0BD84256D42F7E7F0B593B006000F0070
:1030800015000021242209A8FDF759FB39230893D4
:103090003B6808ACE36028230593043B07930121B8
:1030A000223B8020049406960295039301F0A2F936
:1030B000041E0FDD0123019302AB009304AA022337
:1030C000002101F099F90500200001F0A1F9280084
:1030D00013B0F0BD84256D42F9E7C046862040421A
:1030E0007047C046862040427047C0468620404216
:1030F0007047C046862040427047C0468620404206
:103100007047C046862040427047C04686204042F5
:103110007047C04602B4714649084900095C49003D
:103120008E4402BC7047C046002243088B4274D3D1
:1031300003098B425FD3030A8B4244D3030B8B42B8
:1031400028D3030C8B420DD3FF22090212BA030CC1
:103150008B4202D31212090265D0030B8B4219D3A2
:1031600000E0090AC30B8B4201D3CB03C01A5241C2
:10317000830B8B4201D38B03C01A5241430B8B420A
:1031800001D34B03C01A5241030B8B4201D30B03F3
:10319000C01A5241C30A8B4201D3CB02C01A52411A
:1031A000830A8B4201D38B02C01A5241430A8B42DD
:1031B00001D34B02C01A5241030A8B4201D30B02C6
:1031C000C01A5241CDD2C3098B4201D3CB01C01AE0
:1031D000524183098B4201D38B01C01A52414309EA
:1031E0008B4201D34B01C01A524103098B4201D3D8
:1031F0000B01C01A5241C3088B4201D3CB00C01A45
:10320000524183088B4201D38B00C01A52414308BC
:103210008B4201D34B00C01A5241411A00D20146E1
:10322000524110467047FFE701B5002000F006F854
:1032300002BDC0460029F7D076E770477047C04608
:10324000002B11D1002A0FD1002900D1002802D073
:103250000021C943081C07B4024802A1401802908B
:1032600003BDC046D9FFFFFF03B4684601B502980D
:1032700000F030F8019B9E4602B00CBC7047C0467F
:10328000F0B5CE46474615042D0C2E0080B5070438
:10329000140C3F0C9946030C7E435D436743634324
:1032A0007F19340CE4199C46A54203D980235B02A4
:1032B0009846C4444B4643435143250C3604654469
:1032C000360C2404A4195B19591820000CBC904634
:1032D0009946F0BDF0B54F464646D646C0B5040007
:1032E00082B00D00914698468B422FD82CD0414693
:1032F000484600F0B1F829000600200000F0ACF8C4
:10330000331A9C46203B9A4600D576E04B465246FF
:1033100093401F004B46624693401E00AF4228D8A0
:1033200025D05346A41BBD41002B00DA7BE00022D0
:1033300000230092019301235246934001930123FD
:1033400062469340009318E08242D0D900220023C5
:10335000009201930A9B002B01D01C605D600098D5
:10336000019902B01CBC90469946A246F0BDA3420A
:10337000D7D900220023009201936346002BE9D0A5
:10338000FB079846414672080A437B0866460EE0F2
:10339000AB4201D1A2420CD8A41A9D4101202419AC
:1033A0006D410021013E24184D41002E06D0AB4254
:1033B000EED9013E24196D41002EF8D100980199F3
:1033C000534600196941002B23DB2B005246D340A2
:1033D0002A006446E2401C0053461500002B2DDBFA
:1033E00026005746BE40330026006746BE403200E6
:1033F000801A994100900191ACE7624620239B1A04
:103400004A46DA406146130042468A4017001F438D
:1034100080E7624620239B1A2A0066469A402300D2
:10342000F3401343D4E76246202300219B1A002275
:10343000009101920122DA40019280E72023624646
:1034400026009B1ADE402F00B0466646B74046462F
:103450003B003343C8E7C04610B5002903D100F054
:1034600007F8203002E0081C00F002F810BDC0464A
:103470001C2101231B04984201D3000C10391B0AA4
:10348000984201D3000A08391B09984201D3000968
:10349000043902A2105C40187047C04604030202BF
:1034A0000101010100000000000000000FB4F0B5B0
:1034B0005746DE464E464546E0B595B01EAE08CEB0
:1034C00000249A46002357469B4607960B933B7869
:1034D000002B12D07A1C9046252B20D00BAD621CFD
:1034E0002C190B9223711F2A24D8012347469C468E
:1034F0003B78E3441400002BECD1002C04D02100D5
:103500000CA821F0BFFA8344584615B03CBC904645
:103510009946A246AB46F0BC08BC04B018477B787D
:10352000253BDBB2532B01D900F09EFC854A9B0062
:10353000D3589F46002320210CA80B9321F0A2FA18
:103540000B9AD2E70023804A0BAD984691462A0099
:103550004546B04616003033621C34193260237180
:103560001F2A0BD84B4601355B5D002B12D014008F
:10357000621C3419326023711F2AF3D900232021E1
:103580000CA8336021F07EFA4B4601355B5D326852
:10359000002BECD133004646A8461D00331D019395
:1035A00008AB924600210C22180034689946FDF7BA
:1035B000C6F80F231A00494664482240825CC3447F
:1035C0000A7003925246984621090132002901D11E
:1035D00000F0D7FD4E461940415C7170260A01D1BA
:1035E00000F010FE1E404B46865D9E70230B01D1FD
:1035F00000F031FE1900434619404B46415CD9703A
:10360000230C01D100F04BFE1E0043461E404B46EA
:10361000865D1E71230D01D100F04AFE190043465C
:1036200019404B46415C5971230E01D100F076FEE2
:1036300046461E404B46865D240F9E7101D100F028
:1036400090FE015DD97106230293023398465346DA
:10365000EB182A6019711F2A01D900F06BFD541C68
:10366000AA182C6016711F2C01D900F0A6FC029B31
:10367000002B01D100F05CFC4346DE1E4B469A5DF8
:10368000631C2C192B6022711F2B01D900F014FD33
:10369000002E01D100F078FC4246161F4A46925D8A
:1036A0005C1CEB182C601A711F2C01D900F02FFD47
:1036B000002E01D100F092FC43465E1F4B469A5DFE
:1036C000631C2C192B6022711F2B01D900F071FD96
:1036D000002E01D100F00AFD4246961F4A46925D37
:1036E0005C1CEB182C601A711F2C06D900232021BA
:1036F0000CA82B6021F0C6F92C68002E01D100F037
:1037000017FD46464B46073E9A5D631C2C192B60FD
:1037100022711F2B01D900F077FC002E01D100F09F
:103720005AFD039A5C1CEB182C601A7108261F2C9A
:1037300000D80FE2002320210CA82B6021F0A2F971
:103740002C6807E2284400109845001078450010C6
:10375000331D029308AB180036680C2200219946ED
:10376000FCF7EDFF631C9A46002E00DAA6E3002367
:10377000B046012603930BAD0A214046FFF75AFDE0
:103780004A463031CBB213700A2140460593FFF709
:10379000CBFC002801D100F0E9FC0A21FFF74AFD2B
:1037A0004B463031CEB25E7064214046FFF7BCFC20
:1037B000002801D100F017FD0A21FFF73BFD303151
:1037C000CBB24A46FA219370890040460193FFF735
:1037D000ABFC002801D100F02DFD0A21FFF72AFDE6
:1037E0004B463031CEB2DE70E4494046FFF79CFCD8
:1037F000002801D100F049FD0A21FFF71BFD4A46D0
:103800003031CBB21371DE4940460193FFF78CFC97
:10381000002801D100F055FD0A21FFF70BFD4B46B2
:103820003031CEB25E71D7494046FFF77DFC0028AB
:1038300001D100F05BFD0A21FFF7FCFC4A46303164
:10384000CBB29371D04940460193FFF76DFC00283D
:1038500001D100F075FD0A21FFF7ECFC4B46303139
:10386000CEB2DE71C9494046FFF75EFC002801D1A7
:1038700000F091FD0A21FFF7DDFC4A463031CBB262
:103880001372C34940460193FFF74EFC002801D153
:1038900000F0A0FD4B463030C6B25E7208230493A0
:1038A0000233984653462C192B6026711F2B01D9E1
:1038B00000F052FC5346019A5C1CEB182C601A7104
:1038C0001F2C00D971E3049B002B01D100F0CCFC2C
:1038D0004346DE1E4B469A5D631C2C192B602271F9
:1038E0001F2B00D9F1E3002E01D100F0C9FC4246A4
:1038F000161F4A46925D5C1CEB182C601A711F2C37
:1039000001D900F0FBFB002E01D100F0E3FC43469F
:103910005E1F4B469A5D631C2C192B6022711F2B76
:1039200001D900F04FFC002E01D100F0FDFC424611
:10393000961F4A46925D5C1CEB182C601A711F2C76
:1039400006D9002320210CA82B6021F09BF82C68BD
:10395000002E01D100F0EDFC4346DE1F4B469A5D80
:10396000631C2C192B6022711F2B00D955E3002EEC
:1039700001D100F016FD46464A46083E925D5C1CA9
:10398000EB182C601A711F2C00D966E3002E01D1B0
:1039900000F029FD46464B46093E9A5D631C2C19F2
:1039A0002B6022711F2B00D95FE3002E00D16CE346
:1039B000059A5C1CEB182C601A711F2C01D900F0C1
:1039C0009BFC039E0A36B3440237029E7FE5331DFB
:1039D00032780BAD9846631C2C190B9322711F2B68
:1039E00000D97DE2012294461C00E344464602379A
:1039F0006DE5331D019308AB00210C2218003568DA
:103A00009946FCF79CFE63490F231A002A408A5C02
:103A1000984692464A46504610702809621C002873
:103A200000D19FE24E461840085C70702E0A00D10B
:103A3000ADE21E404B468E5D9E702B0B00D12BE3FA
:103A40001800434618404B46085CD8702B0C00D138
:103A50004FE31E0043461E404B468E5D1E712B0DEC
:103A600000D1BDE21800434618404B46085C58712F
:103A70002B0E00D1B2E346461E404B468E5D2D0F05
:103A80009E7100D1CEE3485DD871062302930233C4
:103A900098460BAD2C190B9220711F2A00D959E2C0
:103AA000541CAA182C6016711F2C00D928E2029B06
:103AB000002B00D13CE24346DE1E4B469A5D631C60
:103AC0002C192B6022711F2B00D921E2002E00D16E
:103AD0005AE24246161F4A46925D5C1CEB182C6067
:103AE0001A711F2C00D91BE2002E00D176E243464A
:103AF0005E1F4B469A5D631C2C192B6022711F2B95
:103B000000D939E2002E00D1F0E24246961F4A4623
:103B1000925D5C1CEB182C601A711F2C00D93CE2E2
:103B2000002E00D104E346464B46073E9A5D631CD7
:103B30002C192B6022711F2B00D9B5E2002E00D169
:103B400049E352465C1CEB182C601A7108261F2CA6
:103B500000D9EFE5B3440237019EB8E425220BAD4E
:103B6000631C2C190B9322711F2B00D9C0E1012279
:103B700094461C00E3440237A9E4C0461027000025
:103B8000A086010040420F008096980000E1F505F4
:103B900000CA9A3B88450010331D019308AB0021F1
:103BA0000C22180035689946FCF7C9FDE1492BE75E
:103BB000331D029308AB994635680C22180000218A
:103BC000FCF7BDFD0A212800FFF734FB4A463031DF
:103BD000CBB213700A2128000493FFF7A5FA631CE7
:103BE0009A46002800D103E20A21FFF723FB4B4647
:103BF0003031CEB25E7064212800FFF795FA0028BC
:103C000000D1F8E20A21FFF715FB3031CBB298461C
:103C1000FA214B46424689009A702800FFF784FA41
:103C2000002800D10FE30A21FFF704FB4B46303197
:103C3000CEB2DE70C0492800FFF776FA002800D126
:103C400019E30A21FFF7F6FA3031CBB298464B461A
:103C50004246BA491A712800FFF766FA002800D1D7
:103C60003CE30A21FFF7E6FA4B463031CEB25E71F3
:103C7000B3492800FFF758FA002800D149E30A2188
:103C8000FFF7D8FA3031CBB298464B464246AD49A1
:103C90009A712800FFF748FA002800D159E30A2159
:103CA000FFF7C8FA4B463031CEB2DE71A649280084
:103CB000FFF73AFA002800D178E30A21FFF7BAFAB1
:103CC0003031CBB298464B464246A0491A72280082
:103CD000FFF72AFA002800D171E34B463030C6B214
:103CE0005E72082303930233019353460BAD2C19E4
:103CF0000B9326711F2B00D925E2534642465C1CCC
:103D0000EB182C601A711F2C00D95FE1039B002B6C
:103D100000D1ADE2019BDE1E4B469A5D631C2C195F
:103D20002B6022711F2B00D9D8E1002E00D1B2E206
:103D3000019A5C1C161F4A46925DEB182C601A71A2
:103D40001F2C00D9ECE1002E00D1AEE2019B5E1FDA
:103D50004B469A5D631C2C192B6022711F2B00D9D6
:103D60001FE2002E00D1D0E2019A5C1C961F4A4649
:103D7000925DEB182C601A711F2C06D900232021AC
:103D80000CA82B6020F07EFE2C68002E00D1D4E21F
:103D9000019BDE1F4B469A5D631C2C192B60227120
:103DA0001F2B00D941E1002E00D104E34A46019EB9
:103DB0005C1C083E925DEB182C601A711F2C00D918
:103DC00043E1002E00D102E34B46019E093E9A5D7D
:103DD000631C2C192B6022711F2B00D94DE1002E82
:103DE00000D156E1049A5C1CEB182C601A710A266B
:103DF0001F2C00D8E7E5002320210CA82B6020F021
:103E000041FE2C68DFE5331D994633681A789846E1
:103E1000002A25D000239A463B000BAD4746984622
:103E2000631C2C1900262B6022711F2B0AD8013627
:103E3000BA5D002A11D01C00631C2C192B60227162
:103E40001F2BF4D9534620210CA801362B6020F0FB
:103E500019FEBA5D2B68002AEDD147461C00B34419
:103E60004E460237FFF733FB394B5B22994600235E
:103E70000BAD9A46631C2C1900272B6022711F2B57
:103E80000BD84A460137D25D002A12D01C00631CB1
:103E90002C192B6022711F2BF3D9534620210CA81B
:103EA0002B6020F0EFFD4A460137D25D2B68002AD7
:103EB000ECD1BB441C004746FFF709FB0B932D23B5
:103EC0000BAD2C19237153461F2B00D9A1E173426E
:103ED000984601239C4654460226E24403934BE451
:103EE000002320210CA80B9320F0CCFD0B9B79E53F
:103EF000002320210CA80B9320F0C4FD0B9B36E679
:103F0000002320210CA82B6020F0BCFD2C68CEE5FE
:103F1000002320210CA82B6020F0B4FD2B68D5E5F0
:103F2000002320210CA82B6020F0ACFD2C68DBE5E1
:103F300002260FE67845001010270000A086010039
:103F400040420F008096980000E1F50500CA9A3BB8
:103F50009C450010002320210CA80B9320F092FD1B
:103F60000B9A9DE553460BAD2C190B9223711F2A1A
:103F700063D814000126EDE5002320210CA82B6056
:103F800020F080FD2B68BDE51C000326E2E5002340
:103F900002930233564698467BE5002320210CA865
:103FA0002B6020F06FFD2C68BAE5002320210CA8BF
:103FB0002B6020F067FD2C6885E4002320210CA8ED
:103FC0002B6020F05FFD2C68FFF751FB00232021C0
:103FD0000CA82B6020F056FD2C6897E60426B9E566
:103FE000030030001E00032302930233984650E57D
:103FF0000BAD0B93049B2C19237153461F2B00D937
:10400000C0E154460126DEE4002320210CA82B60E9
:1040100020F038FD2B68FFF780FB002320210CA83F
:104020002B6020F02FFD2B68A1E4002320210CA899
:104030002B6020F027FD2B68B5E60B9020210CA803
:1040400020F020FD01260B9C84E5002320210CA8F4
:104050002B6020F017FD2C68B3E6002320210CA86C
:104060002B6020F00FFD2C6890E4002320210CA889
:104070002B6020F007FD2B6897E4002320210CA87B
:104080002B6020F0FFFC2B68A9E6039E1C0009367C
:1040900099E41C00092696E4030030001E00012369
:1040A000029302339846F4E4002320210CA82B60ED
:1040B00020F0E8FC2B6841E5002320210CA82B60B0
:1040C00020F0E0FC2B68FFF7E3FA002320210CA886
:1040D0002B6020F0D7FC2B68FFF705FC0023202184
:1040E0000CA82B6020F0CEFC2B681EE61C000526D9
:1040F00030E50223029302339846CAE400232021CC
:104100000CA82B6020F0BEFC2C68FFF7FCFB002302
:1041100020210CA82B6020F0B5FC2C68FFF7C8FA12
:10412000002320210CA82B6020F0ACFC2C680AE6B0
:1041300006260FE5002320210CA82B6020F0A2FC0E
:104140002A68FFF78CFA002320210CA80B9320F09B
:1041500099FC0B9B9A46D0E5002320210CA82B60EC
:1041600020F090FC2B689A46FFF7A4FB53462B6087
:10417000059B2C19237153461F2B00D9FAE0544696
:1041800021E453460398EB182A6018711F2A00D8BF
:10419000EFE629600CA8202120F074FC01262C6891
:1041A000D8E4002320210CA82B6020F06BFC2B68A6
:1041B000D7E5002320210CA82B6020F063FC2B689E
:1041C000FFF786FA002320210CA82B6020F05AFC70
:1041D0002B68FFF7A8FB1C000726BBE4042302930F
:1041E0000233984655E4059B019300230493023360
:1041F0009846FFF757FB049B98460023039302332E
:10420000019372E5002302930233039E9846FFF761
:104210001EFA002320210CA80B9320F033FC0B9BEB
:104220009A4654E6030030001E0005230293023331
:1042300098462EE43300019E019301230493023338
:104240009846FFF72FFB3300464698460123039319
:104250000233019349E50B0031001E000123029354
:1042600002339846FFF7F3F9039E0236FFF7ABFBE4
:104270000226FFF7A8FB022303930233019334E5E0
:10428000039E1C000336FFF79EFB022304930233B8
:104290009846FFF707FB1C000326FFF794FB022359
:1042A000029302339846FFF7D2F90426FFF78BFBFF
:1042B0000B0031001E000323029302339846FFF7E0
:1042C000C6F93300019E01930323049302339846F9
:1042D000FFF7E8FA039E0436FFF775FB3300464606
:1042E00098460323039302330193FEE404230493CB
:1042F00002339846FFF7D6FA002320210CA82B6042
:1043000020F0C0FB2C68FFF75CFB1C000526FFF7C4
:104310005AFB0423039302330193E6E4042302933C
:1043200002339846FFF793F9039E1C000536FFF70A
:104330004AFB039E0636FFF746FB0626FFF743FBC4
:104340003300019E01930523049302339846FFF73F
:10435000A9FA330046469846052303930233019396
:10436000C3E40B0031001E0005230293023398467C
:10437000FFF76DF9286020210CA820F083FB2C6842
:10438000FFF721FB0B9020210CA820F07BFB0126DE
:104390000B9CFFF718FB0623049302339846FFF7A4
:1043A00081FA039E1C000736FFF70DFB06230393DB
:1043B0000233019399E41C000726FFF704FB330046
:1043C0004646984607230393023301938DE408265B
:1043D000FFF7F9FA3300019E019307230493023398
:1043E0009846FFF75FFA039E0836FFF7ECFAC046DF
:1043F00011DF704710DF704700B585B00293079B4F
:104400000191039301A9069BFFF7F2FF05B000BDE0
:1044100012DF70470BDF704713DF704715DF7047FF
:1044200017DF704718DF70475C3B0010683E0010D4
:10443000683E0010683E0010683E0010683E0010A4
:10444000683E0010683E0010683E0010683E001094
:10445000683E0010683E0010683E0010683E001084
:10446000683E0010683E0010683E0010683E001074
:10447000683E0010683E0010683E0010683E001064
:10448000683E0010683E0010683E0010683E001054
:10449000683E0010683E0010683E0010683E001044
:1044A000683E0010683E0010683E0010683E001034
:1044B000683E0010683E0010683E0010683E001024
:1044C000683E0010683E0010683E0010683E001014
:1044D000683E0010683E0010683E0010683E001004
:1044E000683E0010683E0010683E0010683E0010F4
:1044F000683E0010F2390010683E0010683E00105F
:10450000683E0010683E0010683E0010683E0010D3
:10451000683E0010683E0010683E0010683E0010C3
:10452000CE39001050370010683E0010683E001071
:10453000683E0010683E001050370010683E0010C2
:10454000683E0010683E0010683E0010683E001093
:10455000683E001044350010683E0010683E0010B0
:10456000063E0010683E0010B03B0010683E001090
:10457000683E0010983B0010303132333435363706
:1045800038396162636465663031323334353637C9
:104590003839414243444546307800005B556E73DC
:1045A0007570706F72746564205461675D000000FF
:1045B00000000000000000000000000000000000FB
:1045C000F0B5CE46474680B58DB000F00DF9002815
:1045D00025D106AB81279846734C08AE7F428021D7
:1045E000012009064042FFF715FF0300C20676D4FA
:1045F000820645D4420614D4020600D59BE08020F2
:10460000400003420CD02100FFF706FF2568AB1CD9
:1046100000DAC5E0002D00DBB1E00021A6E0FEE7F6
:10462000FEE721004020FFF7F7FE21688B1C00DA2F
:10463000A4E00029F1DB00D0A0E023696068082B2A
:1046400000D0AFE0226A0C2A00D0ABE04246FFF770
:10465000E5FE2369984200D0A4E0069A079B0096E5
:10466000A06800F02BF9051E05D1236A3200002155
:104670006068FFF7D5FE29006068FFF7D3FEAEE75C
:1046800021002020FFF7C8FE21688B1C00DA88E09B
:104690000029C2DB00D084E023696068082B69D15F
:1046A0006269042A66D13200FFF7B8FE2369984296
:1046B00060D1636905AA01216068FFF7AFFE6369F5
:1046C000984257D143460293236A0193059B009376
:1046D000A068089A099B00F0C5F8010046E0210097
:1046E0001020FFF799FE21688B1C46DB002994DB24
:1046F00043D12369A5686068082B3BD1A269042ACD
:1047000038D13200FFF78AFE2369984232D1A3697B
:10471000424602216068FFF781FEA369984229D1D1
:10472000069B2800019363690093089A099B00F097
:1047300069F801001AE021008020FFF76DFE216872
:104740008B1C19DB002900DA67E715D12369606843
:10475000082B0FD13200FFF761FE2369984209D17F
:10476000089A099BA06800F0CDF801006068FFF787
:1047700059FE34E73900F9E7FEE7FEE7FEE7002DD2
:104780000ED1236A9946042BF4D100F0E1F82900F8
:1047900008904B4632006068FFF742FE2900E5E7CB
:1047A000FEE7FEE73D0066E7009C0008074B10B5FA
:1047B00002000C0058680B000121FFF72FFE201AA1
:1047C000441EA04180234042984310BD009C000835
:1047D00010B50B000349020048680021FFF720FED6
:1047E00010BDC046009C000810B500F0B3F80028CA
:1047F00000D110BD00F0E8F90028FAD100F0AAF8C5
:10480000F7E7C04630B51D00130083B014002B43FA
:104810001FD00723079A9A431ED10123104A5B42F7
:1048200012196B41002B09D0069B02000093200057
:10483000079B290000F0CEF803B030BDFF2AF3D863
:10484000079B22000193069B00932B0029F044FF55
:10485000F2E787204042EFE786204042ECE7C0467F
:1048600000FFFFFF30B51D00130085B014002B437F
:104870001FD00123104A5B4212196B41002B0BD051
:104880000A9B02000193099B200000932900089BCA
:1048900000F06EF805B030BDFF2AF1D80A9B220067
:1048A0000293099B0193089B00932B0029F018FFAA
:1048B000F0E787204042EDE700FFFFFF30B51D0025
:1048C000130083B014002B4317D001230C4A5B4222
:1048D00012196B41002B07D00200069B2000290013
:1048E00000F00CF903B030BDFF2AF5D8069B22007A
:1048F00000932B0029F022FFF4E787204042F1E7E4
:1049000000FFFFFF70B51D00130014002B4316D0ED
:1049100001230E4A5B4212196B41002B08D00200A2
:104920002900200000F012F9030095330AD070BD71
:10493000FF2AF4D822002B0029F01EFFF7E787207A
:104940004042F4E784204042F1E7C04600FFFFFF09
:104950000020704710B5044C200000F013FA034B00
:10496000283C5C6010BDC046609C0008309C00087C
:10497000F8B5154D1E002B0000F07EFB041E01D083
:104980002000F8BD114F2868390000F001FD041E19
:1049900004D1FD69B54208D28724644280220021F7
:1049A00012013800FBF7CBFEEAE7069BAD1B9D42E8
:1049B00007D8074829003018FFF70AFF079B1D603A
:1049C000ECE71D00F5E7C046309C0008389C000865
:1049D000609C0008F0B557464E46DE4645469A466E
:1049E000FB23E0B583B091460C9A06000F00DB0074
:1049F0009A4269D83E4B4A46984600F03DFB041E59
:104A000011D003003B4D8C334CD080220021120189
:104A10002800FBF794FE200003B03CBC904699466A
:104A2000A246AB46F0BD4346324D1868290000F05F
:104A3000AFFC041EE9D16B6ADB0742D453466B62BC
:104A40000C9B2B6243461B68019301239B462A4B18
:104A50000C9918009A46FFF7A9FE041ED5D1282309
:104A60005B429C46E24453460C9A41465846DA6102
:104A700000F050FA041EC8D143465146186800F0B1
:104A8000C7FC041EC1D143464A463000390000F03D
:104A900077FA041E25D1019B002B18D100F044FBAE
:104AA0000400B2E78022002112012800FBF747FE34
:104AB0000C9B2B6253466B6202239B46002301939F
:104AC000C5E785246442A0E787246442A3E700F099
:104AD0002BFB041E99D101980021FDF705F9040074
:104AE00093E7434600211868FDF7FEF88DE7C046BE
:104AF000309C0008389C0008609C0008F8B5114DF7
:104B00001F002B0000F0B8FA041E01D02000F8BDF1
:104B10000D4E2868310000F03BFC041E06D08022B8
:104B2000002112013000FBF70AFEEFE78022F36953
:104B300012017B60736A0021BB603000FBF7FFFD50
:104B4000E4E7C046309C0008389C0008F8B54746AA
:104B5000CE461B4D80B52B0006000F00904600F09E
:104B60008BFA041E04D020000CBC90469946F8BD78
:104B7000144B28681900994600F00AFC041E05D160
:104B80004B465B6ADB0708D58524644280220021FE
:104B900012014846FBF7D3FDE5E7424630003900F5
:104BA00000F08EFA041EF1D12D6800F0BDFA041E4B
:104BB000ECD128000021FDF797F80400E6E7C04695
:104BC000309C0008389C000810B500F0C5F810BDF6
:104BD000F0B583001A4C5E58A544CA686B460C00B9
:104BE0003100184F1C31DA5105003A006846FBF7D6
:104BF0008AFDF5226946D200300000F0A5FB0028AE
:104C000005D10223641923720F4B9D44F0BD236923
:104C1000002B03D1641901332372F5E76A46D3519F
:104C2000F5226946D200300000F08EFB431E984109
:104C3000012340429843033064192072E4E7C046E0
:104C400054F8FFFFA4070000AC070000F0B5CE4603
:104C50004746002380B53B4C0020A544039300F059
:104C600037FC041E06D02000374B9D440CBC9046F8
:104C70009946F0BD03A9002000F01EFC041EF2D1ED
:104C800000F060FA041EEED1304D039C280000F0C5
:104C9000B7FA290004AE2E4A1C313000B450FBF79D
:104CA00032FDF5223100D200280000F029FB041E5D
:104CB00041D100F08DFA041ED5D1F827254BFF0015
:104CC0009946EB5C3A00581C00949846C1172B009B
:104CD000FCF780FF041EC6D14A46EB5D3100AB54A1
:104CE000434604900120EB55039D00F0E5FB0028AE
:104CF00024D1049B9D4209D9012000F0E9FB041E48
:104D0000B1D1049B013304939D42F5D831000220B8
:104D100000F0D2FB002811D1049B9D4209D902204A
:104D200000F0D6FB041E9ED1049B013304939D42E8
:104D3000F5D8002497E700F04BFA94E78424644206
:104D400091E7C04644F8FFFFBC07000038A4000804
:104D5000A4070000C107000010B500F0A3FB002865
:104D60000DD1F922064CD20000212000FBF7E7FC10
:104D70000123F8222377D200A354FFF767FF10BD69
:104D800038A400080023F0B589B003AC2372637225
:104D9000E3602361F8235E4E02AF6060DB000197A1
:104DA00000960022012000210396FCF73FFF002817
:104DB00001D0012323720197636800220093F82336
:104DC0000220DB000021FCF731FF002801D0012385
:104DD000637200F0B7F9051E02D0280009B0F0BDDB
:104DE00000F060FB051E0BD106A9002000F064FB5B
:104DF000051E05D13900012000F05EFB051E02D022
:104E000000F0E6F9E9E707A9022000F055FB051ECE
:104E1000F6D12369029A934200D02061237A012BB4
:104E200003D021000020FFF7D3FE637A012B03D0CB
:104E300021000120FFF7CCFE00F0CAF9051ECCD1FD
:104E4000039B1B7F012B01D00123237261680B7F21
:104E5000012B01D00123637202232289FF339A427E
:104E600052D0237A012B4CD0637A012B01D0022B34
:104E70003DD0F823802202200021DB005200F252B4
:104E8000FCF732FF051E02D003008C33A5D10023AE
:104E900039000120E468029300F00EFB002833D1B2
:104EA000029B9C420AD9012000F012FB051E00D093
:104EB00093E7029B013302939C42F4D8390002200D
:104EC00000F0FAFA00281FD1029B9C420AD9022066
:104ED00000F0FEFA051E00D07FE7029B013302932B
:104EE0009C42F4D8300000F081F9002575E7F822E3
:104EF0000123D200B3523000FBF705FC0120002152
:104F0000BEE7F822D200F5E784256D4265E7C0468A
:104F100038A4000870B50D0000282CD00024002112
:104F2000164B1A685E6832430CD14A1C01383D2A80
:104F30000ED0203300280DD00C005E6811001A68D6
:104F40003243F2D001313D2901D02033E9E721007D
:104F500000280DD1CC1C20000021FCF7C5FE002844
:104F600002D100202C6070BD03008C33FBD1F8E728
:104F70008E204042F7E787204042F4E768A400080B
:104F8000F0B5454657464E46DE46E0B5984689B0F0
:104F900005000F001600364B002403E001342033D7
:104FA0003D2C49D01A68AA42F8D15A68BA42F5D1C4
:104FB0009A689642F2D12F4B0134994664014C44D1
:104FC000202221006846FBF79EFB236920229B4696
:104FD0006369002120009A46FBF7B1FB43461A683B
:104FE000D31E5B014B441D639E635F634346951E66
:104FF0006D014D44596810222800FBF784FBFFF730
:1050000025FE061E10D05B465246134307D05B4672
:1050100005926946202220000493FBF774FB2022AE
:1050200000212800FBF78BFB300009B03CBC904608
:105030009946A246AB46F0BD43461A680D49D31EB9
:105040005B01CB181D639E635F634346951E6D0134
:105050006D18102259682800FBF755FBFFF7F6FD85
:10506000061EE1D0202200212800FBF768FBDBE7C9
:1050700068A4000838A4000870B50F4C002503E0B0
:10508000013520343D2D14D026688642F8D166685B
:105090008E42F5D1A668B242F2D1EA1C691C074DD6
:1050A00049011A60586849191022FBF72CFB0020AF
:1050B00070BD8C204042FBE768A4000838A40008BB
:1050C00030B5174B89B0002403E0013420333D2C68
:1050D00023D01D688542F8D15D688D42F5D19D6869
:1050E000AA42F2D10F4B013464011C192022210085
:1050F0006846FBF708FB202200212000FBF71FFB7E
:10510000FFF7A4FD051E02D1280009B030BD202202
:1051100069462000FBF7F7FAF6E78C256D42F3E7C6
:1051200068A4000838A4000810B5044A044BD05CF9
:105130000130C117FCF7D8FD10BDC04638A40008E7
:10514000C107000030B58BB00021202202A8FBF778
:10515000F6FA00230093C0239B000493164B01AC86
:105160000593164B16490193802368462383FDF768
:10517000F7FE002801D00BB030BD0C23114A1249B4
:105180006846FDF745FF00280FD1104D69462A00FB
:105190002000FDF771FF002807D16846FDF7B8FD34
:1051A0000028E8D02888FCF74DFE6846FDF7B0FDE2
:1051B00084204042DFE7C046021040060100004064
:1051C000000F00B0E4540010010200000CAC000815
:1051D000054B10B51888FCF735FE002800D110BD2E
:1051E00084204042FBE7C0460CAC0008010010B52B
:1051F00010310C220148FBF786FA10BD00AC000804
:10520000F0B583B06C460E4923000A0060CA60C343
:105210000122009E019F002392197B41009201937D
:105220001A4353425A410B008D681030AD1844CCDC
:1052300044C38D600C22FBF766FA03B0F0BDC04694
:1052400000AC0008F0B51500020089B0109F060000
:105250001148119C008805970F9F029304970E9F99
:10526000019500911032069403970C230B49FDF72A
:1052700087FA051E0CD10F9B21689C4610392160CE
:10528000102261443000FBF73EFA280009B0F0BD5F
:1052900084256D42F9E7C0460CAC000802104006B8
:1052A000F0B5C6460400904600B588B00E9D0F00CC
:1052B0005819102221001E00FBF725FA0E4B220080
:1052C0001888119B10350693109B103205930F9B85
:1052D0000395049343460296019300970C230749D4
:1052E000FDF7A2FA002803D108B004BC9046F0BD37
:1052F00095204042F8E7C0460CAC0008021040067A
:10530000030030B514008BB002000D4809AD0088D1
:105310000695049310250023009103930293103205
:10532000059501940C330749FDF72AFA002804D1AA
:10533000099B102B01D10BB030BD84204042FAE70D
:105340000CAC00080210400630B503008BB015000D
:1053500002000D4809AC00880694002405940494CA
:105360001034029300911032039401950C230749E5
:10537000FDF75AFA002804D1099B002B01D10BB08C
:1053800030BD95204042FAE70CAC00080210400600
:10539000F0B589B005AB01930B0010330093802367
:1053A0000D001B01002200210400FCF73FFC002837
:1053B00001D009B0F0BD059E0694FFF7C3FE00289A
:1053C000F7D134002F00104E0C3C1C37220039005E
:1053D0003000FBF798F907AB03930C4B019702934E
:1053E00000943300042206A92800FFF759FF002883
:1053F00005D1079B9C4202D1FFF7EAFED9E7FFF7F0
:10540000E7FE84204042D4E710AC0008E407000027
:10541000F0B5CE46474680B587B006000C00CD6992
:105420000490FFF78FFE002804D007B00CBC904614
:105430009946F0BD1C232F0098462000FFF7E0FEA0
:1054400005AB0393154B0C370293154BA0449946BB
:10545000019300974346042204A92000FFF7F2FEBF
:10546000002815D1059B9F4212D13A00494640467B
:10547000FBF749F9FFF7ACFE0028D6D123002A003C
:1054800000901033183230000021FCF7A3FBCCE76A
:10549000FFF79EFE84204042C7E7C046F4070000A5
:1054A00010AC000810B529F0F3FA431E984183238D
:1054B0004042984310BDC04610B50A00042129F0AF
:1054C00057FB431E984183234042984310BDC0467A
:1054D00010B529F0B5FB431E984183234042984301
:1054E00010BDC04673746F726167655F6B6579004C
:1054F00000000000000000000000000000000000AC
:10550000F0B5CE46474680B58DB000F0E9F80028EA
:1055100022D106AB81269846644C08AD76428021A4
:10552000012009064042FEF775FFC30616D4830624
:105530006FD4430642D403060FD521008020FEF726
:105540006BFF0028EBD121688B1C00DA94E0002966
:1055500000DB95E000218BE0FEE7FEE72100102054
:10556000FEF75AFF0028DAD121688B1C00DA9CE094
:105570000029EFDB00D098E023696068082B00D099
:105580007BE0A769042F78D1626991462A00FEF773
:1055900045FF082871D13B00424602216068FEF7B2
:1055A0003DFF042869D1069B01934B460093A068F8
:1055B000089A099B00F0C6F8010059E0210040203C
:1055C000FEF72AFF0028AAD121688B1C6CDB00297A
:1055D000C0DB69D123696068082B63D1226A0C2A79
:1055E00060D14246FEF71AFF08285BD1069A079B56
:1055F0000095A06800F094F9071E05D101000C2366
:105600002A006068FEF70CFF39006068FEF70AFFA9
:1056100085E721002020FEF7FFFE002800D07EE76E
:1056200021688B1C2BDB002994DB28D1236960685F
:10563000082B22D16769042F1FD1226A91462A00C4
:10564000FEF7ECFE082818D13B0005AA012160688E
:10565000FEF7E4FE042810D1434602934B46019323
:10566000059B0093A068089A099B00F0F5F80100DB
:105670006068FEF7D7FE52E7FEE73100F8E7FEE785
:105680000029F9D123696068082BF6D12A00FEF7BA
:10569000C5FE0828F1D1089A099BA06800F06EF9B0
:1056A0000100E5E73700AFE7FEE7FEE760C200086C
:1056B00010B50B000349020048680121FEF7AEFE59
:1056C00010BDC04660C2000810B50B0003490200BF
:1056D00048680021FEF7A4FE10BDC04660C2000865
:1056E00010B5002000F07EF9144C0100200000F0FD
:1056F000FDF900280BD0200000F0FEF9002800D0B2
:1057000010BD00F06FF90100200000F0EFF901205A
:1057100000F068F90A4C0100200000F0E7F90028C9
:10572000EED0200000F0E8F90028E9D1013000F0C7
:1057300059F90100200000F0D9F9E1E790C600080E
:10574000A4C60008F0B5DE4657464E464546110051
:10575000E0B5194385B0002900D16DE007210F9C09
:105760008C4366D10393374B0292984602AA01C339
:1057700012CA12C380235B00984257D0324B99461D
:10578000324C41462200484600F02AFA071E42D118
:10579000A368DB0753D44146484600F0B1FA071E20
:1057A0003CD180230E9EDB009E4200D91E00284B78
:1057B00031009A461800FFF77BFF534601930F9B79
:1057C0000E9A009341463300484600F099F9071EAF
:1057D00024D10E9B9C1B03D120E07619641B1DD0A5
:1057E00080232500DB009C4200D91D002900504683
:1057F000FFF75EFF53462A000093414633004846B8
:1058000000F014FA83460028E7D04146484600F0ED
:1058100077FA5F4602E003008C33C2D0380005B04F
:105820003CBC90469946A246AB46F0BD094B994612
:10583000A6E786277F42F1E787277F42EEE78527A5
:105840007F42EBE7B8C6000890C60008C4C600084F
:1058500090C20008A4C60008F0B54E46DE46574682
:1058600045461100E0B585B00E9E19434AD003931A
:10587000264B0292994602AA01C312CA12C3802380
:105880005B0098423BD0224B9A46224C494622006C
:10589000504600F0A5F9071E27D12468B44231D341
:1058A0000F9BA41B9C4228D8109B1C601A4B984647
:1058B0008023DB009B4606E029004046FFF704FFFB
:1058C0007619641B11D025005C4501D98025ED00B7
:1058D00043462A00009349463300504600F096FAAA
:1058E000071EE9D00023109A1360380005B03CBCB5
:1058F00090469946A246AB46F0BD1C00D4E7074B44
:105900009A46C2E787277F42EFE7C046B8C600083D
:1059100090C60008C4C6000890C20008A4C60008CB
:10592000110070B582B0069C19431BD00F4901933A
:105930000B0000926A4601C360CA60C380235B000B
:1059400098420DD00A480B4D2A0000F049F9002872
:1059500004D12B6823606360AB68A36002B070BDA4
:105960000548F0E787204042F8E7C046B8C600087F
:1059700090C60008C4C60008A4C60008110070B58F
:10598000194382B0002922D0124C019323000092C7
:105990006A4601C322CA22C380235B00984211D009
:1059A0000D4E0E4D21002A00300000F019F900289C
:1059B00006D1AB68DB0707D42100300000F0A0F966
:1059C00002B070BD064EECE785204042F8E7872024
:1059D0004042F5E7B8C6000890C60008C4C60008F3
:1059E000A4C6000810B5044B8000C45820002368EA
:1059F0009847200010BDC046B06B0010F0B54E4671
:105A00004546DE465746E0B5C3B04D9D06008B4681
:105A100090469946002D29D080235B009A4610E0DD
:105A20000094434602AA59463000F768B847002858
:105A300015D14C9BA0449C46A44463462D1B4C931B
:105A400014D02C00554501D98024640000944C9B4F
:105A500002AA49463000B768B8470028E0D043B0F2
:105A60003CBC90469946A246AB46F0BD0020F6E706
:105A700010B5040082B01C3001A927F0B9FE618C7A
:105A80000198FDF751FB238DA084002B0AD0638D74
:105A9000002B02D127F0EEFE6085200000F0EAF92D
:105AA00002B010BD27F0CEFE2085F0E710B504004F
:105AB00082B01C3001A927F0F5FE618C0198FDF73A
:105AC00033FB238DA084002B0BD0638D002B03D1DF
:105AD00027F02AFF03306085200000F0CBF902B0E8
:105AE00010BD27F009FF28302085EEE710B50160D2
:105AF00000F05AFB10BDC04610B500F0DFFD10BD30
:105B0000F0B54746CE4680B59946036891B01B8DE7
:105B100004008846170093425FD304AA00F0C8FA35
:105B200000285AD004AB05AE08AD0093029601954B
:105B3000189B3A004146200000F0C4FC002844D1E4
:105B40004B46002B1FD04A460021E86800F0A8FF12
:105B500000283FD1199B2A0001934B463100009346
:105B60002000002300F020FA002833D14B4629689A
:105B700020003768AB6000F095FA2A683060390081
:105B8000200000F0DDFE32000899200000F0DCFE6D
:105B900000281FD12A000499200000F069FF002886
:105BA00018D10499200000F045FA002812D12B6882
:105BB000002B02D14B46002B04D1200000F0B0FB9B
:105BC000002807D1200000F07BFB11B00CBC9046F0
:105BD0009946F0BD84204042F7E787204042F4E731
:105BE00070B58CB0150003AA04000E0000F060FA36
:105BF000002817D1200004AA039900F0D9FB041E45
:105C00000DD10C2209A93000FAF76EFD002809D148
:105C1000079B6B60069B01932B60089BAB60200089
:105C20000CB070BD8C246442F9E7C04670B590B0EA
:105C3000160004AA04001D0000F03AFA00285BD107
:105C400008AA0499200000F0B3FB002854D105AA4B
:105C50000899200000F0FCFB00284AD10A9B03931E
:105C60009D4246D80B9B320029001800039300F098
:105C700017FF00283DD1149B0096019308AA2B0022
:105C800005A9200000F090F9002832D10A9BAD1937
:105C900003939D4226D808992000059D00F002FA42
:105CA000089A05902900200000F04AFE05AA0899EC
:105CB000200000F049FE00281BD108AA049920000A
:105CC00000F0D6FE002814D10499200000F0B2F9AB
:105CD00000280ED1089B002B06D1200000F0F0FA1E
:105CE00010B070BD0A95D6E7200000F019FB00281F
:105CF000F3D084204042F3E78C204042F0E7C046D6
:105D0000F0B54646D6464F46C0B503688EB005AAE4
:105D100005005E8C00F0CCF9002800D070E006AAE7
:105D20000599280000F044FB002805D00EB01CBCEB
:105D300090469946A246F0BD0BA800F0BDFE002893
:105D40005ED1079B20229846099B002106A8069F4A
:105D50009946FAF7F4FC06AA0599280000F088FE97
:105D60000028E3D12B685B8D002B30D0002200246B
:105D700092460BE006AA2100280000F079FE0028D8
:105D8000D4D12B685B8D0134A34222D9059AA2425B
:105D9000F9D006AA2100280000F00AFB0028C5D18E
:105DA000069B0393BB42E5D10BA800F085FE0028BB
:105DB000E0D1079B4345DDD99E4200D91E004A46EB
:105DC0009B1A0793099B9C460393E244D2E7002366
:105DD0009A465346019343464A460093390033009E
:105DE000280000F06BF80028A0D1002F04D0280074
:105DF00000F096FA002806D1280000F061FA95E735
:105E00008C20404292E7842040428FE7F0B58FB06B
:105E1000170005AA04000D001E0000F049F9002833
:105E200025D106AA0599200000F0C2FA00281BD14E
:105E30000C220BA92800FAF757FC002817D1089B61
:105E40003A0031001800039300F02AFE002801D028
:105E50000FB0F0BD149B3200009306A93B00200058
:105E600000F086F80028F3D084204042F0E78C2030
:105E70004042EDE710B5838C012B12D9032B10D0D3
:105E8000418D448C4901022B0DD0008D023B5A00FC
:105E9000D3189B0008315B18A34203DCA0420BD946
:105EA000FEE7FEE7FEE70B00008D1433E31A98428D
:105EB00001DC0123EBE7FEE710BDC046F0B5C646A6
:105EC00000B588B0170005AA05000E00984600F03E
:105ED000BFFA041E04D0200008B004BC9046F0BDF8
:105EE000079B31009C46280067440393079700F006
:105EF000D9F80F9B0700002B23D1069A0E9B05991A
:105F00009A4212D33200280000F01AFD05AA31008F
:105F10002800059700F018FD041E23D1002EDAD0CA
:105F20002868036998470400D5E7981A01900B0088
:105F3000009239002868FFF761FD00280FD105990C
:105F4000E0E7059B010003930F9B0E9A01934346E4
:105F500028680093039BFFF751FD0028CDD08424CF
:105F60006442B8E732003900280000F0E9FCB2E7EB
:105F7000F0B587B00D001400096803AA06001F00E1
:105F800000F066FA00280BD103994B1C08D030684A
:105F90006B680097E3180C9A8468A04707B0F0BDBF
:105FA00084204042FAE7C046F0B54746CE46160088
:105FB00080B50F0083B011681C00050000F072F876
:105FC00073687A689C466444A31A019300928046E1
:105FD00001003B682868FFF711FD00280AD10A9BE1
:105FE00028680093C3680B9A994641462300C84726
:105FF000002804D003B00CBC90469946F0BDF1686F
:1060000073688C4663441A002968B868498C3B68F9
:10601000091A891A0191009241462868FFF7EEFC9F
:106020000028E7D13368002BE4D02868036998473B
:10603000E0E7C046F0B507000569C668006883B0B0
:10604000838C022B20D0023B5A00D21892000832D7
:106050004C010194009233002900FFF7CFFC002887
:1060600010D13F68B98C022919D002394B00591858
:10607000890022007B8D28325B01083352185B189F
:10608000934203D803B0F0BD1422E1E79B1A0193B9
:106090000092330029003800FFF7B0FCF2E70C2132
:1060A000E7E7C046002901D0406870470069FCE777
:1060B000F0B545464E46DE465746E0B50500006859
:1060C0008DB0438D89469046002B67D00024202652
:1060D00042E02B68049A9B8C022B5AD0023B9A42D6
:1060E0004BD209A800F0E8FC002829D12868079ABB
:1060F000038D9A4241D8069B03939A423DD3049B59
:1061000005990393002B16D1438D9B46838C9A46A9
:10611000022B40D002235B429C46E24453465B0084
:106120009C46D44463469B009C465B465B01083317
:106130006344994221D3408C00F0B2FC00281CD16A
:106140000C22494609A8FAF7CFFA002829D0286876
:106150000134438DA34221D9818C022917D0023901
:106160004B00591889006301009608335B18876853
:1061700004AAE968B847071EABD084277F423800DD
:106180000DB03CBC90469946A246AB46F0BD0C21F2
:10619000E9E70123A3E70C239C46C6E78C277F424F
:1061A000EDE743461C60EAE7F0B50400006887B0FD
:1061B00043689847002801D007B0F0BD0825206843
:1061C00000958668002302AA0021B047002817D056
:1061D00020688668082304AA009301210023B047A1
:1061E00000280AD16B461B7D012B06D16B465A7DD8
:1061F0002C232068C35C9A4239D184204042DBE7DB
:106200006B4620681B7B8668012BE3D16B462C27ED
:106210005A7BC35D9A42DDD00095002304AA012178
:10622000B047002826D001230021206823610823DD
:106230000093E160221D85680023A8470028DCD177
:10624000237A012BD9D120682B33627AC35C9A421E
:10625000D3D04369216998470028ADD123689A8C2F
:10626000022AA9D961685A6918009047A4E7002357
:106270000121DBE76B46197D012904D02368180052
:1062800000210123D2E76B4620685A7DC55D0300DB
:106290009542F4D06B465D7B002A09D10023012D85
:1062A000C4D1954289410023494295425B41BDE7F3
:1062B000002DF6D1531E594259415A1E9341B5E75C
:1062C0002C2230B5437A04000133DBB243720068FC
:1062D00083B0825C9A4201D1002363720823009349
:1062E000221DC56800232169A847002804D1206821
:1062F00003699847002801D003B030BD2369E168E5
:106300002068E3602161436998470028F4D123683D
:106310009A8C022AF0D961685A6918009047EBE715
:106320000C2330B5040089B0006800938568043BF5
:1063300005AAE168A847002823D1236805999A8C0B
:10634000914230D2079A0292069A0392588C029A8E
:10635000039900F0A5FB002825D1059B002202939C
:10636000012B10D9069B029393421CD12068E3684D
:106370002169448C079DA41A641B01940092FFF7C5
:106380003DFB09B030BD2368998C5A8D02290DD090
:1063900002394B005B189B0052010832D218069B51
:1063A00002939342E2D098204042EAE70C23F3E7BD
:1063B00070B5050000681400828C82B0022A3ED0BD
:1063C000023A53009A18920049010B0008339B18B7
:1063D0002022009286682200E968B047061E2BD171
:1063E0002B6822689B8C022B2BD0023B9A422CD22A
:1063F0002000143000F060FB00281DD12868E268FE
:10640000038D9A4221D8A3689A421ED323686168FB
:10641000002B0CD1848C438D022C14D0023C6500DF
:106420002C19A4005B0108331B198B420DD8408C3A
:1064300000F036FB002808D1300002B070BD0C22FD
:10644000C2E70123D2E70C24ECE798267642F3E773
:1064500070B514000C2205004B0082B000685B1878
:1064600000929B00083386682200E968B047002844
:1064700012D12B6821689A8C91421ED2588CA26846
:10648000616800F00DFB002817D122680023012A63
:1064900004D962689A4210D102B070BD2A68918C0A
:1064A000538D02290CD002394A00521892005B0128
:1064B00008339B1862689A42EED098204042EBE77E
:1064C0000C22F4E7F0B557464E46DE464546E0B5A9
:1064D0008DB00393169B04009B460C2302919146BA
:1064E000189D0068082700269A461DE020682A6843
:1064F000838C9A4200D3B0E0AA68408C696800F0AF
:10650000CFFA021E206800D0A7E0296800230129E5
:1065100000D892E06968994200D09EE0AB680C37E1
:10652000994500D8A2E00136838C022B00D178E097
:10653000023B9E4200D378E05346009383682A00D2
:106540009846E1683B00C0470028CFD084235B42D7
:1065500098462068438D002B55D00825002620271B
:1065600041E02368049A9B8C022B64D0023B9A4240
:1065700049D209A800F0A0FA002829D12068079A7A
:10658000038D9A423FD8069B02939A423BD3049BC9
:1065900005990293002B16D1438D9A46838C994618
:1065A000022B60D002235B429C46E1444B465B00D9
:1065B0009C46CC4463469B009C4653465B01083393
:1065C00063448B421FD8408C00F06AFA00281AD12D
:1065D00009A800F071FA002864D120680136438DC3
:1065E00020359E420FD2828C022A22D0023A5300DA
:1065F0009B189B0000978268EB189146E16804AAFB
:10660000C8470028ADD05A462B4B13608E235B42FF
:10661000984640460DB03CBC90469946A246AB46D3
:10662000F0BD01239E4200D286E78E235B4298464E
:1066300090E70C23DEE7012399E7818C438D022943
:106640000FD002398C464900614489005B01083350
:106650005B186968994200D160E784235B429846E1
:1066600078E70C21F2E70C239C46A6E79046179AA0
:1066700002991660428CD31A179A536013004A4647
:106680001800DA6014300C22FAF73DF80023179A4C
:10669000206893601300039A1A614A46AB689B1AFC
:1066A000AB6057E75B461E604346002BAED1024B02
:1066B0009E42AED1AAE7C046FFFF0000F0B54E46AD
:1066C0004546DE465746E0B508258FB00400006811
:1066D00000958668002303AA0021B047002800D057
:1066E000E3E06B4620681B7C8668012B00D1DFE06D
:1066F00006AB994608234A46009301210023B04780
:10670000002800D0F3E04B461B79012B00D0EEE0CF
:106710004B462C2221685B798A5C9A4200D1E6E0E4
:1067200000250122E260256120682900436998471D
:10673000071E00D0B1E0012629002068714043699E
:106740009847071E00D0A8E060722068838C428DB5
:10675000022B00D1C5E002216160991E4B0059183F
:1067600026722661E76089005201130008335B1826
:106770000493428C0121D31A0593002303930C3315
:106780000093C568043B03AAA847071E00D084E015
:10679000256804906B8C0593AE8C022E00D19AE094
:1067A00003239846032E13D06B692800414698476F
:1067B00025680743AE8C022E07D043469A1E01235C
:1067C0009C46F31EE0449A42EED3002F00D090E0A6
:1067D00014239A46083B00279B4615E0F31E9F4270
:1067E00016D2FB1C03935B460093EE68534603AA44
:1067F00041462800B0470C239C460137E24400285C
:1068000000D06BE02568AE8C23699846022EE5D156
:10681000202200214846F9F792FF6B8D002B1FD0F4
:10682000202300279A4617E0023E73009E19B60007
:1068300052467B01009208339B194A46EE68414656
:106840002800B047002849D12369256898466B8DF8
:106850000137BB4204D9AE8C022EE5D10C26E7E706
:106860002C22637A0133DBB26372AA5C9A4201D1B3
:106870000023637208230093221DEE680023414623
:106880002800B047002829D1206803699847071ECF
:1068900003D12369E268E360226138000FB03CBC99
:1068A00090469946A246AB46F0BD206886681FE731
:1068B0006B462C275A7CC35D9A4200D118E706AB81
:1068C0009946009500234A460121B047002813D07D
:1068D0000125002226E72369984699E784277F420D
:1068E000DBE7666026722661E7600C213CE7002545
:1068F0001AE792277F42D0E74B461A79012AE7D15F
:1069000021685B79C95D994216D06946487C002BA5
:106910000AD10025012800D004E7984292410025C1
:10692000524298426D41FDE60028F6D15D1E6A4252
:106930006A416B1E9D41F5E615000022F2E6C04655
:10694000002A00D041607047F0B5CE4647460400AB
:1069500080B500680D0089B02169C668002D23D17B
:106960000C23116021690093043BB04700286AD1D1
:106970002769E66820686B1C5D00ED18AD002A00F1
:10698000818C0832022961D002394B005B189B00D0
:106990005D1B0195009233003900FFF72FF809B015
:1069A0000CBC90469946F0BD0C276B005B199B0010
:1069B000984600970833B946B047002843D14B4664
:1069C000206800938368E668994605AA0823310089
:1069D0002769C847002836D1236805999A8C9142C7
:1069E00031D2079A0292069A0392588C029A03991E
:1069F00000F056F8002826D1059B0293029A002346
:106A0000012A25D9069A02929A421CD10C232068A9
:106A10000093C3680597994605AA08232169C847CA
:106A2000002810D12068012DA5D943460C3B0193C5
:106A300014231422009339003300FEF7DFFF0028EF
:106A4000ADD1206897E784204042A8E70C239FE758
:106A50002268538D928C022A07D0023A51008A187C
:106A600092005B0108339B18CCE70C22F9E7C04683
:106A700030B50500006883B0848C022C0ED0023C37
:106A800063001C19A40049010B0008331B192024C2
:106A900000942969C468A04703B030BD0C24F2E714
:106AA000814205D8401A904280418623984370471E
:106AB00087204042FBE7C0460378002B24D143786F
:106AC000002B21D18378002B1ED1C378002B1BD142
:106AD0000379002B18D14379002B15D18379002B32
:106AE00012D1C379002B0FD1037A002B0CD1437A3A
:106AF000002B09D1837A002B06D1C07A434258413A
:106B00008B234042984300E000207047836910B512
:106B10009B6800209847431E984191234042984328
:106B200010BDC04610B50C001100428C5443C26920
:106B3000944682696344E31818005469029AA04796
:106B4000431E984191234042984310BD10B50C005C
:106B50001100428C5443C269944682696344E3182D
:106B600018009469029AA047431E9841912340421D
:106B7000984310BD0020704770B50400408C0E0093
:106B8000002813D0002504E0238C608CED18A84267
:106B90000CD9E36970439C46A36960444019DB69E2
:106BA00098470028F0D09220404200E0002070BDBD
:106BB00000C2000830C20008000000000000000011
:106BC000024A034BD358036000207047C04D0108B0
:106BD00004140000F0B5DE4657464E464546E0B583
:106BE000A9B000F00DF9002806D029B03CBC9046B1
:106BF0009946A246AB46F0BD80217D48090202F0CD
:106C000047FA07F055FD002875D105F0F3FC002880
:106C1000EBD112AB1800282200219846F9F78FFD1E
:106C200001235B429B46734C0AAD8021012009067B
:106C30004042FDF7EFFB102318425AD01CA9180060
:106C4000FDF7EAFB002855D11C998B1C56DB002967
:106C500055DB53D1282342461D98FDF7DFFB28283A
:106C600059D05B4601334FD02022002102A8F9F70A
:106C700066FD202200212800F9F761FD042701E0CC
:106C8000171E41D01CA98C467A1E930063441B69D1
:106C9000002BF5D0434602932823039321AB99465A
:106CA000A0235B0101269A46BE423FD24B460321F8
:106CB0001B685046DA1C8A4351466158401A82428A
:106CC0005DD81D985218019060185146009062508E
:106CD000020031000198FDF7A1FB02AA4946944643
:106CE0000098F300D05004C9634489465A600136C5
:106CF000DAE7FEE7FEE79320404276E7FEE7010091
:106D00001D98FDF78FFB90E784277F4239001D987F
:106D1000FDF788FB89E743461B689B463F2BA3D9B9
:106D2000012384275B429B467F42EFE7042101E079
:106D3000111E33D01CA884464A1E930063441E6A69
:106D4000002EF5D0A0267601A2590023B146009767
:106D50008C4608E0A7181218D8002F5001332818C5
:106D60004160634517D01CA882460327990051440F
:106D7000096AC81CB8434F46BF1AB842EAD9A022D4
:106D800000218D271C4B52012000A150E1507F4271
:106D9000F9F7D5FCBAE7A2511E00009F1E9B3900EF
:106DA0000093009A144B02A8E2505B46134A9B00E2
:106DB000D3582A0099463300C8470023B14607003C
:106DC0001E004E4509D0F200AB1831005B68AA588E
:106DD0001D98FDF725FB0136F3E7A0220021064BA5
:106DE00052012000A150E150F9F7A9FC8EE7C046FE
:106DF000C0CD0008C04D010804140000DCE60110FD
:106E0000892210B5520100210248F9F798FC0020B0
:106E100010BDC046C86101080023F0B583B006006C
:106E200001A80D0014000193FFF7CAFE00282AD123
:106E30002B68002B58D1002C59D02E4B206019689C
:106E4000002922D0892292009A58002A30D0892223
:106E5000D2009A58002A2FD0274A9A58002A2FD0B9
:106E6000892212019A58002A2ED0244A9A58002AC0
:106E70002ED0234A9A58002A2ED0224A9A58002A05
:106E80002ED08520404203B0F0BD012294460A0175
:106E90005218D200521801219200019F995099185E
:106EA0004F608E6061460C329B1829602360EAE7D0
:106EB000022201219446EAE7032202219446E6E7F2
:106EC000042203219446E2E7052204219446DEE7EA
:106ED000062205219446DAE7072206219446D6E7E2
:106EE000083207219446D2E789204042CBE7872029
:106EF0004042C8E7C86101086C060000B40A0000FF
:106F0000D80C0000FC0E0000F0B5C646002300B50A
:106F100082B00568804601A80193FFF751FE071E65
:106F200028D1013D072D2AD82C016019C000154E2B
:106F3000401980003358012B21D133185A68019928
:106F40008A421CD19B680C30013B30180022032B75
:106F500002D80D4A9B009A580021F9F7F0FB002354
:106F600042466419E4006519AD0073517519AB60B0
:106F70006B601360380002B004BC9046F0BD8727F8
:106F80007F42F7E7C8610108DCE70110002370B514
:106F900082B0050001A80E0014000193FFF710FE57
:106FA000002816D1013E072E15D831018919C900D4
:106FB0000A4A891989008B58012B0CD153189E68F5
:106FC000AE4208D15B68019DAB4204D10C318918F7
:106FD000216002B070BD89204042FAE7C861010813
:106FE000F0B5CE4647461400002280B583B001922A
:106FF00001292AD1022B28D14368282B25D1636887
:10700000042B22D103682768DE68A36801AA98468A
:10701000E36831003E6001209946FFF7B7FF051E87
:1070200005D0280003B00CBC90469946F0BD230063
:107030003E600C334A464146019804F055FB051E5C
:10704000EFD03800FFF760FFEBE782256D42E8E7FD
:10705000F0B5002483B00194022921D1012B1FD166
:107060004368282B1CD15368042B19D10368156879
:10707000D9688668C76801AA29600120FFF786FFE2
:10708000041E02D0200003B0F0BD3A003100019888
:1070900004F008FB041EF5D02800FFF735FFF1E7E8
:1070A00082246442EEE7C046F0B5002483B0009429
:1070B00001292AD1012B28D15368042B25D14368FB
:1070C000282B22D103681668D9689F680191DD8852
:1070D0000021280000F068FB041E02D0200003B04D
:1070E000F0BD6A4601A90120FFF796FE041EF5D106
:1070F000019B3A0033602900009804F0C9FA041E8D
:10710000ECD03000FFF700FFE8E782246442E5E7B7
:10711000F0B5002483B0009401292AD1012B28D195
:107120005368042B25D14368282B22D103681668A5
:10713000D9689F680191DD880021280000F034FBA8
:10714000041E02D0200003B0F0BD6A4601A9012050
:10715000FFF762FE041EF5D1019B3A00336029005F
:10716000009804F09AFA041EECD03000FFF7CCFE31
:10717000E8E782246442E5E7F0B5D6464F46464646
:1071800014000022C0B584B00392022930D1022B32
:107190002ED14368282B2BD16368042B28D1036898
:1071A0002668D968C36887689846A368012099460D
:1071B000E3683160E26003AA9A46FFF7E7FE051E26
:1071C00006D0280004B01CBC90469946A246F0BDEB
:1071D00053460C34009301944B46424639000398C1
:1071E00004F0AEFA051EECD03000FFF78DFEE8E7A4
:1071F00082256D42E5E7C046F0B5C6461400002280
:1072000000B582B0019201292CD1022B2AD143680A
:10721000282B27D16368042B24D103682668D968FA
:10722000E368A76801203160E26001AA9846FFF791
:10723000ADFE051E04D0280002B004BC9046F0BD8F
:10724000230042460C333900019804F0ADFA0500E2
:107250003000002D03D1FFF757FE0500EBE7FFF7E5
:1072600053FEE8E782256D42E5E7C04630B50024CD
:1072700083B00194012922D1012B20D14368282B0E
:107280001DD15368042B1AD103681568D96801AA67
:1072900029600120FFF77AFE002802D0200003B009
:1072A00030BD019804F01EF904002800002C03D121
:1072B000FFF72AFE0400F1E7FFF726FEEEE782243F
:1072C0006442EBE7862040427047C0468620404239
:1072D0007047C04670B5002482B00094012923D1C4
:1072E000012B21D15368042B1ED14368282B1BD1BD
:1072F00001681568CB688E6801936A462B6001A906
:107300000320FFF789FD041E02D0200002B070BDEB
:10731000019B31002B60009803F0A6F9041EF4D005
:107320002800FFF7F1FDF0E782246442EDE7C04654
:10733000F0B5002483B00194022921D1012B1FD183
:107340004368282B1CD15368042B19D10368156896
:10735000D9688668C76801AA29600320FFF716FE6E
:10736000041E02D0200003B0F0BD3A0031000198A5
:1073700003F0BCF9041EF5D02800FFF7C5FDF1E7C6
:1073800082246442EEE7C046F0B5C64614000022EF
:1073900000B582B0019201292CD1022B2AD1436879
:1073A000282B27D16368042B24D103682668D96869
:1073B000E368A76803203160E26001AA9846FFF7FE
:1073C000E5FD051E04D0280002B004BC9046F0BDC7
:1073D000230042460C333900019803F091F905006F
:1073E0003000002D03D1FFF78FFD0500EBE7FFF71D
:1073F0008BFDE8E782256D42E5E7C046F0B5002445
:1074000083B00194022926D1012B24D14368282B73
:1074100021D15368042B1ED103681568D96886688A
:10742000C76801AA29600320FFF7B0FD041E02D03F
:10743000200003B0F0BD3A003100019803F0B2FB28
:1074400004002800002C03D1FFF75EFD0400EFE7E5
:10745000FFF75AFDECE782246442E9E730B50024E7
:1074600083B00194012922D1012B20D14368282B1C
:107470001DD15368042B1AD103681568D96801AA75
:1074800029600320FFF782FD002802D0200003B00E
:1074900030BD019803F09AF804002800002C03D1B5
:1074A000FFF732FD0400F1E7FFF72EFDEEE782243F
:1074B0006442EBE730B5002483B0009401940129C5
:1074C00024D1012B22D14368282B1FD15368042BD0
:1074D0001CD103681568D9686A460320FFF756FD7A
:1074E000041E02D0200003B030BD01AA29000320F1
:1074F000FFF792FC041EF5D10199009803F072FB8E
:10750000041EEFD02800FFF7FFFCEBE78224644263
:10751000E8E7C046862040427047C0468620404289
:107520007047C046F0B5C646002400B582B000944E
:1075300001292FD1012B2DD15368042B2AD1436867
:10754000282B27D105680021EB6817680193EE8886
:10755000AB683000984600F027F9041E04D02000E4
:1075600002B004BC9046F0BDEB686A463B6001A9DE
:107570000220FFF751FC041EF1D1019B42463B6003
:107580003100009803F078FC041EE8D03800FFF7C3
:10759000BBFCE4E782246442E1E7C046F0B5C6469E
:1075A000002400B582B0009401292FD1012B2DD1E8
:1075B0005368042B2AD14368282B27D10568002162
:1075C000EB6817680193EE88AB683000984600F0CE
:1075D000EBF8041E04D0200002B004BC9046F0BDBD
:1075E000EB686A463B6001A90220FFF715FC041E08
:1075F000F1D1019B42463B603100009803F041FC11
:10760000041EE8D03800FFF77FFCE4E782246442E0
:10761000E1E7C046F0B5002483B00194022921D1EE
:10762000012B1FD14368282B1CD15368042B19D17F
:1076300003681568D9688668C76801AA29600220AE
:10764000FFF7A4FC041E02D0200003B0F0BD3A00F6
:107650003100019803F01AFC041EF5D02800FFF752
:1076600053FCF1E782246442EEE7C046F0B5C6461B
:107670001400002200B582B0019201292CD1022B06
:107680002AD14368282B27D16368042B24D10368AF
:107690002668D968E368A76802203160E26001AA21
:1076A0009846FFF773FC051E04D0280002B004BC06
:1076B0009046F0BD230042460C333900019803F098
:1076C00015FC05003000002D03D1FFF71DFC05005F
:1076D000EBE7FFF719FCE8E782256D42E5E7C046D6
:1076E000F0B5002483B00194022926D1012B24D1C6
:1076F0004368282B21D15368042B1ED103681568D9
:10770000D9688668C76801AA29600220FFF73EFC95
:10771000041E02D0200003B0F0BD3A0031000198F1
:1077200003F013FC04002800002C03D1FFF7ECFB4E
:107730000400EFE7FFF7E8FBECE782246442E9E7A7
:1077400030B5002483B00194012922D1012B20D12E
:107750004368282B1DD15368042B1AD10368156880
:10776000D96801AA29600220FFF710FC002802D086
:10777000200003B030BD019803F05EFA0400280039
:10778000002C03D1FFF7C0FB0400F1E7FFF7BCFBBF
:10779000EEE782246442EBE7862040427047C04611
:1077A000862040427047C046002330B583B00400B5
:1077B00001A80D000193FFF703FA002800D07AE03A
:1077C000554B9A79002A03D09A88A24200D17AE0D8
:1077D0009A7B002A03D09A89A24200D17DE09A7D4B
:1077E000002A00D069E09A7F002A03D09A8BA24237
:1077F00000D186E026229A5C002A03D09A8CA2420D
:1078000000D180E02E229A5C002A03D09A8DA242F9
:1078100000D17AE036229A5C002A03D09A8EA242E6
:1078200000D174E03E229A5C002A02D09A8FA242D4
:1078300055D046229A5C002A03D044229A5AA2428A
:107840004FD04E229A5C002A03D04C229A5AA24270
:1078500049D056229A5C002A03D054229A5AA24256
:1078600043D05E229A5C002A03D05C229A5AA2423C
:107870003DD066229A5C002A03D064229A5AA24222
:1078800037D06E229A5C002A03D06C229A5AA24208
:1078900031D076229A5C002A03D074229A5AA242EE
:1078A0002BD07E229A5C002A03D07C229A5AA242D4
:1078B00025D08820404203B030BD9A8AA24200D031
:1078C00091E7022200E00022D1005B5801998B422F
:1078D0001FD1002DEFD02A60EDE70122F4E7072247
:1078E000F2E70822F0E70922EEE70A22ECE70B2292
:1078F000EAE70C22E8E70D22E6E70E22E4E70F2292
:10790000E2E70322E0E70422DEE70522DCE70622C5
:10791000DAE785204042CEE7E8720108304B9A79D9
:10792000002A3BD09A7B002A3CD09A7D002A3BD08B
:107930009A7F002A3AD026229A5C002A38D02E223A
:107940009A5C002A36D036229A5C002A36D03E2233
:107950009A5C002A34D046229A5C002A2CD04E220F
:107960009A5C002A2ED056229A5C002A2CD05E22E5
:107970009A5C002A2AD066229A5C002A28D06E22BD
:107980009A5C002A26D076229A5C002A24D07E2295
:107990009B5C002B22D08D20404270470023036067
:1079A0000020FAE70123FAE70223F8E70323F6E7CA
:1079B0000423F4E70523F2E70823F0E70623EEE7C4
:1079C0000723ECE70923EAE70A23E8E70B23E6E7C6
:1079D0000C23E4E70D23E2E70E23E0E70F33DEE7B5
:1079E000E872010830B583B0040001A80D00FFF76C
:1079F000E7F8002807D1054B019AE400E250012284
:107A00001B199D809A7103B030BDC046E872010811
:107A10000023F0B58BB0242206000F0001A800213E
:107A20000093F8F78CFE6846FFF7CAF8051E00D0F1
:107A300089E0B64CA379002B04D0009B22689342C6
:107A400000D193E0A37B002B04D0A368009A93425B
:107A500000D198E0A37D002B04D02369009A9342C3
:107A600000D19DE0A37F002B04D0A369009A93422C
:107A700000D1A2E02623E35C002B04D0236A009A05
:107A8000934200D1E1E02E23E35C002B04D0A36AF3
:107A9000009A934200D1CBE03623E35C002B04D064
:107AA000236B009A934200D1A8E03E23E35C002BB5
:107AB00004D0A36B009A934200D1ACE04623E35C70
:107AC000002B04D0236C009A934200D188E04E230F
:107AD000E35C002B04D0A36C009A934200D1C1E078
:107AE0005623E35C002B04D0236D009A934200D10F
:107AF000C6E05E23E35C002B04D0A36D009A9342A2
:107B000000D1CBE06623E35C002B04D0236E009A07
:107B1000934200D1D0E06E23E35C002B04D0A36E2F
:107B2000009A934200D1D5E07623E35C002B04D089
:107B3000236F009A934200D1DAE07E23E35C002BAE
:107B400004D18C256D4228000BB0F0BDA36F009AC4
:107B50009342F6D17C2301A9E05A02F0A3FB00284E
:107B6000EFD1039B9E42ECD10F2332E0A08801A904
:107B700002F098FB002800D064E7039B9E4200D0EF
:107B800060E7002325E0A08901A902F08BFB002813
:107B900000D05FE7039B9E4200D05BE7012318E023
:107BA000A08A01A902F07EFB002800D05AE7039BBF
:107BB0009E4200D056E702230BE0A08B01A902F001
:107BC00071FB002800D055E7039B9E4200D051E78F
:107BD0000323002FB7D0DB00E418A3883B80B2E773
:107BE000442301A9E05A02F05DFB002800D06EE7B3
:107BF000039B9E4200D06AE70823EAE7A08E01A912
:107C000002F050FB002800D04FE7039B9E4200D0BB
:107C10004BE70623DDE7A08F01A902F043FB002814
:107C200000D04BE7039B9E4200D047E70723D0E7F5
:107C3000A08D01A902F036FB002800D02CE7039BA1
:107C40009E4200D028E70523C3E7A08C01A902F0DB
:107C500029FB002800D016E7039B9E4200D012E7C4
:107C60000423B6E74C2301A9E05A02F01BFB0028CD
:107C700000D035E7039B9E4200D031E70923A8E7F7
:107C8000542301A9E05A02F00DFB002800D030E790
:107C9000039B9E4200D02CE70A239AE75C2301A9AC
:107CA000E05A02F0FFFA002800D02BE7039B9E4227
:107CB00000D027E70B238CE7642301A9E05A02F0E8
:107CC000F1FA002800D026E7039B9E4200D022E76D
:107CD0000C237EE76C2301A9E05A02F0E3FA0028A6
:107CE00000D021E7039B9E4200D01DE70D2370E7E3
:107CF000742301A9E05A02F0D5FA002800D01CE74D
:107D0000039B9E4200D018E70E2362E7E872010849
:107D1000862040427047C046862040427047C04699
:107D2000F0B5CE46474680B583B0032955D1012B27
:107D300053D14368282B50D1C368242B4DD15368AD
:107D4000022B4AD113684A4C984600230193A37929
:107D5000856806694769002B42D0A37B002B59D068
:107D6000A37D002B59D0A37F002B5CD02623E35C9E
:107D7000002B5BD02E23E35C002B5AD03623E35C30
:107D8000002B4DD03E23E35C002B55D04623E35C13
:107D9000002B54D04E23E35C002B53D05623E35CDE
:107DA000002B52D05E23E35C002B51D06623E35CB2
:107DB000002B50D06E23E35C002B4FD07623E35C86
:107DC000002B4ED07E23E35C002B4DD08D20404213
:107DD00003B00CBC90469946F0BD82204042F7E7C4
:107DE0000023994601A8FEF7EBFE0028F0D1434698
:107DF0003A003100280002F0EAFA0028E8D14B46A8
:107E0000019ADB00E250E41843461B88A38001235B
:107E1000A371DDE701239946E4E702239946E1E7F0
:107E200006239946DEE703239946DBE704239946B8
:107E3000D8E705239946D5E707239946D2E70823D3
:107E40009946CFE709239946CCE70A239946C9E723
:107E50000B239946C6E70C239946C3E70D239946A1
:107E6000C0E70E239946BDE70F239946BAE7C046FF
:107E7000E872010810B5022916D1012B14D143680C
:107E8000282B11D1C368042B0ED15368022B0BD1C0
:107E9000836811681868C0231B06C218054B9A42F4
:107EA00005D800F05DFB10BD82204042FBE7862034
:107EB0004042F8E7FFFFFF3F70B582B0012900D0D4
:107EC000A3E0002B00D0A0E04268282A00D09CE06C
:107ED000026801A8D5880193FEF772FE002800D041
:107EE0007EE0594CA379002B03D0A388AB4200D18C
:107EF000A4E0A37B002B03D0A389AB4200D19FE079
:107F0000A37D002B03D0A38AAB4200D19AE0A37FCC
:107F1000002B03D0A38BAB4200D179E02623E35C96
:107F2000002B03D0A38CAB4200D173E02E23E35C83
:107F3000002B03D0A38DAB4200D16DE03623E35C70
:107F4000002B03D0A38EAB4200D167E03E23E35C5D
:107F5000002B02D0A38FAB4262D04623E35C002B00
:107F600003D04423E35AAB425CD04E23E35C002BA6
:107F700003D04C23E35AAB4256D05623E35C002B8C
:107F800003D05423E35AAB4250D05E23E35C002B72
:107F900003D05C23E35AAB424AD06623E35C002B58
:107FA00003D06423E35AAB4244D06E23E35C002B3E
:107FB00003D06C23E35AAB423ED07623E35C002B24
:107FC00003D07423E35AAB420CD07E23E35C002B36
:107FD00004D07C23E35A0F26AB4204D088204042D1
:107FE00002B070BD0E268520F600A359019A4042CA
:107FF0009342F5D1280004F0B8FB0028F0D100230B
:10800000A051A419A080A371EAE782204042E7E7CB
:108010000326E8E70426E6E70526E4E70626E2E786
:108020000726E0E70826DEE70926DCE70A26DAE786
:108030000B26D8E70C26D6E70D26D4E70026D2E794
:108040000126D0E70226CEE7E872010870B582B0BB
:10805000012900D0A3E0002B00D0A0E04268282A2C
:1080600000D09CE0026801A8D5880193FEF7A8FD26
:10807000002800D07EE0594CA379002B03D0A388C0
:10808000AB4200D1A4E0A37B002B03D0A389AB4279
:1080900000D19FE0A37D002B03D0A38AAB4200D187
:1080A0009AE0A37F002B03D0A38BAB4200D179E0F1
:1080B0002623E35C002B03D0A38CAB4200D173E0FA
:1080C0002E23E35C002B03D0A38DAB4200D16DE0E7
:1080D0003623E35C002B03D0A38EAB4200D167E0D4
:1080E0003E23E35C002B02D0A38FAB4262D0462339
:1080F000E35C002B03D04423E35AAB425CD04E2315
:10810000E35C002B03D04C23E35AAB4256D05623FA
:10811000E35C002B03D05423E35AAB4250D05E23E0
:10812000E35C002B03D05C23E35AAB424AD06623C6
:10813000E35C002B03D06423E35AAB4244D06E23AC
:10814000E35C002B03D06C23E35AAB423ED0762392
:10815000E35C002B03D07423E35AAB420CD07E23A4
:10816000E35C002B04D07C23E35A0F26AB4204D0FF
:108170008820404202B070BD0E268520F600A3592B
:10818000019A40429342F5D1280002F051F80028AC
:10819000F0D10023A051A419A080A371EAE78220A6
:1081A0004042E7E70326E8E70426E6E70526E4E79A
:1081B0000626E2E70726E0E70826DEE70926DCE7F1
:1081C0000A26DAE70B26D8E70C26D6E70D26D4E7F1
:1081D0000026D2E70126D0E70226CEE7E8720108A2
:1081E00010B501290DD1012B0BD14368282B08D1E3
:1081F0005368242B05D103681168D88802F052F81F
:1082000010BD82204042FBE710B501290CD1012BA3
:108210000AD14368282B07D15368242B04D1106856
:1082200002F015F8002010BD82204042FBE7C04656
:1082300010B501290CD1012B0AD14368282B07D195
:10824000131D12CA0268D088220002F095F810BDF2
:1082500082204042FBE7C046F0B5140083B00129FC
:108260001AD1012B18D14368282B15D1036801A915
:10827000DD8816682800576800F052F9231D3A007F
:108280003100002804D1280002F08BF803B0F0BDC3
:10829000019800F0D5F9F9E782204042F6E7C046A0
:1082A000F0B5C64600B582B0022954D1012B52D197
:1082B0004368282B4FD15368022B4CD1C368242B21
:1082C00049D103683F4CDE888368176898460023CD
:1082D0000193A379002B41D0A37B002B54D0A37D25
:1082E000002B53D0A37F002B54D02623E35C002B1C
:1082F00052D02E23E35C002B50D03623E35C002BBE
:1083000046D03E23E35C002B4AD04623E35C002B9F
:1083100048D04E23E35C002B46D05623E35C002B71
:1083200044D05E23E35C002B42D06623E35C002B49
:1083300040D06E23E35C002B3ED07623E35C002B21
:108340003CD07E23E35C002B3AD08D20404202B02B
:1083500004BC9046F0BD82204042F8E7002501A809
:10836000FEF72EFC0028F2D13A004146300002F020
:1083700059F80028EBD1019BED0063513B8864194B
:10838000A3800123A371E2E70125E8E70225E6E7E0
:108390000625E4E70325E2E70425E0E70525DEE717
:1083A0000725DCE70825DAE70925D8E70A25D6E717
:1083B0000B25D4E70C25D2E70D25D0E70E25CEE717
:1083C0000F25CCE7E8720108F0B583B002294FD140
:1083D000012B4DD14368282B4AD1C368242B47D1A8
:1083E0005368022B44D100233C4C0193A3791668B7
:1083F0008768002B3FD0A37B002B51D0A37D002B9F
:1084000050D0A37F002B51D02623E35C002B4FD00C
:108410002E23E35C002B4DD03623E35C002B43D0AE
:108420003E23E35C002B47D04623E35C002B45D082
:108430004E23E35C002B43D05623E35C002B41D05A
:108440005E23E35C002B3FD06623E35C002B3DD032
:108450006E23E35C002B3BD07623E35C002B39D00A
:108460007E23E35C002B37D08D20404203B0F0BD6B
:1084700082204042FAE7002501A8FEF7A1FB002870
:10848000F4D13100380003F0DFFF0028EED1019B6A
:10849000ED00635133886419A3800123A371E5E7DC
:1084A0000125E9E70225E7E70625E5E70325E3E7F8
:1084B0000425E1E70525DFE70725DDE70825DBE7FC
:1084C0000925D9E70A25D7E70B25D5E70C25D3E7FA
:1084D0000D25D1E70E25CFE70F25CDE7E87201087E
:1084E00030B504008BB00D002422002101A8F8F75C
:1084F00026F901A9200001F0D5FE002808D0074C7C
:10850000002D00D02C60200026F03AF90BB030BDD1
:1085100001A8039C01F09BFEF2E7C046FFFFFF7F2E
:1085200030B504008BB00D002422002101A8F8F71B
:1085300006F901A9200001F0B5FE002808D0074C7B
:10854000002D00D02C60200026F028F90BB030BDA3
:1085500001A8039C01F07BFEF2E7C046FFFFFF7F0E
:1085600030B5A5B004000D00242200210AA8F8F7B8
:10857000E6F844232000099326F002F9002842D0AF
:1085800029002000FFF744FA002801D125B030BDB2
:1085900004A8FFF7C3F90028F8D106AA05A920000E
:1085A00026F006F90028F1D109AB009308AA13AB15
:1085B00007A9200026F02CF90028E7D1059B079990
:1085C0000D93069B0E93119B0393002B19D0002350
:1085D00000220AA801F046FE089B0C4A934200D9EB
:1085E0000B4B02AA138713A92B00099A0AA80C9413
:1085F00001F0EDFE0028C9D129880498FFF7F2F9AF
:10860000C4E70A91E8E78C204042BFE7F8FF00008A
:10861000FFFF000010B584B0089C0294079C0194F1
:10862000069C009426F03CF904B010BD10B582B051
:10863000059C0194049C009426F064F902B010BDDE
:1086400010B526F08FF910BDF0B5DE4657464E4600
:108650004546E0B514008A1E8DB0012A3FD8012B93
:108660003DD14368282B3AD105686B6AEE880B939D
:108670008368AF689846C368994623689A466368DA
:108680009B46032926D000230A9309930023002147
:1086900063603000FFF788F8002814D15B4605932B
:1086A000534604934B46039343462A0002930A9B86
:1086B00004340193099B1432009306940B9B3900F8
:1086C000300003F0BDF80DB03CBC90469946A24680
:1086D000AB46F0BD0369099343690A93D6E782204C
:1086E0004042F0E7F0B5DE4657464E464546E0B517
:1086F00014008A1E8DB0012A3FD8012B3DD8436853
:10870000282B3AD105686B6AEE880B938368AF68B3
:108710009846C368994623689A4663689B4603292E
:1087200026D000230A9309930023002163603000C0
:10873000FFF73AF8002814D15B460593534604939B
:108740004B46039343462A0002930A9B0434019349
:10875000099B1432009306940B9B3900300003F000
:10876000E1F80DB03CBC90469946A246AB46F0BD40
:108770000369099343690A93D6E782204042F0E7F0
:10878000862040427047C046862040427047C0461F
:10879000862040427047C046862040427047C0460F
:1087A000862040427047C046862040427047C046FF
:1087B000862040427047C046862040427047C046EF
:1087C000862040427047C046862040427047C046DF
:1087D000F0B5D6464F464646C0B5140086B00229CD
:1087E00031D1012B2FD14368282B2CD10368876806
:1087F000DD889E68C3680021984613682800994662
:1088000053689A46FEF7D0FF002805D006B01CBC7E
:1088100090469946A246F0BD05A92800FFF760FEE4
:10882000534601934B4604340093029443463A0066
:108830003100002803D1280002F0BEFBE6E70598CE
:10884000FFF7E8FEE2E782204042DFE7F0B5CE46E0
:10885000474680B585B003292DD1002B2BD1436825
:10886000282B28D103688668DC889D680369C7685F
:1088700098464369002120009946FEF795FF00289D
:1088800004D005B00CBC90469946F0BD03A9200069
:10889000FFF726FE4B460193434632000093290022
:1088A0003B00002803D1200002F08AFCE9E703988E
:1088B000FFF7BCFEE5E782204042E2E7F0B54E4616
:1088C0004546DE465746E0B515008A1E95B00400C1
:1088D0000E00012A4CD8012B4AD14368282B47D1DE
:1088E00003682422DF889B680021994683689A46A2
:1088F000C3680BA807932B689B466B689846F7F7ED
:108900001EFF032E31D00024002600213800FEF780
:108910004BFF002806D015B03CBC90469946A246B5
:10892000AB46F0BD0BA9380001F0BCFC0028F2D129
:1089300004AB9B8E0BA809930B9B089301F087FC5B
:10894000089A114B1340114A934214D043460393A3
:108950005B4604350293049501940096079B5246AA
:108960004946380002F0E0FCD5E726696469CCE7A7
:1089700082204042CFE7099B0733DB089845E5D2C8
:108980008A204042C7E7C046FFFFFFEF00000160BA
:10899000F0B5DE4657464E464546E0B514008A1E01
:1089A00089B0012A35D8012B33D14368282B30D127
:1089B0000368C768DD889E688368079323689A46C2
:1089C00063689B4603291FD00023994698460021DF
:1089D0002800FEF7E9FE00280FD15B4603935346BB
:1089E00002934B46019343460434009304943B00A6
:1089F000079A3100280002F00DFD09B03CBC9046FA
:108A00009946A246AB46F0BD03699846436999462C
:108A1000DDE782204042F0E770B5002482B0009488
:108A2000012927D1012B25D15368042B22D143687A
:108A3000282B1FD103681668D9686A460191042063
:108A400001A99D68FEF7E8F9041E0AD1019B009870
:108A500033600A4B9D4207D0290003F0E5FB041E5A
:108A600004D1200002B070BD0560FAE73000FEF7C7
:108A70004BFAF6E782246442F3E7C046000F00B0E9
:108A800030B583B001291AD1012B18D14368282BA6
:108A900015D15368042B12D1002403681568D968D6
:108AA00001AA04200194FEF771FA002802D02C607C
:108AB00003B030BD2900019803F030F9F8E78220B7
:108AC0004042F5E710B582B0012914D1002B12D134
:108AD0004268282A0FD102680420D168146901AACB
:108AE0000193FEF753FA002803D12100019803F007
:108AF0001FF902B010BD82204042FAE7F0B5C64629
:108B000000B582B002293ED1002B3CD14268282A10
:108B100039D10268C7689688D16882680420904677
:108B20006A460093FEF732FA041E0BD1009D1A4BE1
:108B30002A689A420BD03B0042463100280003F0DD
:108B400099FB0400200002B004BC9046F0BD134B1A
:108B50009E421BD101A8FEF733F8041EF2D13E1D40
:108B60003100012000F0C4FAA861002811D00422CD
:108B700001A9F7F7C8FDAB693A00181D4146F7F7A0
:108B8000C2FDEE61DEE782246442DBE787246442B3
:108B9000D8E78D246442D5E7000F00B00102000041
:108BA00030B583B0012916D1012B14D14368282B8D
:108BB00011D130CA036801AAD968002304200193A7
:108BC000FEF7E4F9002804D12A002100019803F0FF
:108BD000BDF803B030BD82204042FAE770B582B0E4
:108BE00001291ED1002B1CD14268282A19D1026804
:108BF0000021D48896882000D5680193FEF7D4FD23
:108C0000002801D002B070BD01AA29000430FEF78F
:108C1000BDF90028F6D122003100019803F031FBA4
:108C2000F0E782204042EDE7F0B585B002292DD172
:108C3000012B2BD14368282B28D1C368242B25D1A5
:108C40005368022B22D103688568D9680023146811
:108C5000042002AA0293FEF799F9002801D005B07A
:108C6000F0BD03A8FEF75AFE0028F8D10299194B6F
:108C70000A689A420DD02200280003F085FA0028E5
:108C8000EDD121880398FEF7ADFEE8E7822040424F
:108C9000E5E72E8B0736F608402E18D8CB690F0073
:108CA0009C46D937FF378869002301960097002238
:108CB000614625F09BFE002806D1230032003900D2
:108CC000280001F084FBDAE793204042C7E78D20BB
:108CD0004042C4E7000F00B070B582B001293BD11B
:108CE000012B39D14368282B36D15368042B33D15B
:108CF00003681668DC68002301AA01932100346030
:108D00000420FEF743F9002500280DD13460019CB2
:108D1000134B22689A420AD0200002F075FE051E0D
:108D200015D03000FEF7F0F8280002B070BDA06941
:108D3000002806D0E2690021F7F701FDA06900F0E4
:108D4000DFF98622002192002000F7F7F8FC3000BE
:108D5000FEF7DAF80500E7E782256D42E4E7C04652
:108D6000000F00B0F0B5C64600B584B0022926D188
:108D7000002B24D14268282A21D10268C168D488F6
:108D800087688846039300212000D5689688FEF7FF
:108D90000BFD002803D004B004BC9046F0BD03AA2C
:108DA00029000430FEF7F2F80028F4D143462200EF
:108DB000009331003B00039803F08AFAEBE782202E
:108DC0004042E8E710B5012908D1012B06D14368DC
:108DD000282B03D103CA03F0CFFA10BD82204042F2
:108DE000FBE7C04630B585B0022914D1012B12D162
:108DF0004368282B0FD104688568C368E188A068A0
:108E0000141D029454680194126800922A0003F021
:108E1000DDFA05B030BD82204042FAE70D4A016814
:108E20000123914213D10C4AC16991420FD182684A
:108E30009A420CD8C268002A02D001698A4206D040
:108E40004269131E03D083699B1A5842434118009C
:108E50007047C04655AA00FF669911EE0F4B70B5DA
:108E60009E680124002E0AD03000FFF7D7FF041EB1
:108E700012D1F368002B0FD13569002D01D12000EC
:108E800070BD2800FFF7CAFF002805D1EB68B34288
:108E900002D12E002D69F0E70124F0E76873010884
:108EA000F8B53B4E0C003368002B4FD0B368002B55
:108EB0004CD00D004543002848D0002915D00100B2
:108EC0002800FAF731F9A04240D12B1D3ED80323E8
:108ED00029001D4201D099430431F46803E062681F
:108EE0008A4235D2A469002CF9D12000F8BDF36084
:108EF0003DE00B002033E3189F60264F203A5A6074
:108F000022691F60244FDC601A61DF61002A00D0F3
:108F1000D360624658619A61002815D083619A69CE
:108F2000002A00D053612361002301226361A36101
:108F30003369A2606160134223D120342A000021EA
:108F40002000F7F7FCFBD0E7F360E8E70024CCE76C
:108F5000A768002F19D1A369521A60699C46232A79
:108F6000C7D80123A36063460028C0D08361A369EA
:108F7000002B00D0586100236361A3613369DB07D4
:108F8000DBD5FFF76BFF0028D7D00120F7F75EFB9A
:108F90006873010855AA00FF669911EEF8B500281C
:108FA0005DD03A4E3368002B59D0B268002A56D0B3
:108FB000834203D872689B18984202D30120F7F7C6
:108FC00045FB20380400FFF729FF0028F6D1A368ED
:108FD000012BF3D1E568A060002D14D0AB68002B05
:108FE0003ED163686A682033D3186B6023692B61B4
:108FF000002B00D0DD6027002000202200212C0063
:10900000F7F79DFB3D002069002835D08368002BD1
:1090100032D16368426820339B18636062690369D8
:10902000A1692361002A1DD1002921D142698169EA
:109030006261A161002A1DD09461A269002A00D05A
:109040005461002B00D0DC6020220021F7F777FB71
:1090500033699B0703D5FFF701FF0028AED1F8BDA8
:109060000500D0E79161A1690029DFD04A61DDE701
:10907000F160F8E7F460E0E7002DE9D1F368A3615F
:10908000002B00D05C61F460E2E7C0466873010821
:1090900070B5124E0D000400002114223000F7F7C5
:1090A0004EFB0F490F4800F033F8232D15D9032349
:1090B000234003D0043DE41A5D1904342A00002142
:1090C0002000F7F73CFB084B7560B4603460236008
:1090D000064B203D6560E361F46070BD6873010874
:1090E0009D8F0010A18E001055AA00FF669911EE09
:1090F00010B5024B1B68984710BDC04680CD0008D4
:1091000010B5024B1B68984710BDC04684CD0008BF
:10911000024B1860024B00201960704780CD000898
:1091200084CD000810B50A1E03D0024B00211B6835
:10913000984710BD88CD0008030000B57F3304DADE
:10914000FF234042DB011840404203006C334DD006
:1091500003006C3300DDC3E0984B984200D1ECE192
:1091600064DC974B984225D032DC964B984246D02F
:1091700016DC954B984200D1DFE10ADC934B984214
:109180004AD09723924A5B42904200D1E5E1842382
:1091900011E0904B984200D1D5E08F4A9623F2E738
:1091A0008E4B984238D008DC8D4B984261D08D4B65
:1091B0009842ECD186235B42CFE18B4B98421ED084
:1091C0008A4B984255D08A4B9842E0D19223F2E7DD
:1091D000884B98424DD014DC874B9842EAD007DC8C
:1091E000864B984245D0864B9842D0D18A23E2E7FD
:1091F000844B984200D1A0E1834B9842C7D18D2384
:10920000D9E7824B984207D008DC814B984200D1C5
:1092100093E1804B9842BAD19323CCE77E4B98429E
:10922000EDD07E4B9842E1D07D4BC1E77D4B98421B
:10923000C0D028DC7C4B98421BD010DC7B4B984282
:1092400017D007DC7A4B984202D07A4B98429ED1D5
:109250009723B0E7784B9842DED0784A9EE7784B68
:10926000984206D007DC774B9842C8D0764B98429C
:109270008DD187239FE7754B9842FAD0744B984263
:10928000F7D0744BA0E7744B984293D012DC734B29
:109290009842EED008DC724B984203D0714B984252
:1092A00000D074E7852386E76F4B984200D181E7B1
:1092B0006E4B7DE703007A33AED003007A3305DCD2
:1092C0006B4B984200D138E16A4BA3E7030070333F
:1092D000A2D003006E33BBD0723000D057E769E7ED
:1092E0000300293398D00300293300DDD0E00300C8
:1092F0003A3335D003003A3334DC03006033B8D05E
:109300000300603312DC03006633B2D0030066331F
:1093100006DC03006A3300D171E76830A9D036E774
:1093200003006433A5D06230A3D030E7030051338B
:109330009FD00300513308DC0300563300D1FCE01A
:10934000543000D023E7892335E70300403307D0AA
:109350000300403300DA1AE73D30012800D916E750
:10936000942328E703003433FAD00300343316DCA7
:109370000300373300D14FE70300373307DC030026
:10938000393300D148E7383000D113E7FFE6030056
:10939000363300D10EE7353000D13DE7F7E6030064
:1093A000313300D138E70300313365DC0300333358
:1093B00000D131E7323000D1FCE6E8E680BCFFFFA7
:1093C00080AFFFFF809EFFFF009DFFFF009CFFFF1F
:1093D000809CFFFF809DFFFF009EFFFF80ADFFFF91
:1093E000009FFFFF809FFFFF80AEFFFF00AFFFFFEA
:1093F00000AEFFFF80B3FFFF80B1FFFF80B0FFFF33
:1094000000B1FFFF00B2FFFF80B2FFFF80BAFFFF95
:1094100000B4FFFF80B4FFFF80BBFFFF00BCFFFF75
:1094200000BBFFFF80C3FFFF80BFFFFF00BEFFFF49
:1094300000BDFFFF80BDFFFF80BEFFFF00BFFFFF3D
:1094400080C1FFFF80C0FFFF00C1FFFF80C2FFFFA0
:1094500000C3FFFF00C2FFFF80C6FFFF00C5FFFF84
:1094600000C4FFFF80C4FFFF80C5FFFF00C6FFFFF1
:1094700000C7FFFF80C7FFFF03002D3300D1CBE6FD
:1094800003002B3300D1C7E62F3000D07FE6C3E6C0
:109490000300133300D1BFE60300133331DC0300B4
:1094A000223313DC0300243300DB83E6030027337D
:1094B00000D1B1E60300273300DADAE603002633F1
:1094C00000D177E6253000D1A6E660E60300183328
:1094D00000D16FE60300183307DC0300203300D10E
:1094E00068E6193000D197E651E60300163300D143
:1094F00060E60300163300DA8EE6143000D1B8E6D9
:1095000045E603000C3300D1B3E603000C3316DC50
:109510000300103300D172E60300103306DC0300B1
:1095200012330AD0113000D176E630E603000E3354
:1095300000D19EE60E3000DD9BE695233BE6831DC1
:1095400000D196E6831D0ADC03000A3300D190E6C1
:109550008A235B42083000D019E6180000BD831C46
:1095600000D133E600239842F7D0031D00D00EE669
:109570007FE6C046832270B50C00920000210500F2
:109580000C30F7F7DCF8FF2122002B4B2B488A43E5
:109590002340834202D02A4B9A4229D10C40802199
:1095A000284B49042143CB18022B36D9264BCB1824
:1095B000012B37D9254B994236D0254B99421AD0E9
:1095C000244B994227D0244B994233D0234B9942C4
:1095D0002AD0234B994229D0224B994224D0224BA6
:1095E000994223D0214B994222D0214B994221D03C
:1095F000862040420EE020231148824206D01D48BA
:10960000824203D11C4A89180129F1D8FF22002087
:109610005343AB6070BD3023EEE71023084882420D
:10962000EDD1E5E71423F9E71C23F7E72023F5E75D
:109630003023F3E74023F1E700FDFFFF00010020A6
:1096400000020020FFFFFFFEFCFFFFFE08000001FC
:10965000090000010A0000010B0000010C000001DC
:109660000D000001100000011100000112000001B6
:109670001300000100030020F7FFFFFEF0B51F00FC
:10968000002387B03B600C9B06000D001400002BEC
:1096900009D00368C0221900D2051140914200D1BF
:1096A0009CE087264BE0002A00D19AE0C02280216E
:1096B0000368D2051A40C9058A4211D1026AA24242
:1096C00000D98EE0C1692800F7F71DF8306A0C99BF
:1096D000221A2818F7F733F8336A3B60002620E097
:1096E00041491A0C12048A421ED10C9A002A1BD13D
:1096F000338B0733DB1001939C4200D271E0F06999
:109700001A0029007C300CF059FCFFF715FD061EED
:1097100007D1019B0C99E21AE818F7F710F8019BA2
:109720003B60300007B0F0BD304A31491A408A42F0
:1097300007D0304A1340304A934227D086267642DB
:10974000EFE704A810F008FC2C4B0493F369059391
:109750000C9B002B07D1E0223368D2051340C022B6
:10976000D205934217D12B1904AA290003A8039309
:1097700011F0B8FC061E14DA220000212800F6F7CA
:10978000DEFF3000FFF7D8FC0600CAE704A810F09F
:10979000E3FB1B4BD9E72200290004A811F006FDCA
:1097A000E8E74300A3420DD8241A2C190200210037
:1097B0002800F6F7A8FF320000212000F6F7BFFFCF
:1097C0003E608BE7A042FBD2241A02002919280030
:1097D000F6F7A2FFA81922000021EFE7002C00D025
:1097E0007EE78A26ABE7C04600000370FFFFFFEF6D
:1097F000000001600000FFEF00000360940E021003
:10980000340E0210F0B50B6889B006000D00002B75
:1098100006D00268934203D08720404209B0F0BDD1
:109820002B6A002B30D032681B4B13401B4A9342EB
:10983000F2D102AF38000CF0B7F905A80CF0B4F97A
:109840000021019700910B000A00F06903F0D6F99E
:10985000041E0DD12A6AE96905A80CF03EFB041E1E
:1098600006D105A938000CF01FFD041E00D00C4CD9
:1098700038000CF09FF905A80CF09CF9002C03D0DF
:109880002000FFF759FCC9E700202B8B8342C5D08D
:10989000328B9A42C2D0BFE7FFFFFFEF00000160AA
:1098A00080BFFFFF70B51500FE22D2050400024004
:1098B000C020C004824201D12E4A1440FA228020E6
:1098C000D2052240C004824237D12B4A94422CD088
:1098D0000FD82A4A94420AD006D8294AA41802224C
:1098E000012C11D9002035E0264A9442FAD10722F2
:1098F0000AE0254A94421ED011D8244A944216D038
:10990000042223488442EDD122480918002004296A
:1099100020D80800F9F7FEFB2B1F172729001E4A45
:10992000944206D01D480622ECE70522ECE703220C
:10993000EAE70822E8E70A22E6E7194A002094420B
:1099400008D10122E0E70520002B00D01870290083
:109950000EF022FA70BD0320402DF5D00130802D8D
:10996000F2D14035F0E70720EEE70920ECE70220CE
:10997000EAE7C046FFC0FFFF0100C0040100800409
:1099800000FF9FFB05008004050000060200C004E4
:109990000300C004FFFFFFBF0100400602004006B5
:1099A0000200C002CC235B00C358084A10B59342A2
:1099B00003D0074A934204D010BD08300EF08EF851
:1099C000FAE708300FF0F9FEF6E7C046011040064E
:1099D0000210400670B505001E4B1F4A1D409542FF
:1099E00004D01E4C1E4E0440B44230D10B40934272
:1099F00004D01A4C1A4E0C40B44228D10400FF2661
:109A00004C40B44323D1954204D0144C144D04402F
:109A1000AC4208D1C5B2002D05D0802464042C438B
:109A2000104DAC4211D0934204D00C4B0C4A0B4069
:109A300093420CD1CAB200218A4206D080235B0433
:109A40001343084A934200D10100080070BD002171
:109A5000FBE7C04600FFFEFF0000021000FFFCFF16
:109A600000000410FF00000170B50122814224D0E3
:109A70000A00134B134D1A40AA4205D0124C134E44
:109A80000C400022B44218D10340AB4205D00E4B2B
:109A90000E4C03400022A3420FD1FF2405000022F8
:109AA0002540954209D080235B042B43084DAB42EF
:109AB00003D14140A1434A424A41100070BDC04613
:109AC00000FFFEFF0000021000FFFCFF000004107A
:109AD000FF000001F0B585B0019300230F000B607B
:109AE00003A91600039302F0D9FD051E1ED1E02341
:109AF000039CDB0522681340C022D205934201D1AA
:109B000001239E43E3683340B34212D1019B002BF3
:109B10000BD019002069FFF7A7FF002805D1019994
:109B20006069FFF7A1FF002803D03C60280005B062
:109B3000F0BD85256D42F9E7174B70B515009842C9
:109B40000ED005D8154B98421BD08620404217E016
:109B5000A223DB05984203D0A423DB059842F4D16D
:109B600007240C4016D10731C90869600120FFF7AE
:109B7000BFFA030028602000002B01D16C608D38F3
:109B800070BD40230A009A43802AE9D080235B00FD
:109B90009942E5D08720D9E701000050010000403C
:109BA000F8B516001A000023040040680F00136087
:109BB000984205D1144BE2681A4208D0872021E070
:109BC0000123A16802F0C8FD0028F3D0F8BD228B64
:109BD0000E4B9A4215D80125638BAB43EED1310071
:109BE000380002F097FD0028F0D131680A00C8CC97
:109BF000C8C2C8CCC8C2236813601B0CAB434B83DC
:109C0000E4E786204042E1E7FCE0FFFFF8FF0000C8
:109C1000F7B50D006B46016804000E8B0733320068
:109C200009682800FFF73EFE6060002807D0344B2B
:109C3000344A2B40934204D0334A93423DD0862687
:109C40000EE0CC23314A5B00E25010220433E25490
:109C500023680E3A1B6893432D4A934202D087260D
:109C6000764228E02700083738000DF010FF6B46D9
:109C70002268D979D269330038000DF00EFFFFF762
:109C80005BFA061E37D1FE23C021DB052B40C90439
:109C900000228B4201D1AA04920ECE204000205C0B
:109CA000904226D300228B4201D1AD04AA0E9E23FE
:109CB0000026FF33E2543000FEBDCC23154A5B0082
:109CC000E25010220433E25423680E3A1B68934397
:109CD0000F4A9342C3D12700083738000FF0E0FA4B
:109CE0006B462268D979D269330038000FF0DFFA69
:109CF000C5E7872676422000FFF754FEDBE7C04623
:109D0000FFC0FFFF010040060200400601104006B0
:109D1000010000400210400610B5FF230C000100B6
:109D20000C4A9943914212D10340802040041843C9
:109D3000094BC01803280AD8084B8000C05810F0FF
:109D400047F801210200200003F01CF810BD00209C
:109D5000F5E7C04600000312F8FFFFFE08E8011017
:109D600070B50D000400AC210120FFF7C1F9286097
:109D700000280ED0123CA4B205F0C0FA00210C2C31
:109D800001D8054B195D286807F06CFBFFF7D4F983
:109D900070BD8D204042FBE7F9E70110F7B51D00CB
:109DA00000230E0001A917000193FFF7D9FF041E3D
:109DB00017D101993B0088313200019805F022FC4F
:109DC000FFF7BAF9041E0CD101990198883105F00A
:109DD00093FCFFF7B1F9041E03D1019B2B60200017
:109DE000FEBD01980028FAD005F01AFB0198FFF794
:109DF00087F9F4E7F0B515000024BFB0060006A807
:109E000003930F0005940EF08FFE2B782000013B8A
:109E1000DBB20C2B01D81A4AD05C05AB3A003100FA
:109E2000FFF7BCFF041E1ED10122059906A80EF003
:109E3000C9FEFFF781F9041E15D10200290006A80A
:109E40000EF0C0FEFFF778F9041E0CD10D4B039AFB
:109E500001930D4B4599009306A8449B0EF0E2FE3A
:109E6000FFF76AF9040006A80EF08EFE059805F0CB
:109E7000D7FA0598FFF744F920003FB0F0BDC0467F
:109E8000ECE7011010760108C38A0110F7B5FF2333
:109E900006001D4F9E431D4B05000091019203409B
:109EA000BB4204D01A4B1B4A0340934220D1EBB271
:109EB000002B1DD0802252041343174A9B18032BFA
:109EC00016D8164A9B009C5820000FF081FF019B7A
:109ED0001870BE420ED1B54211D0002C11D0200016
:109EE0000FF072FF009B984209D08720404207E0A4
:109EF0000024E9E70A4B9E4201D1002C01D000204A
:109F0000FEBD8620F2E7C0460000021000FFFEFF03
:109F100000FFFCFF00000410F8FFFFFE08E801103E
:109F200000000310C023F0B5150080220768DB0590
:109F300089B004000E003B40D205934225D1964BD8
:109F4000E9009D4200D923E1944B994200D91FE1D9
:109F5000020038001C32FFF7EFFD071E00D0A3E01F
:109F6000002D04D02A003100E069F6F7CCFBC022B6
:109F700080212368D2051A40C9058A4200D0F3E047
:109F8000236AD800208300278EE0854A3B0C1B04FF
:109F9000934200D08BE00023B8B20593153301281B
:109FA0004AD0022848D0032846D00433042843D09E
:109FB000052841D0053306283ED007283CD0082884
:109FC0003AD00633092837D00A2835D010330B2869
:109FD00032D00C2830D014330D282DD00E282BD0A1
:109FE000343B0F2828D0102826D0112824D0043341
:109FF000122821D013281FD0043314281CD0152870
:10A000001AD00433162817D0172815D01033182863
:10A0100012D0123319280FD0223B1A280CD010333B
:10A020001B2809D010331C2806D0203B1D2803D044
:10A0300018331E2800D0002387279D4200D0A8E0B7
:10A0400005A9FFF78DFE071E26D105982A003100CD
:10A050007C300BF042FFFFF76FF8071E1CD105990B
:10A0600005987C3105F056FEFFF766F8071E13D100
:10A0700005984C4D03000200010001954A4D28331C
:10A080007C328831009505F053FCFFF755F8071E28
:10A0900002D1059BE3616AE70598002804D005F02A
:10A0A000BFF90598FFF72CF8380009B0F0BD3F4A1A
:10A0B000934208D12300B8B21C332A00FFF76EFE8A
:10A0C000071EF1D153E73A4B3A4A3B4093425FD1E6
:10A0D00003A80FF041FFE023DB051F409F4236D16C
:10A0E00000232A000093310003A810F007FEFFF7B9
:10A0F00023F8071E27D103A80FF064FF01282CD1F5
:10A10000049D280002F044FE8023C0005B019842B9
:10A1100026D805A80BF048FD3B003A0001970097B0
:10A1200005A9280002F06AFDFFF706F8071E05D111
:10A1300005A80BF074FE430700D0863F05A80BF07E
:10A1400039FD002F0ED003A80FF00AFFACE72A005C
:10A15000310003A810F0FCFEC9E787277F42F2E731
:10A160008627FBE7E56102E7114A12491A408A4255
:10A1700004D1E06902F00CFEC00003E70E4A0020A3
:10A1800013400A4A934200D0FCE6E369986DF9E671
:10A1900086277F4288E7C046FFFFFF1FF8FF0000C9
:10A1A0000000037010760108C38A011000000360EC
:10A1B000FFFFFFEF000001600000FFEF70B500251A
:10A1C00003680400AB4209D0C0228021D2051A40A6
:10A1D000C9058A4209D1E069FEF792FF24220021D5
:10A1E0002000F6F7ACFA280070BD0A4A0A491A4066
:10A1F0008A4203D1C06903F033FEECE7074A1340FB
:10A20000074A934203D1C06905F00AF9E3E79725AD
:10A210006D42E3E7FFFFFFEF000001600000FFEF8A
:10A220000000036010B5002801D0FFF7C7FF10BD84
:10A2300007B503000020834208D001A9180002F0EE
:10A240002DFA002802D10198FFF7B8FF0EBD10B516
:10A250000400C069FEF754FF242200212000F6F715
:10A260006EFA10BDF7B500260400019117001D001D
:10A27000B34209D019000120FEF73AFF061E0ED0A6
:10A280002A003900F6F73FFAE069002801D0FEF70E
:10A2900037FF0020019BE66125622360FEBD8D2013
:10A2A0004042FBE7F0B5050089B008000C00FFF75D
:10A2B000CEFF002328001A0004A9FFF70BFC051E9F
:10A2C0004ED1049B21001A00C1CAC1C1C1CAC1C17B
:10A2D00012680A60D203D20F628324491A688A4244
:10A2E00002D023498A423BD105AF3800DD690BF02B
:10A2F0005BFC00232800019700931A00190002F06C
:10A300007DFC00260500B0421AD11A4938000CF035
:10A3100012F80500B04213D038000BF0A1FD0390F5
:10A3200001000120FEF7E4FE061E1CD00100039A86
:10A3300038000BF043FE051E02D1039BE661236249
:10A3400038000BF037FC002D02D03000FEF7D8FEAD
:10A350002800FEF7F1FE051E02D02000FFF777FF70
:10A36000280009B0F0BD10256D42E9E7000001604A
:10A3700000000170010001007FB51C0000230D00EA
:10A3800016002360012203A9FFF7A4FB002806D1D1
:10A3900000902300320029000398FFF76FF904B002
:10A3A00070BD7FB5160000220D001C001A6003A9C5
:10A3B0001300FFF78FFB002807D101233200009321
:10A3C000290023000398FFF759F904B070BDF0B5D8
:10A3D0001F00002385B0050001911600029303932E
:10A3E0009A4216D003AB02AA3900FFF7D9FB041E2C
:10A3F00012D1320001990298FFF794FD041E0BD18F
:10A4000029000298FFF7FEF9041E05D1200005B0CF
:10A41000F0BD87246442F9E70298FFF703FF0023A9
:10A420003B80F3E7F0B595B000230BAC059222001A
:10A430008446079308930E00A1C9A1C2A1C9A1C275
:10A44000A1C9A1C2022207A960460993FFF742FBF6
:10A45000051E00D0A7E031000798FFF7D3F9051ECD
:10A4600000D0A0E0079E27693369049702939F42BA
:10A4700004D019003800FFF7ADFA049065697369DC
:10A48000280003939D4202D01900FFF7A3FA049B12
:10A49000002B05D1002F03D0029B002B00D080E0C1
:10A4A000002805D1002D03D0039B002B00D078E0BD
:10A4B000F368E26860611340E360049B08AA2361CB
:10A4C000059909AB2000FFF76BFB051E00D06AE081
:10A4D000C0228021089B079E02933368D2051A4050
:10A4E000C9058A4203D1348B0734E40809E0314AB4
:10A4F00093422ED10923348B64080134E4085C4371
:10A500003B3421000120FEF7F3FD8D25071E49D0C5
:10A5100000230100009322000AAB3000FFF7AEF8E1
:10A52000051E0AD1336839000393039A029B1A600F
:10A5300018000A9AFFF7F6FC050038002100FEF724
:10A54000F1FD3800FEF7DCFD002D2CD1280015B000
:10A55000F0BD194A934203D1348BE4081034D0E79C
:10A56000164A934205D10324338BDB085C435A34EB
:10A57000C7E7134A934205D10324338BDB085C43BE
:10A580004A34BEE70F4A1B0C1B049342ABD00E4A61
:10A5900004009342B5D1348B0734E40864000134DD
:10A5A000AFE787256D420898FFF73CFE0023059A28
:10A5B0001380CBE700000170000001600000027012
:10A5C00000000260000003700000036003680D4A91
:10A5D00010B50400934207D80B4A93420BD2002BCC
:10A5E0000CD0892040420BE0084A9342F9D804304D
:10A5F00007F018FA02E0043007F0DAF900202060D2
:10A6000010BDC04609000001080000010B00000158
:10A6100010B504008021F830FEF784FD2000FFF71C
:10A62000D5FF10BD036870B505000E481818032843
:10A6300014D82B1DF8F76EFD02020E0E180007F05D
:10A64000D7F9041E02D02800FFF7C0FF2000FEF754
:10A6500073FD70BD180007F005FAF2E7892040424B
:10A66000F7E7C046F8FFFFFE036870B506000D006F
:10A67000002B36D11C4BC818032824D8341DF8F7FA
:10A6800049FD0210151D200007F08CF90121200062
:10A6900007F0A2F9041E20D135602000FEF74CFD22
:10A6A0001AE0200007F07EF90021F0E7200007F013
:10A6B000B3F90121200007F0C9F9EBE7200007F00A
:10A6C000ABF90021F6E7FE20FF23C0051B0608407A
:10A6D000C01843425841873870BD3000FFF776FFFD
:10A6E000DBE789204042F7E7F8FFFFFE002310B5C3
:10A6F0009A4202D0FFF796FF0300180010BD000039
:10A70000F7B580241F00036864041600DBB2334AE7
:10A7100023439A18050001911024022A2DD9304AAA
:10A7200004349A18012A28D92E4A0834934224D096
:10A730002D4A0434934220D02C4A103493421CD02A
:10A740002B4A1034934218D02A4A243C934214D006
:10A75000294A0434934210D0284A043C93420CD036
:10A76000274A0434934208D0264A1034934204D036
:10A77000254A9B185C425C41A4013E60002E04D037
:10A78000320021210198F5F7DAFFB4421CD82B687A
:10A790001E4A981803281DD82B1D0199F8F7BAFCFA
:10A7A00002021010180007F031F9FEF7C5FC061E72
:10A7B0000CD13C602800FFF709FF06003000FEBD09
:10A7C000180007F05DF9F0E78A2676422800FFF7C7
:10A7D000FDFEF3E789267642F0E7C046FFFFFFFE65
:10A7E000FCFFFFFE08000001090000010A00000153
:10A7F0000B0000010C0000010D0000011000000121
:10A800001100000112000001EDFFFFFEF8FFFFFE46
:10A81000F0B5A5B001936B46039280221B795204D8
:10A8200013434F4A029199180500102202292DD98D
:10A830004C4904325918012928D94B4908328B4216
:10A8400024D04A4904328B4220D0494910328B42ED
:10A850001CD0484910328B4218D04749243A8B42C9
:10A8600014D0464904328B4210D04549043A8B42F9
:10A870000CD0444904328B4208D0434910328B42F9
:10A8800004D0424A9B185A4253419A01019B3449D1
:10A890005B180A2B06D83E49CE5C802E03D986244D
:10A8A000644242E00026B242F9D8039C04AFB442AD
:10A8B0003ED901992800FFF7D7FE041E31D1039A33
:10A8C00002992800FFF712FF041E2AD103AB802251
:10A8D00039002800FFF714FF041E22D1002336217F
:10A8E000039C9C422CD1331B1A0038193621029349
:10A8F000F5F725FF002004AAA04226D12B00F8334B
:10A900001818029A5C21F5F71AFF01992800FFF741
:10A91000ABFE041E05D1320039002800FFF7E6FE29
:10A920000400802104A8FEF7FDFB200025B0F0BD47
:10A93000002CD8D0220002993800F5F7E4FECDE7CC
:10A94000FA5C4A40FA540133CBE7F8239C466A216B
:10A95000835C84444B40614601306B54CCE7C04675
:10A96000FFFFFFFEFCFFFFFE0800000109000001E1
:10A970000A0000010B0000010C0000010D000001A5
:10A98000100000011100000112000001EDFFFFFEA8
:10A9900018E8011070B51E00244B0400049D9A4273
:10A9A0002ED003339A4213D00223FF3387209A42DA
:10A9B0001BD1A378012B36D120000B002A003100D7
:10A9C0001430FFF725FF002801D10223A37070BDCA
:10A9D0008378002B27D1002D0ED029000120FEF70F
:10A9E00087FB6060002802D18D204042EFE72A00FB
:10A9F0003100F5F788FEA5600123A3700020E6E78B
:10AA00008378022B0FD1002D0BD029000120FEF7F7
:10AA10006FFBE0600028E7D02A003100F5F773FEF5
:10AA200025610323E9E78920DFE7C0460102000032
:10AA3000F0B5C5B00700009101921E00802B2FD801
:10AA4000002503AC1A00637002AB2900981D257025
:10AA5000F5F775FE02AB06339B191D7062789D1CDD
:10AA60005A70280032000199F5F74DFEBB78AD19F8
:10AA70002A1B012B11D13800009B21001430FFF755
:10AA8000C7FE051E01D10223BB70822120004900B0
:10AA9000FEF748FB280045B0F0BD89256D42F4E77C
:10AAA00087256D42F6E70000F0B5002607681E4BCB
:10AAB00095B0FB1805000091019203960A2B01D86E
:10AAC0001A4AD65C03AB402204A92800FFF718FEFF
:10AAD000041E25D139002800FFF7C6FD041E1BD136
:10AAE00029003200F8312800FFF700FE041E13D1C0
:10AAF000039A04A92800FFF7F9FD041E0CD103AB4B
:10AB0000402204A92800FFF7FBFD041E04D1019A8E
:10AB100004A90098F5F7F7FD039904A8FEF702FBD6
:10AB2000200015B0F0BDC046FFFFFFFE18E8011081
:10AB30007FB503790D0004001100DA072CD5062239
:10AB40001340022B28D042798A4222D80368134945
:10AB50008B4213D1694608300DF01AFD061E04D150
:10AB6000627969462800F5F7CEFD68461021FEF7A8
:10AB7000D9FA3000FEF7E0FA04B070BD08490B4086
:10AB8000A02189048B4207D129000830FFF78CFFF0
:10AB9000F2E78A204042EFE78920FBE70200C0028B
:10ABA0000000C07FF0B593B002AC0D00160001AB01
:10ABB00040222100FFF7A4FD00280AD1019FB742DF
:10ABC00005D1020003009F4205D1002A01D0952043
:10ABD000404213B0F0BDE95CE65C013371400A43CA
:10ABE000F1E700000B6870B505000C00002B1BD1CD
:10ABF00003680E4A934207D80D4A93420CD2002BA9
:10AC000012D0862040420EE00A4A9342F9D8011D34
:10AC1000201D06F00FFF03E0011D201D06F0D0FEF1
:10AC200000202B68236070BD8920EBE7090000013C
:10AC3000080000010B0000010021036810B50400AA
:10AC40008B420BD00F4A93420AD108300DF0C0F866
:10AC5000E02200212379216013402371080010BDF8
:10AC6000094A1340A0229204934203D10830FFF70F
:10AC7000CFFCEDE7C0225200F5F761FD8921494282
:10AC8000ECE7C0460200C0020000C07FF0B51D0026
:10AC90001E006B1E9D4180236D421B01AD0285B0DD
:10ACA000ED18664B019101681340040017000093F2
:10ACB000002900D0B9E0E02203600379134003715A
:10ACC000009B1A005E4B9A4227D108300DF07AF8AB
:10ACD000002E03D010232279134323713B002A0056
:10ACE00003A90198FEF7F6FE061E12D1009BBD04D3
:10ACF0001A00534BAD0E03999A4249D10F8B0300B2
:10AD000009683A000098FEF7CDFD011E1DD1862688
:10AD100076422000FFF790FF14E0A022494B9204F6
:10AD20003B40934201D18160D2E7FE26FE23F60527
:10AD30003E401B06F618C02277427E415200873EF5
:10AD4000F5F7FDFC300005B0F0BD2600436908367C
:10AD50006371039B300000930DF06AFA002805D15F
:10AD6000009B3A00D96930000DF07EFBFEF7E4F954
:10AD70000600002D05D0032DC9D96379AB4232D32B
:10AD80006571002EC5D10123227913432371D9E7C0
:10AD9000A0222C4B92043B40934249D1FBB2802726
:10ADA000294A7F043B439A18022A35D9274A9A1820
:10ADB000012A2FD9264A934201D11C220DE0254AAF
:10ADC000934201D1202208E0234A934201D130224C
:10ADD00003E0224A934208D140226271A22208680D
:10ADE000D20590421AD0872692E71D4A9342E4D0BA
:10ADF0001C4A9342E6D01C4A9342DED01B4A93423F
:10AE0000E0D01B4A9342E2D01A4A9342E4D0002396
:10AE100063717CE71422E0E71022DEE720000A6A73
:10AE20000830C969FFF7F4FCA2E78926764289E772
:10AE3000002D00D16BE7862676429CE7FFC0FFFF1E
:10AE40000200C0020000C07FFFFFFFFEFCFFFFFE0C
:10AE500008000001090000010A0000010B000001C8
:10AE60000C0000010D0000011000000111000001A4
:10AE7000120000011300000110B50123FFF706FFC7
:10AE800010BD10B50023FFF701FF10BD70B5040021
:10AE90000079C30703D489256D42280070BD0623BD
:10AEA0000340022BF7D00823034323710D48236886
:10AEB00083420BD1200008300DF000FBFEF73CF977
:10AEC000051EEAD02000FFF7B7FEE6E7064803407C
:10AED000A02080048342DED120000830FFF706FC6A
:10AEE000EEE7C0460200C0020000C07FF7B51F00B9
:10AEF0000368040001911600002B03D189256D42DF
:10AF00002800FEBD3A60002A03D021210198F5F700
:10AF100016FC2379DB06F1D5320001992000FFF7FA
:10AF200007FE05002000002D0CD1FFF785FE051E51
:10AF300002D163793B60E3E7320021210198F5F704
:10AF4000FEFBDDE7FFF778FEDAE7F0B5036893B0C4
:10AF500006000191002B2BD0102304791C4027D12F
:10AF6000477997421ED1402202A9FFF7E1FD230055
:10AF700005009F420ED8002C14D1002D14D13000B2
:10AF8000FFF75AFE0500402102A8FEF7CBF8280083
:10AF900013B0F0BD019A02A9D25CC95C01334A40EA
:10AFA0001443E6E795256D423000FFF745FEEAE7DA
:10AFB00089256D42EBE70000F0B593B00892079346
:10AFC000199A1A9B0C001A60002A00D1DCE080223A
:10AFD0000B00D2000BA9FEF77DFD051E1AD10B9ABE
:10AFE000E0211368C90518000840884249D1684922
:10AFF0008B425CD10FAFD66907993A002000FEF76B
:10B0000045FF051E06D1300001F0C2FE199B8342A8
:10B0100004D28A3D199A212118982AE0FF239C43E3
:10B020005C4B9C422AD12A002900300001F0AAFE84
:10B03000189B594A0393089B58490293079B300079
:10B0400001933B780093012302F05CFD041E04D1C0
:10B05000300001F09DFE1A9B18602000FEF76CF88E
:10B06000051ED7D121211A9B1868199B1A1A189B03
:10B070001818F5F764FB280013B0F0BD484B9C424C
:10B0800002D087256D42C5E73A783000012101F0F2
:10B0900079FE189B00950393089B3F4A0293079BF8
:10B0A0003E4901933000012302F0F6FBCEE73D4913
:10B0B00086250B403C498B42E4D13C4B3C49234024
:10B0C0008B42DED1D6690CA8B36DDD1DED080AF008
:10B0D0006BFD0FA80AF068FD6B000993199B6A00CD
:10B0E00093424FD337007C37E3033CD5E4B2002CC6
:10B0F00037D080235B041C432E4BE418032C30D83C
:10B100002D4BA400E0580EF063FE234B02900493F5
:10B11000224B0FAA0393079B0CA90193089B3000B5
:10B1200000933B000DF030FE041E0DD12A0018994B
:10B130000CA80AF043FF041E06D1189B2A005919D7
:10B140000FA80AF03BFF04000CA80AF033FD0FA87B
:10B150000AF030FD002C00D07FE71A9B099A1A6094
:10B160007BE70020CFE70C4B0FAA03930B4B0CA9F6
:10B170000293079B30000193089B00933B0003F070
:10B1800099FAD1E70D4CDFE78A256D4273E7C04697
:10B19000000001700000021010760108C38A01103F
:10B1A000000003100000FFEF0000036000FFFEFF3F
:10B1B00000000610F8FFFFFE08E8011000B1FFFFD5
:10B1C000F0B591B00792802206930D000B0012019A
:10B1D00009A9FEF77FFC041E36D1099A4749136876
:10B1E00047481940814248D10DAFD66906993A00C7
:10B1F0002800FEF74BFE041E26D1300001F0C8FDEA
:10B20000179B834202D0952464421DE0FF239D4397
:10B210003C4B9D421BD122002100300001F0B2FDC9
:10B22000169B394A0393079B38490293069B3000CB
:10B2300001933B780093230002F0F0FD344B9842D9
:10B24000E1D0FDF779FF0400200011B0F0BD314BD3
:10B250009D4251D13A783000012101F093FD169BB7
:10B2600000940393079B284A0293069B2749019366
:10B270003000230002F052FDE0E727490B40274948
:10B280008B4237D1264B1D40264B9D4234D1D76986
:10B290000AAEBB6D30000733DB080DAD05930AF035
:10B2A00083FC28000AF080FC059B179A5B009A42F9
:10B2B000A9D1059A169930000AF00FFE041E11D18B
:10B2C000169B059A280099180AF007FE041E09D15A
:10B2D0003B00019588330096069A0799380003F0E1
:10B2E000BDFA040030000AF065FC28000AF062FC98
:10B2F0002000A6E7862487E7872485E7FFFFFFEF86
:10B30000000001600000021010760108C38A0110DD
:10B3100000BFFFFF000003100000FFEF000003600C
:10B3200000FFFEFF00000610F0B51F0000238BB0E9
:10B330000792149A0E0013600A00FF339A432F4BB2
:10B3400006929A4205D0119B002B02D087246442BA
:10B3500034E080223300520009A9FEF7BBFB041E33
:10B360002CD1099AC0211368C905180008408842E9
:10B37000ECD123490B4023498B423BD1D5692800AE
:10B3800001F006FD139B984236D81F4B9E4218D100
:10B39000129B00970293079B1C4A01931C492300B0
:10B3A000280002F069F8041E04D1280001F0F0FC26
:10B3B000149B18602000FDF7BFFE040020000BB0B6
:10B3C000F0BD069B1A000D4B9A42BFD129003000F8
:10B3D000FEF7A2FC129B02970493079B0B4A039370
:10B3E000119B0B490193109B28000093230001F04F
:10B3F0003BFFD8E78624AAE78A24A8E700000312C7
:10B40000FFFFFFEF0000016000000212107601084C
:10B41000C38A0110F0B58BB0079300231700149A6C
:10B420002B4E13600A00FF339A430D000692B2427E
:10B4300005D0119B002B02D0872040422BE08022B8
:10B440002B00920009A9FEF745FB002823D1099B98
:10B45000E0211A68C905100008408842ECD11D4956
:10B460008A4233D1DC69200001F092FC079B9842AC
:10B47000E2D1194B9D4210D1139B01970393129B6C
:10B48000164A0293149B164900932000012302F0F0
:10B49000DFF9FDF751FE0BB0F0BD069BB342CBD1F7
:10B4A00021002800FEF738FC139B03970593129B9D
:10B4B0000A4A0493149B0A490293119B20000193AA
:10B4C000109B0093012301F0F7FFE2E78620B4E729
:10B4D0000000031200000170000002121076010843
:10B4E000C38A011070B5002503680400AB4210D078
:10B4F000FE22D20513408022D20493420BD10830A1
:10B500000CF066FCF8222379256013406571A57163
:10B510002371280070BD89256D42FAE7F0B585B02A
:10B5200004000091160001938025012B12D0AD007C
:10B530002168002900D09BE0FE238022DB053340F8
:10B54000D204934208D04C222000F5F7F8F8872562
:10B550006D428AE06D00EBE701222700237908376E
:10B56000934303329343023A134323716171A171F0
:10B57000380026600CF026FC2A00330003A900984E
:10B58000FEF7A8FA051E6DD103990B8B096800938D
:10B59000009A03003000FEF785F9011E60D03800E4
:10B5A0000CF046FE051E48D10399019B009AC9691B
:10B5B00038000CF025FC051E3FD12F4B9E4242D097
:10B5C0002E4B9E424AD00122237990211343FF2221
:10B5D000D20523713240C90401238A4214D0039B4F
:10B5E00027491A6810238A420ED02649083B8A420E
:10B5F0000AD0254908338A4206D0244B0121D218AB
:10B60000002391425B41DBB2A371730215D5039B0A
:10B610001B491A6810238A420ED01A49083B8A42F5
:10B620000AD0194908338A4206D0184B0121D21892
:10B63000002391425B41DBB263712800FDF77CFD82
:10B64000051E12D00EE0042138000CF0AFFD0028DA
:10B6500010D10123227913432371C0E70100F3E7DE
:10B6600086256D422000FFF73DFF280005B0F0BDA4
:10B6700089256DE70500E0E7000160040101600431
:10B68000010000400200004003000040FCFFFFBF3B
:10B6900010B50123FFF742FF10BD10B50023FFF7DF
:10B6A0003DFF10BD037970B5040006200340022B56
:10B6B00017D1637993420ED120001A0008300CF0A4
:10B6C000BFFBFDF739FD051E07D104232279134383
:10B6D0002371280070BD87256D422000FFF702FF0F
:10B6E000F7E789256D42F4E770B50C0006211E00CE
:10B6F000037905000B40022B1CD14379934213D8E8
:10B700001A0021000D480DF0DCF9002805D0FDF7E6
:10B7100013FD041E0AD1200070BD6A792100326039
:10B720002800FFF7BFFFF4E78A2464422800FFF7F0
:10B73000D9FEF0E789246442EDE7C046107601089F
:10B74000F0B585B00393036804000F001600002BCA
:10B7500027D0FF22D205134090223500D204934215
:10B7600006D08579C36A2900F018F7F7DDFC454358
:10B770000A9B9D420FD820000B9B3200009339009A
:10B78000039B08300CF08AFBFDF7D6FC051E04D1A4
:10B79000280005B0F0BD8A256D422000FFF7A2FE0B
:10B7A000F6E789256D42F3E7F0B51E00037985B011
:10B7B00004000D001700DA073CD506221340022BC7
:10B7C00038D01023C356012B06D11C4B02689A4275
:10B7D00002D1C36A002B28D120003200694608300C
:10B7E0000CF076FC00280CD0FDF7A6FC0500002329
:10B7F000684633601021FDF795FC2000FFF772FECC
:10B8000010E03268002A05D0BA4211D869462800F3
:10B81000F4F779FF10216846FDF784FC2000FFF75C
:10B8200061FE0500280005B0F0BD87256D42DEE70A
:10B830008A25FBE789256D42F4E7C04600016004D4
:10B84000F0B51E000023F3B009927E9A0AAD136092
:10B8500080220B000F0052002900FEF73BF9041E66
:10B860003ED139002800FEF7D3F9041E38D19E27B7
:10B87000FF37EB5D7B9A7D999A188A4247D87B996E
:10B880007C9A26485218CC214900695881422AD115
:10B8900005937C9B069204937A9B00960393799B75
:10B8A0007B9A0293789B012101930CA8099B0DF0D0
:10B8B0003FFFFDF741FC041E07D07D9B002B04D009
:10B8C0001A0000217C98F4F73AFF0AAD2800FEF731
:10B8D00069F8002C04D1EB5D7B9A9B187E9A13606B
:10B8E000200073B0F0BD0E48814213D105937C9BBC
:10B8F000049203937A9B099A0293799B7B99019313
:10B90000789B0CA8009333000CF008F9D1E78A2447
:10B910006442DAE786246442E2E7C0460210400649
:10B9200001104006F0B5F1B00793002316007C9A91
:10B9300008AD136080220B000F0092002900FEF773
:10B94000C9F8041E3DD139002800FEF761F9041E34
:10B9500037D19E27FF37EB5D799A934247D8D11AAA
:10B960007B9A8A4246D3CC204000789A2858244CAF
:10B970005218A04228D17A980393779B059001939F
:10B980007898769B0490029200933200079B0AA855
:10B990000DF0E9FEFDF7D0FB041E07D07B9B002BCA
:10B9A00004D01A0000217A98F4F7C9FE08AD2800E7
:10B9B000FDF7F8FF002C04D1EB5D799AD31A7C9A3D
:10B9C0001360200071B0F0BD0E4CA04214D105935D
:10B9D0007A9B04920393789B32000293779B0AA888
:10B9E0000193769B0093079B0CF0DAF8D2E787244B
:10B9F0006442DBE78A24FBE786246442E1E7C04631
:10BA00000210400601104006FE22C0210368D20544
:10BA100070B51A40040089058A4213D11D4A1340AB
:10BA2000802292051343FF22190091431A4A914242
:10BA300012D1E068FDF764FB20001430FEF7E8FD4A
:10BA4000050002E00025AB42EDD1862120008900EF
:10BA5000FDF768FB280070BD104A5B0A5B02934249
:10BA600014D12069002805D06169FDF75BFB2069CE
:10BA7000FDF746FBA069002805D0E169FDF752FB00
:10BA8000A069FDF73DFB20002030D7E789256D42F6
:10BA9000DBE7C046FFFF0308000100200002002092
:10BAA000F0B585B00293FE230E00C0210568DB05CA
:10BAB00004002B4089058B4204D182490D4080212E
:10BAC00089050D430223FF339E4207D004D37E49EC
:10BAD0007118032900D88EE0872694E0A421C905B7
:10BAE0008A4201D0002AF7D1FF212A0077488A43F1
:10BAF000824200D0B7E00D408021754A49040D43D1
:10BB000096427AD0734A964200D190E09E42E3D1A9
:10BB10000327714BE15C039339400FD120002B00C8
:10BB20000A001430FEF774FE061E00D0BCE0039B32
:10BB3000E25C0123BA431343039AA3540322039BF9
:10BB4000E35C1340012B5DD1270014370A9A029958
:10BB50003800FEF7CBFD061E00D0A5E021008D3198
:10BB60004022FF313800FEF79FFF061E00D09BE009
:10BB70005A4A1023AA18022A2DD9594A0433AA185E
:10BB8000012A28D9574A0833954224D0564A04330B
:10BB9000954220D0554A103395421CD0544A103358
:10BBA000954218D0534A243B954214D0524A04334C
:10BBB000954210D0514A043B95420CD0504A043370
:10BBC000954208D04F4A1033954204D04E4BED18A1
:10BBD0006B425D41AB0183229200A35400224B4B88
:10BBE000E254039B0332E35C93431A0002231343A2
:10BBF000039AA35418E0464972E70322364FE35DE7
:10BC0000134202D0892676424EE020002B000A9A89
:10BC100002991430FEF7FCFD061E45D10323E25DB8
:10BC20009A43023B1343E355300005B0F0BD2A4D63
:10BC3000635DDA439207E5D05B07E3D40A9B236197
:10BC4000002B0AD019000120FDF752FAE06000280D
:10BC500033D00A9A0299F4F756FD0423625D002658
:10BC600013436355E0E72B4882420CD10D408021FD
:10BC7000200032000A9B49040093029B29430C30A8
:10BC8000FEF788FE0EE02448824218D10D40802144
:10BC9000200049040C3029439E4209D10A9B029A94
:10BCA000FEF7C6FE061EBFD02000FFF7ADFEBBE7C5
:10BCB0000A9B32000093029BE2E78D26A3E78926C8
:10BCC0007642B1E7FFFF0308FFFDFFFF0001002000
:10BCD00002020000030200000E020000FFFFFFFE50
:10BCE000FCFFFFFE08000001090000010A0000013E
:10BCF0000B0000010C0000010D000001100000010C
:10BD00001100000112000001EDFFFFFE0D02000016
:10BD10000100005000020020000300200368002BF7
:10BD200003D0836800200B60704789204042FBE706
:10BD30000368002B05D083688B4205D38160002007
:10BD4000704789204042FBE78720FBE7F0B5C7B08A
:10BD50000292FE220591C0210368D20504001A4018
:10BD600089058A420DD1B64A1340802292051343B9
:10BD7000A26802998A4209D200238F25A3606D42EE
:10BD8000A7E0002BF4D189256D427CE002990029BF
:10BD900002D1002A00D1F5E102991800521AA260DE
:10BDA000FF22A8499043884200D0B6E08027134084
:10BDB0007F041F43A44B1026FB18022B2DD9A34B45
:10BDC0000436FB18012B28D9A14B08369F4224D0FA
:10BDD000A04B04369F4220D09F4B10369F421CD070
:10BDE0009E4B10369F4218D09D4B243E9F4214D04C
:10BDF0009C4B04369F4210D09B4B043E9F420CD07C
:10BE00009A4B04369F4208D0994B10369F4204D07B
:10BE1000984BFE1873425E41B6019749625C9307E6
:10BE20009B0F012B00D8ABE1530700D4A8E10323FB
:10BE300013436354029B0093059B0493009B002BC8
:10BE400020D083239B00E15C009B751AEDB29D42DC
:10BE500001D96B461D782300CD33FF332A005918D2
:10BE600004980393F4F74FFC8322049B92005B1920
:10BE70000493009B5B1B0093A35CED18009BA554EF
:10BE8000002B03D10025280047B0F0BD7B4AA35CFE
:10BE9000FF2B00D174E101338321A35400238900D7
:10BEA000635423002100143301938D313B00320091
:10BEB000FF310198FEF7ACFC051E0AD16F4AA35C66
:10BEC000012B11D12269E1680198FEF70FFC051ED4
:10BED00012D026682000FFF797FD2660029A2121E4
:10BEE0000598F4F72CFCCEE7320003990198FEF791
:10BEF000FDFB051EE6D0ECE7604B0122E11801983E
:10BF0000FEF790FB051EE4D1402203990198FEF74D
:10BF1000CBFD051E00D191E7DBE75948590A4902DC
:10BF2000814200D02FE7802713407F041F43464BF8
:10BF3000FB18079310230093079B022B38D9142377
:10BF40000093424BFB18012B32D91C22404B00922C
:10BF50009F422DD03F4B043200929F4228D03E4B4F
:10BF6000103200929F4223D03C4B103200929F42ED
:10BF70001ED03B4B243A00929F4219D0394B0432D9
:10BF800000929F4214D0384B043A00929F420FD047
:10BF9000364B043200929F420AD0354B1032009249
:10BFA0009F4205D0334BFB185A4253419B010093EB
:10BFB000029B0393059B0493039B002B00D161E735
:10BFC000267B002E00D0C0E0079B022B2CD91F4BF4
:10BFD000FB18012B2AD91E4B9F422BD01D4B9F4291
:10BFE0002AD01D4B9F4229D01C4B9F4220D01C4B76
:10BFF0009F421FD01B4B9F421ED01B4B9F4219D00C
:10C000001A4B9F4218D01A4B9F4217D01D4B9F428C
:10C0100000D14036F822002108A8F4F790FB637B9A
:10C02000FF2B31D19725AAE61026F3E71426F1E776
:10C030004026EFE71C26EDE72026EBE73026E9E770
:10C04000FFFF030800010020FFFFFFFEFCFFFFFED3
:10C0500008000001090000010A0000010B000001B6
:10C060000C0000010D000001100000011100000192
:10C0700012000001EDFFFFFE0E0200000D020000A5
:10C0800000020020130000010133637323002033FA
:10C09000267308A918000193FEF7A4FD051E44D1DC
:10C0A000637B012B4CD1E269A1690198FEF71EFB6D
:10C0B000051E3AD1626921690198FEF717FB051E3A
:10C0C00033D123009933FF333200190001980693CE
:10C0D000FEF7EAFC051E28D1019908A8FEF782FDAB
:10C0E000051E22D1320006990198FEF7FFFA051EBF
:10C0F0001BD1E269A1690198FEF7F8FA051E14D177
:10C10000626921690198FEF7F1FA051E0DD121003F
:10C11000D9313200FF310198FEF7C6FC051E04D16B
:10C12000019908A8FEF75EFD050008A8FEF74EFA83
:10C13000002D00D0CDE6002800D13DE70500C8E67F
:10C14000210099313200FF31B6E7039B35009E4252
:10C1500001D96B461D7B009B2A00991B2600D9360E
:10C16000C9B2FF3671180498F4F7CDFA049B5B1935
:10C170000493039B5B1B0393237B5D1B25731BE7CE
:10C180008925FCE58F25FFE50023F0B585B00293F6
:10C190000393038B050000910192002B3ED00126F2
:10C1A0000B7933423DD003AB02AA0199FDF7F8FCAD
:10C1B000041E25D1C023029FDB0539682A8B0B4062
:10C1C0008021D51DED08C9058B4222D1530720D10E
:10C1D00030002900FCF78CFF061E1DD001002A004C
:10C1E0000098FFF7B3FD041E05D12A003100380086
:10C1F000FDF798FE04003000FCF782FF002C05D00C
:10C200000298FEF70FF80023019A1380200005B072
:10C21000F0BD87246442F3E78D24FBE78724644262
:10C22000F4E78524FBE70000036870B504000D0007
:10C23000002B18D1FE23DB050B408022C021920584
:10C2400089058B420BD10A492940114391420DD0F7
:10C250002000FDF78FF9002800D1256070BD9342C2
:10C2600004D12900F4E789204042F7E78720FBE763
:10C27000FFFF030807B5009313000022FFF710FC2F
:10C280000EBD7FB50400100080220E00236852010D
:10C2900003A9FDF71FFC051E05D02000FFF7B4FB26
:10C2A000280004B070BD0223FF339E4204D12279DE
:10C2B000013BFF3B13432371039A3100136A2000B3
:10C2C0000093D3691268FFF7EBFB0500E8E7000075
:10C2D000F0B50600FE251000C02299B00393336824
:10C2E000ED050F001D40920595423DD1802205A924
:10C2F0005201FDF7EFFB041E2ED1FC2331681B0415
:10C300000B401D431A4B059A06909D4227D1136896
:10C3100018491B0C1B048B4224D106AB019342230A
:10C320000093D26907AB1E990398FDF763FD041EC5
:10C3300009D1A422069BD2050093390007AB300037
:10C34000FFF7AEFB0400069907A8FCF7EBFE002CF4
:10C3500002D03000FFF758FB200019B0F0BD862452
:10C360006442F0E78724FBE787246442F4E7C04691
:10C370000000203000000370F8B5CF23104A9B0066
:10C38000D35C07000E00DB0716D580250C00ED00FE
:10C39000B919091B0B48AC4203D822000CF091FBE1
:10C3A00004E02A000CF08DFB002802D0FCF7C4FE4C
:10C3B000F8BD054BE418EBE789204042F8E7C0469A
:10C3C0007C7301081076010800FCFFFFF0B51F0028
:10C3D000FE2305001600C022DB0585B008002B40B7
:10C3E0009205934202D0872464421DE080222B00F4
:10C3F000520103A9FDF76EFB041E15D1104B039AE1
:10C400009D421BD113680F491B0C1B048B42EAD1C0
:10C410000C9B390001930B9B30000093D2690A9B5F
:10C42000FDF7E8FC041E06D00B990A98FFF7A4FF5D
:10C430000C9B0B9A1A60200005B0F0BD8624D3E750
:10C4400000002030000003700023F0B587B0049393
:10C450000593038B07000391002B00D19FE005ABF0
:10C4600004AAFDF79DFB041E2AD1049DFA693E8BA8
:10C470003C6A2868002A02D1002C00D08DE0C0233D
:10C480008021DB050340C9058B4210D12A00310011
:10C490001C32FDF751FB041E12D1296AE869FFF72F
:10C4A0006BFF041E0CD10024200007B0F0BD3D4BF3
:10C4B000984240D180235B019E4208D98624644281
:10C4C0000498FDF7AFFE0023039A1380ECE70723DF
:10C4D0003340F3D1002C13D0042CEFD811191C00D9
:10C4E0001378240201321C439142F9D1002CE5DB80
:10C4F000AC210120FCF7FCFD071E03D18D24DEE7F3
:10C50000294CF5E70022110000F02EFC00943300C6
:10C51000264A2749380001F0DBFC041E09D0380008
:10C5200001F09EFC3800FCF7EBFD2000FCF704FE58
:10C53000B7E7EF61B8E71F4A030C1B049342BDD174
:10C54000123880B200270C2801D81B4B1F5C380022
:10C5500002F082FE002CB1D1002FAFD00028ADD068
:10C5600083889E4219D1AC210120FCF7C1FD061E33
:10C57000C4D002F0C3FE38000C4B0D4A310003F06A
:10C5800099FC071E07D0300002F04AFF3000FCF78C
:10C59000B7FD3800CAE7EE6186E787248FE7872476
:10C5A000644281E70000017001000100107601087B
:10C5B000C38A011000000370F9E7011010B500F004
:10C5C00093F8CF23084C9B00E25C06231A4205D067
:10C5D00006480CF0BEF9064863689847D021200051
:10C5E0008900FCF79FFD10BD7C73010810760108DF
:10C5F00084730108F0B5224B85B00393CF23214CFF
:10C600009B00E35C0026DB0733D42368B34201D1EF
:10C610001D4B23606368002B01D11C4B63601C4FD2
:10C62000236838009847CF251A4EAD0030000CF033
:10C6300086F90623625D18499A43043B1343635508
:10C6400003233A000093300003AB0CF093F9FCF79E
:10C6500073FD061E10D10623625D9A43023B13430D
:10C66000635500F035F8061E06D10123625D1343C1
:10C670006355300005B0F0BDFFF7A0FFF9E7C046F5
:10C68000505341007C7301083990011081900110D2
:10C690008473010810760108A390011090230B4ABF
:10C6A000DB00D35CDB070CD5431E98B21F280BD8E8
:10C6B0002420584380180368002B05D00860002010
:10C6C000704789204042FBE78820FBE7BC760108E1
:10C6D000902201230349D200885C03438B5400203D
:10C6E0007047C046BC76010870B50024242630008F
:10C6F0006043074D01344019FDF760FD202CF6D151
:10C7000090220121D200AB5C8B43AB5470BDC0467C
:10C71000BC760108902330B50E4CDB00E35CDB07F0
:10C7200013D52023242503800288002A03D18D20DD
:10C730000A60404230BD2B00013A5343E3180B60BE
:10C740001B68002B03D00280EEE78920F1E7180078
:10C75000F0E7C046BC760108002A01D00023136030
:10C760000138434258418738704707B5030000201D
:10C77000834208D001A91800FFF790FF002802D1DA
:10C780000198FDF71BFD0EBDF0B597B002920600B3
:10C7900040220D0006A800210393F3F7D0FF0023E9
:10C7A00005931C9B18680DF00FFB0190002D07D11D
:10C7B0002C0006A84021FCF7B5FC200017B0F0BD06
:10C7C000019B00959D4200D900931C980DF0D4F96F
:10C7D000041EEED1039A02991C980DF0EDF9041E87
:10C7E000E7D1042205A91C980DF0E6F9041EE0D15A
:10C7F00006AF39001C980DF0F9F9041ED9D1009B41
:10C800009C4206D105AAD37836190133D3702D1B6B
:10C81000CCE7335DE25D534033550134EFE7000070
:10C82000F0B51E00002385B005000F0001920293B1
:10C830000393984260D00DF025F9041E03D13B4DBF
:10C84000280005B0F0BD280002AA03A90DF032FBB4
:10C85000051EF4D120000DF0B7FA029A009083185B
:10C860001A0008327F2AEAD8010002320A318A42CD
:10C87000E5D3B242E3D834000A3CE41A0A2CDED9EC
:10C880000A9B0A9A9F1C1D700123033C5370FF21D1
:10C8900022003800F3F753FF30213B1959701D7007
:10C8A000029C00982200083282189A70E2B2D97075
:10C8B000111D19710621DF1D59719A71039922000A
:10C8C0003800F3F720FF05233F193B70013BFC18AC
:10C8D000BB70009B20001A00FB707D700199F3F77C
:10C8E00012FF0A9B009A9B19A418A342A8D03100FA
:10C8F0000A98FCF717FCA2E78E42A0D3761A0A2EFC
:10C900009DD90A9B0A9A18709C1C0123033E537000
:10C91000FF2132002000A619F3F711FF3570701CBB
:10C920003A000199F3F7EFFE8AE7C04680BFFFFFA8
:10C93000F8B5050008354768040028000E0009F026
:10C940008FFA874201D02848F8BD80236268DB0057
:10C950009A42F8D80021280009F0EDFC0028F2DD09
:10C960000021280009F005FA0028ECD0002E1FD184
:10C9700020000021143009F0DEFC0028E3DD002E49
:10C9800014D020000021443009F0D5FC0028DADD65
:10C9900020000021503009F0CEFC0028D3DD20001B
:10C9A00000215C3009F0C7FC0028CCDD0020CBE77B
:10C9B00025002C350021280009F0BDFC0028C2DD2F
:10C9C0000021280009F0D5F90028BCD00C35002141
:10C9D000280009F0B0FC0028B5DD0021280009F08E
:10C9E000C8F90028C4D1AEE780BFFFFF70B50400CE
:10C9F0001D0000290AD006000836300009F06DFA43
:10CA0000002818D1300009F02BFA6060002D0AD1FF
:10CA1000059B002B12D1079B002B18D1099B002BE3
:10CA20001ED1002070BD2000049A29002C3009F08E
:10CA300054FA0028ECD00F4BC018F3E72000069AF8
:10CA40000599383009F049FA0028F4D1E3E72000CD
:10CA5000089A0799203009F040FA0028EBD1DDE769
:10CA600020000A9A1430099909F037FA0028D8D022
:10CA7000E1E7C04680BFFFFF0300F0B508338BB08D
:10CA8000039000211800069309F055FC039B002138
:10CA90002C3305001800049309F04DFC039B07009C
:10CAA000383300211800059309F045FC039B0290E0
:10CAB000203300211800079309F03DFC039B0890E8
:10CAC000143300211800099309F035FC002F00D120
:10CAD0008DE0029B002B00D171E0089B002B00D160
:10CAE0006DE00200531E9A41002D62D0029C3C432F
:10CAF00000D069E0089B2600002B02D00600731EC0
:10CB00009E41089B23431C1E1ED10123002800D1F7
:10CB1000002321003143114308910B4347D0002DDE
:10CB200019D1002F17D0029B002B14D0059A04991D
:10CB3000069809F014FD002808D02F4BC0180BB040
:10CB4000F0BD3A00D2E7029E0024E1E7069809F022
:10CB500087F9039B5860002E20D0059B079A00930D
:10CB60000999049B069801F09DFA0028E5D1089BDD
:10CB7000002B0ED0039B079A5C330193039B05990E
:10CB800050330093039B0498443301F033FD002895
:10CB9000D3D108990398FFF7CBFED0E7002CE6D05D
:10CBA000079B099A0599049801F062FBDDE712489A
:10CBB000C5E73E1EC8D0029B1E1EC5D00AE02A1E35
:10CBC000F7D00022029C3C433E1E00D199E7029B15
:10CBD000002BB8D00024089BA34202D10400601EA1
:10CBE00084412E1E00D193E70026330091E7002DEB
:10CBF000A7D12A002E00A7E780BFFFFFF7B51E00D0
:10CC00000300083304000F001800002115000193F1
:10CC100009F091FB002803D1002D2FD02A483AE0DB
:10CC2000200000212C3009F086FB0028F4D02000E1
:10CC30000021383009F07FFB0028EDD020000021D2
:10CC4000203009F078FB0028E6D0200000211430C5
:10CC500009F071FB0028DFD0002F16D1002D1BD169
:10CC6000002E21D1089B002B26D1099B181E12D023
:10CC700021000998143108F0D9FF0CE0002ECDD125
:10CC8000089B002BCAD1002FEFD00199380008F083
:10CC9000CDFF0028E2D0FEBD210028002C3108F095
:10CCA000C5FF0028DCD0F6E721003000383108F05D
:10CCB000BDFF0028D6D0EEE721000898203108F00B
:10CCC000B5FF0028D1D0E6E780BFFFFFF8B504002C
:10CCD0000F000830002116001D0009F02CFB002871
:10CCE00001D12048F8BD200000212C3009F023FBA1
:10CCF0000028F6D020000021383009F01CFB002865
:10CD0000EFD020000021203009F015FB0028E8D0EA
:10CD100020000021143009F00EFB0028E1D0002F84
:10CD200005D1002E0DD1002D13D10020DAE721000E
:10CD30003800443108F07AFF0028F2D0094BC018BF
:10CD4000D0E721003000503108F070FF0028F5D105
:10CD5000E9E7210028005C3108F068FF0028EDD1E8
:10CD6000E3E7C04680BFFFFF70B504000E0015006A
:10CD70000021A422F3F7E3FC2300A834A4331E60AF
:10CD8000256070BD0300A830A433196002607047AD
:10CD90004068704770B500210400FFF7C9FD051E0B
:10CDA00018D126000836300009F039F87F2811D94B
:10CDB00014342900200008F0DCFF00280AD02000ED
:10CDC00009F02DF8012805D93100200009F06CFA8E
:10CDD000002800DB014D280070BDC04600BEFFFFEB
:10CDE000F0B585B00400FFF7D5FF002802D0164843
:10CDF00005B0F0BD01212000FFF79AFD0028F6D113
:10CE00002500260027002300029001902000143303
:10CE10002C3538362037009332003B00290008308B
:10CE200001F00EFB0028E2D1220023005C325034D6
:10CE30000192443300943A003100280001F074FA62
:10CE40000028D5D0D3E7C04600BEFFFF70B5040070
:10CE50000D00FFF79FFF002814D12800FFF7C0FF47
:10CE600000280FD1290020000831083009F01CFAF1
:10CE7000002807D1290020001431143009F014FAD9
:10CE8000002800D0004870BD00BEFFFFF0B50C00C8
:10CE900087B0002105001600FFF74AFD002830D1B9
:10CEA00003A808F081FE21006A6803A809F015F8BC
:10CEB000041E19D12C000834210003A809F0F4F94C
:10CEC00000281BDA2A006F6803A968352300143292
:10CED0000095080009F062FE041E05D13A003100F9
:10CEE00003A809F06BF8040003A808F063FE002C07
:10CEF00001D0054BE418200007B0F0BD04246442C3
:10CF0000F2E7024CF7E7C04680BDFFFF80BFFFFF9E
:10CF1000F0B5A7B002910121050007921C00FFF7B0
:10CF200007FD002800D094E108A808F03DFE0BA8FA
:10CF300008F03AFE0EA808F037FE11A808F034FEFB
:10CF4000029B002B05D01AA808F02EFE1DA808F0A1
:10CF50002BFE14A808F028FE17A808F025FE20A82C
:10CF600008F022FE23A808F01FFE21006A6808A826
:10CF700008F0B3FF041E00D03CE12F000837390051
:10CF800008A809F091F9002800DB5BE108A920A8B6
:10CF900008F04CFE041E00D02CE12B004433039318
:10CFA0000C330493029B002B00D181E02B00A033B3
:10CFB0001B68002B00D1D9E02E008C3632003100E6
:10CFC000300009F0CCFA041E00D013E13A00310021
:10CFD000300009F073FD041E00D00BE10C36320066
:10CFE0003100300009F0BBFA041E00D002E13A0023
:10CFF0003100300009F062FD041E00D0FAE02A0082
:10D0000008A98C32080009F0AAFA041E00D0F1E049
:10D0100008A93A00080009F051FD041E00D0E9E01B
:10D02000290001222C310BA809F087FA041E00D038
:10D03000E0E02900012238310EA809F07EFA041E32
:10D0400000D0D7E0079B029A1C2111A80AF04AF8E9
:10D05000041E00D0CEE011AA0BA91AA809F07FFA8D
:10D06000041E00D0C6E01AA9039A080009F00BFAC2
:10D07000041E00D0BEE0079B029A1C2111A80AF0F2
:10D0800031F8041E00D0B5E011AA0EA91DA809F0C0
:10D0900066FA041E00D0ADE01DA9049A080009F04C
:10D0A000F2F9041E00D0A5E01DAB04931AAB039364
:10D0B0002B002C33059348330093039A059B08A952
:10D0C00014A809F06BFD041E00D093E02E002B0085
:10D0D000383680330093049A330008A917A809F062
:10D0E0005DFD041E00D085E017AA14A908A809F068
:10D0F000EEF9041E00D07DE02A0008A95C3214A8D5
:10D1000009F02DFA041E75D1059A14A908A809F092
:10D11000D5FC041E6ED1320008A914A809F01FFA2C
:10D12000041E67D114AA17A908A809F0ACF9041EB7
:10D1300060D1029B002B4ED12B002A006833009354
:10D1400014323B0008A923A809F028FD041E51D180
:10D1500020A923A809F0A8F8002800D077E06A6881
:10D160002C9908A808F02AFF040043E00C2305933B
:10D17000059B013B0593002B00D166E02B00983303
:10D1800006936B68029A591E0698079B09F0AAFF3E
:10D19000041E2FD12E008C363A000699300009F07B
:10D1A00027FF041E26D10121300009F0C4F8002811
:10D1B000DED13A00069930000AF08CF8041E19D12D
:10D1C0002B002A006833009314323B0031003000FA
:10D1D00009F0E4FC10E72A0008A99832080009F0D9
:10D1E000BEF9041E06D108A93A00080009F066FC41
:10D1F000041EA1D00BA808F0DDFC0EA808F0DAFC94
:10D2000011A808F0D7FC029B002B05D01AA808F043
:10D21000D1FC1DA808F0CEFC08A808F0CBFC14A88F
:10D2200008F0C8FC17A808F0C5FC23A808F0C2FC49
:10D2300020A808F0BFFC002C01D0074BE418200008
:10D2400027B0F0BD04246442D4E7044CD2E7044C78
:10D25000D0E7044CF3E7C04600BDFFFF80BBFFFFF3
:10D2600080BCFFFF80BFFFFFF0B58DB0029005913D
:10D2700006920793012B08D10300A4331B68012BEE
:10D2800003D0454C20000DB0F0BD059B002BF8D01D
:10D29000029BA8331868C0B20CF0F4FB061EF0D055
:10D2A000029B5B6803930CF08FFD43000493149B77
:10D2B000420002339B18149A07009342E1D3039A69
:10D2C0009342DED800211698F3F739FA169B169A86
:10D2D0000133049300230499137006983A00059BC8
:10D2E0009847002802D02D4BC418CBE7049B139A13
:10D2F000DD192B00129930000CF092FC041EC1D1F4
:10D30000039B149A981A02387B00C019C01A012393
:10D3100028180370002A03D001301599F3F7F3F9A8
:10D3200009A80CF0BBFB0022310009A80CF0E8FBB7
:10D33000041E18D1039D169B7E1C013D9E19ED1BFA
:10D3400009AB0093049A3B0029003000FFF71CFA58
:10D35000041E08D109AB009332002B003900049859
:10D36000FFF712FA040009A80CF09EFB002C00D075
:10D3700088E7079B002B06D1169A02981100FFF749
:10D3800085FD04007EE7169B069A00930599029896
:10D39000FFF7BEFDF5E7C04680BFFFFF80BBFFFF84
:10D3A000F0B587B006000F00049203930E9D012B89
:10D3B00007D10300A4331B68002B02D02C4807B010
:10D3C000F0BD0C9B70680C33F8D80C9B0B33834278
:10D3D000F4D80C9BC01A00232B70039B0338002B3E
:10D3E0002FD1002FEAD00233AC1C6B7023180593A9
:10D3F000059B9C4212D1002323700C9B002B04D070
:10D40000601C1A000D99F3F77EF9039B002B22D1C3
:10D410002A0029003000FFF739FDD0E7642302938A
:10D42000012221000498B8472378002B1BD1029BCE
:10D43000013B0293002B01D00028F1D00D4BC01806
:10D44000BDE70123FF226B70AB1C1C189C42D2D09D
:10D450001A700133FAE700952B00049A3900300066
:10D46000FFF756FDABE70028E8D10134C0E7C0461E
:10D4700080BFFFFF80BBFFFFF0B50700A4373F6808
:10D4800087B00C9C0D9D0E9E002F03D0012F08D05D
:10D49000084804E0029601950094FFF781FF07B069
:10D4A000F0BD029400240496039501940094FFF7C4
:10D4B000DBFEF4E700BFFFFFF0B5694C1D00A5449B
:10D4C000069104000792012B09D10300A4331B68C5
:10D4D000012B04D0634C2000634B9D44F0BD636876
:10D4E0001A000493FC23103A9B009A42F2D82300BE
:10D4F000A8331868C0B20CF0C5FA061EEAD00CF0CA
:10D5000063FC049A471C7B00039005939342E1D887
:10D510001CAA002D1ED1FFAB983319682000FFF71D
:10D52000B5FC041E0CD109A80CF0B8FA2200310099
:10D5300009A80CF0E5FA041E16D009A80CF0B4FAFC
:10D5400080211CA8C900FBF7EDFD40210CA8FBF7CA
:10D55000E9FDC0E7FFAB009298331B68079A069974
:10D560002000FFF7D5FCDCE759201CABDD19049B3C
:10D5700006AC5F1E039B0019FF1A09AB00932A003B
:10D580003B000399FFF700F9041ED6D1592209ABDD
:10D5900006A900935218039B39002800FFF7F4F8FE
:10D5A000041ECAD109A80CF07FFAFFAAFFA90CAD8E
:10D5B00090328C312B001268096830000CF030FB7F
:10D5C000041EBDD1582206AB9B181E78592306AA0B
:10D5D0009B18039A99180200039B76B29A4229D3AA
:10D5E0000020C918059A049B0D009B1A5B189C46E5
:10D5F00002000127AC4524D101208B5C5840064332
:10D6000076B2002E27D101328918049B1CAA8A1AEF
:10D610009A1AFFABA0331B689A421ED8FFAB943313
:10D620001B681A60002A8BD0FFAB9C331868F3F795
:10D630006AF885E7535D885C013243401E43F6B2C9
:10D64000CAE72B780135184343420343DBB2DB09B9
:10D650007B40D218CEE7054C72E7054C70E7C04618
:10D660008CFBFFFF80BFFFFF7404000000BFFFFFC3
:10D6700000BCFFFFF0B5734C1D004368A544039345
:10D68000012D05D10300A4331B68002B00D0D7E087
:10D69000FC24039BA400103BA34200D9D0E008AFB8
:10D6A000002D28D1FFAB40333A001968FFF7EEFB9D
:10D6B000041E00D0AFE03B7801257C7802276C4047
:10D6C000234300242100082006AA1218D25D013746
:10D6D0005042C00F684004436042D2432043C60F0B
:10D6E0006E40B446C017D2B282431343039A6144DA
:10D6F000BA42E8D123E0FFAB009740331B68FFF745
:10D7000007FC041E00D086E03B78012DD4D1022016
:10D7100021007A7842401343C25D013056423243C1
:10D72000D2B2D2096A401443E4B262422243D2B276
:10D73000D2096A40D2B28918039A8242ECD1FFA87A
:10D74000039A483000680B3A824200D90200080070
:10D750000838C00F034301206442E40F444003989B
:10D760002343C71E7F1A390058421843C01751403F
:10D7700001407940571AFF0F3B4388247D4282269F
:10D780005F423B43DB17DB43E4012C40F60166407C
:10D79000304044409C460B2064420826634606AF56
:10D7A000BF193F5C1F4006AB9B191F54039B013000
:10D7B0008342F2D113004B401D40039B4D40991A08
:10D7C00008AB5918002A18D0531B06935318079317
:10D7D000531E6E4205930800F3170493431C9C46A6
:10D7E000079B634520D1059B049FCB181878013611
:10D7F00007401F70069BB342EDD1FFAB48331B6857
:10D80000002B04D0FFAB44331868F2F77CFFFFAB6A
:10D810003C331B681D60802108A8C900FBF782FC0F
:10D820002000094B9D44F0BD03784778FFB2039771
:10D830007B40049F3B40039F7B4003706046CDE7E5
:10D84000024CEDE7DCFBFFFF2404000080BFFFFF7C
:10D85000F0B50400A434246887B00D9D0E9E0F9F80
:10D86000002C03D0012C0AD00A4806E00C9C039738
:10D87000029601950094FFF7FDFE07B0F0BD0C9CE9
:10D880000597029400240496039501940094FFF7F1
:10D8900013FEF2E700BFFFFFF0B5A1B00A9326AB7D
:10D8A000039018780A9B05910992012B08D1039BDC
:10D8B000A4331B68012B03D05D4C200021B0F0BDC8
:10D8C000059B002BF8D0039B5B680293002806D0D1
:10D8D0000CF0D8F80028EFD00CF076FA2790039BD4
:10D8E000A8331868C0B20CF0CDF8071EE4D00CF0D5
:10D8F0006BFA029A049043009A42DDD30233060089
:10D90000934201D9961E361A029A00212998F2F7FD
:10D9100016FF320010A90998059B9847041E02D0F3
:10D92000444BC418C9E7039B0DAD08331800069398
:10D9300008F075FA049A029B10A99B1A0793299A7A
:10D94000023B9B1BD3185A1C089201220B901A70A1
:10D9500008983200F2F7D7FE28000CF09FF822005A
:10D96000390028000CF0CCF8041E48D128000CF037
:10D9700003F9041E43D1089B08229F19390028008F
:10D980000CF01AF9041E3AD1279A289928000CF0B5
:10D9900013F9041E33D1320010A928000CF00CF941
:10D9A000041E2CD1390028000CF020F9041E26D1C9
:10D9B00007230B9807990138184043425841299B87
:10D9C0000139091A009518183A00049BFEF7DCFE8D
:10D9D000041E14D1069808F022FAFF22029B40216F
:10D9E000DB000133181A0241299B10A81B78134051
:10D9F000299A1370BC23049ABB54FBF793FB0DA820
:10DA00000CF052F8002C00D057E70A9B002B06D1EF
:10DA1000299A03981100FFF739FA04004DE7299B72
:10DA2000099A009305990398FFF772FAF5E7C04643
:10DA300080BFFFFF80BBFFFFF0B585B01E000AABC3
:10DA40000500029103921878012E04D12B00A43313
:10DA50001B68002B50D10D9B0C9A00936B680B999F
:10DA6000FEF7DEFE041E07D1002E08D10D9A280015
:10DA70001100FFF70BFA0400200005B0F0BD696843
:10DA80000120FBF735FB061E08D069680120FBF773
:10DA90002FFB071E05D13000FBF732FB1024644238
:10DAA000EAE700960D9B039A02992800FFF730FAE7
:10DAB000041E11D13A0031002800FFF7E7F9041ED7
:10DAC0000AD1010003006A689A420CD1002911D1E1
:10DAD00031000D98F2F717FE3000FBF711FB38000C
:10DAE000FBF70EFBC8E70D9DF85CED5C0133684069
:10DAF0000143E9E7014CEFE7014CBDE700BDFFFF43
:10DB000080BFFFFFF0B50500A43585B02D680AACD5
:10DB100024780C9E0D9F002D03D0012D0AD00948BA
:10DB200006E00B9D0397029601950094FFF784FF92
:10DB300005B0F0BD0B9D0397029601950094FFF789
:10DB4000ABFEF5E700BFFFFFF0B56F4C0500A54445
:10DB5000FFA88C3000780390FFA8983000780490DC
:10DB6000012B09D12800A4300068012804D0674C9B
:10DB70002000674B9D44F0BD6E68FC203400103CD3
:10DB800080008442F3D81CA8002B00D0ADE0FFAB8E
:10DB9000A033020019682800FFF778F9041EE7D1C6
:10DBA000771E1CABDB5DBC2B00D0AAE0039B002BD7
:10DBB00009D018000BF066FF0028D8D00CF004F94B
:10DBC000FFAB9033186004980BF05CFF041ECED0BE
:10DBD0000CF0FAF808220021039007A8F2F7AFFD35
:10DBE0002800083008F01BF9431E049304981CAA6F
:10DBF000F3001178C31A08331941B8D1612504AB79
:10DC0000ED1803005B0701D037001500039B0233BA
:10DC1000BB42ACD809AE30000BF040FF210000221F
:10DC200030000BF06DFF041E5BD1039B0096D943BF
:10DC3000C9196B1805936A18039B2800FEF7A4FD09
:10DC4000041E4ED1FF22049B6021F800C01A02413D
:10DC500004AB5B181B78134004AA52181370059B81
:10DC60005A1E2B780135691E8A4201D9002BF8D043
:10DC7000012B42D1059B5E1BFFAB9C331B6801331C
:10DC800004D0FFAB9C331B689E4236D109A80BF031
:10DC900073FF041E25D1082207A909A80BF08CFFE9
:10DCA000041E1ED1FFAB90331A68FFAB9433196882
:10DCB00009A80BF081FF041E13D13200290009A826
:10DCC0000BF07AFF041E0CD10CA909A80BF08EFFF3
:10DCD000041E06D1039A0CA90598F2F705FD041E4F
:10DCE0000DD109A80BF0E0FE42E7FFAB0090A03396
:10DCF0001B682800FFF70CF950E7064CF1E7064CCB
:10DD0000EFE7044C34E7C0468CFBFFFF80BFFFFF0A
:10DD10007404000000BFFFFF80BCFFFF70B505006A
:10DD200086B0A8350AAC24782E682500002E00D0D5
:10DD3000F5B20D9E0395059601260C9D764202953F
:10DD40000B9D049601950094FFF7FEFE06B070BD92
:10DD5000F0B587B003930CAB1C78039B0290049141
:10DD600005924768012B04D10300A4331B68002BE4
:10DD700045D139000120FBF7BBF9061E41D039001F
:10DD80000120FBF7B5F9051E3ED000903B002000B6
:10DD90000E9A0D99FEF744FD041E0FD1039B002B34
:10DDA0001FD132000F990298FFF770F8041E05D1B9
:10DDB000020003009F421CD1002A28D13000390004
:10DDC000FBF7B0F93000FBF79BF9002D06D02800D7
:10DDD0003900FBF7A7F92800FBF792F9200007B0FC
:10DDE000F0BD00960F9B059A04990298FFF790F8F2
:10DDF000DCE7F15CE85C013341400A43DAE7054CBB
:10DE0000ECE710246442E9E710246442D6E7024CB0
:10DE1000D4E7C04680BFFFFF80BCFFFFF0B5050020
:10DE2000A43585B02D680AAC24780C9E0D9F002D7A
:10DE300003D0012D0AD0094806E00B9D03970296F6
:10DE400001950094FFF784FF05B0F0BD0B9D03978B
:10DE5000029601950094FFF761FFF5E700BFFFFF11
:10DE600010B5041E32D08C3007F0A4FE200098308C
:10DE700007F0A0FE2000683007F09CFE2000203054
:10DE800007F098FE2000383007F094FE20002C3078
:10DE900007F090FE2000143007F08CFE20000830C0
:10DEA00007F088FE2000803007F084FE20007430E8
:10DEB00007F080FE20005C3007F07CFE2000503030
:10DEC00007F078FE2000443007F074FE10BD00001B
:10DED000F0B595B00600069107921D007F2B00D883
:10DEE000DAE01A9B022B00DCD6E0EB0700D5D3E08A
:10DEF0008023DB00AB429B415B425B000BA8059398
:10DF000007F052FE0EA807F04FFE11A807F04CFED6
:10DF1000330014331A991800029307F010FF041EFF
:10DF200000D0A6E06B0804930890C72D01D9633B8D
:10DF3000089301356B0809933700079B2C37009332
:10DF4000059A069B0499380009F036FB041E00D0A0
:10DF50008FE03500079B38350093059A069B04999E
:10DF6000280009F029FB041E00D082E02A003900B5
:10DF70000BA808F0ACFA041E00D07AE00BA807F05A
:10DF80004EFF089B9842D7D90B9B002B03DA290040
:10DF9000380007F07EFE01223900380008F0CDFA83
:10DFA000041E66D101222900280008F0C6FA041ECA
:10DFB0005FD12A0039000BA808F0D1FA041E58D10D
:10DFC0000BAA02990EA809F013F8041E51D10121E1
:10DFD0000EA808F0B0F90028AED12A0039000EA82A
:10DFE00009F006F8041E44D101000EAB0BAA11A8DB
:10DFF00008F0C0FB041E3CD13300203311AA029963
:10E000001800039309F066F9041E32D1039807F053
:10E0100006FF099B98428FD901223900380008F089
:10E020007AFA041E25D101222900280008F073FA8B
:10E03000041E1ED1330008332A0039001800029351
:10E0400008F08DFA041E14D1029807F009FF33007E
:10E050005C3301930C3B70600093039A0C3B2900E6
:10E06000380000F0C7FA041E03D13000FEF7B8FEF6
:10E0700004000BA807F09EFD0EA807F09BFD11A859
:10E0800007F098FD002C04D03000FFF7E9FE034BA9
:10E09000E418200015B0F0BD014CFAE780BEFFFF88
:10E0A00080BFFFFFF0B59BB005000F0014006F4963
:10E0B00036220CA81E00F2F726FB002E04D1042401
:10E0C000644220001BB0F0BD209B002BF7D0B3684A
:10E0D000002BF4D1209B99680029F0D1280008F08A
:10E0E0002AF90028EBDD0121200008F024F900289E
:10E0F000E5DD2900200008F0D7F80028DFDA01214B
:10E10000380008F018F90028D9DD2900380008F097
:10E11000CBF80028D3DA09A807F046FD06A807F0D7
:10E1200043FD21003A0006A808F019FA041E0FD199
:10E1300006A90122080008F000FA041E08D106A86A
:10E1400007F04DFE83B20393002B08D104246442F0
:10E1500009A807F02FFD06A807F02CFDB1E781B252
:10E1600006A807F0B9FF041EF2D10722AB6807002A
:10E170001B681340013B5A425341DBB29AB20492EE
:10E180000CAAD3180593059B09A8D95D07F0D7FD04
:10E190002A0009A9300008F02BFF041ED8D1012164
:10E1A000300008F0C8F8002806D0049B0137DB19BE
:10E1B0009BB2352BE7D9C9E7209B09A9009306AA92
:10E1C0002B00080008F0EAFC041EC1D101230293D1
:10E1D000012109A808F0AFF800283FD009A90122C1
:10E1E000080008F098F9041EB2D12A0009A93000ED
:10E1F00008F0FEFE041EABD10121300008F09BF8B0
:10E2000001280DD12900300008F04EF8431C07D139
:10E21000210033002A00209808F0ACFA040097E7A8
:10E2200009A90122080008F088F9041E90D109AA62
:10E230001100100008F093F9041E89D109A92A00E1
:10E24000080008F03BFC041E00D081E7029B01336C
:10E250009BB20293029A039B9342B9D2012109A86F
:10E2600008F069F80028A0D070E7C04623E8011044
:10E27000F0B589B006000D0001921C1E04D10426E1
:10E280007642300009B0F0BD0021180008F053F8C4
:10E29000071EF4D10121300008F04DF80028EEDD12
:10E2A0000121280008F047F80028E8DD390001982E
:10E2B00008F041F80028E2D002A807F075FC05A894
:10E2C00007F072FC3100012202A808F036F9061EA0
:10E2D00022D10122290005A808F02FF9061E1BD122
:10E2E00005AA02A9200008F083FE061E14D102A987
:10E2F00005AA080008F033F9061E0DD102AA010094
:10E300002300100008F036FA061E05D102AA019972
:10E31000200008F0DFFF060002A807F04BFC05A86C
:10E3200007F048FCADE70000F0B587B00400684690
:10E330001F000D00160007F037FC03A807F034FC9F
:10E34000002F07D10C9B002B2DD10D9B002B48D10A
:10E35000002402E0002C09D1374C684607F02AFC63
:10E3600003A807F027FC200007B0F0BD0122210020
:10E37000684608F0E2F8002853D13200390003A8BB
:10E3800008F0A5F800284CD103A96A46080008F057
:10E3900095FB002845D1010003A807F0CCFF002819
:10E3A000D0D0264CD9E7002DD6D0012229006846CE
:10E3B00008F0C3F8002834D132000C9903A808F003
:10E3C00086F800282DD103A96A46080008F076FBDC
:10E3D000002826D1010003A807F0ADFF0028E0D1F6
:10E3E000B3E7002CB8D0002DB6D02A000D996846AE
:10E3F00008F0B5F8002814D101226946684608F0F3
:10E400009CF800280DD122006946684608F056FBAA
:10E41000002806D10100684607F08DFF0028C0D112
:10E4200096E7064B9842BCD0034B984200D193E745
:10E43000024BC41891E7C04680BFFFFF00BEFFFF3C
:10E44000F0B589B0050002A801930E00170007F08F
:10E45000ABFB05A807F0A8FB0F9B002B00D191E0B8
:10E46000002E08D0109B0F9A3221300009F071F86D
:10E47000002800D0BAE0002F00D188E0109B0F9A4E
:10E480003221380009F065F8002800D0AEE0002EF7
:10E4900000D17CE0002D1AD03A00310002A808F02B
:10E4A0005EF8041E76D10121280007F044FF002801
:10E4B00000DC9BE0290002A807F0F6FE002800D04F
:10E4C00094E0019B002B00D073E0002E61D0002F60
:10E4D0005FD0019B002B5CD00E9B002B59D00121FB
:10E4E000300007F028FF002800DC7FE00121380021
:10E4F00007F021FF002800DC78E00E9A019902A8BD
:10E5000008F02DF8041E45D102A90122080008F0E8
:10E5100014F8041E3ED10122310005A808F00DF8C0
:10E52000041E37D102A905AA080008F0C7FA041E84
:10E5300030D1010002A807F0FEFE002856D10E9A45
:10E54000019902A808F00BF8041E23D102A90122A8
:10E55000080007F0F2FF041E1CD10122390005A8B3
:10E5600007F0EBFF041E15D102A905AA080008F068
:10E57000A5FA041E0ED1010002A807F0DCFE041E5D
:10E5800008D033E0002E02D0002F00D082E7002D0B
:10E5900097D1002402A807F00DFB05A807F00AFB9D
:10E5A000002C03D0124B9C4200D0E418200009B08C
:10E5B000F0BD0E9B002B00D187E70121019807F0E9
:10E5C000BAFE002812DD01210E9807F0B4FE0028E3
:10E5D0000CDD2900019807F067FE002806DA290003
:10E5E0000E9807F061FE002800DA6EE7004CD1E7D4
:10E5F00000BEFFFFF0B587B0019003A81F000D001B
:10E60000160007F0D1FA002F0CD10C9B002B1DD166
:10E610000D9B1C1E14D0019A29000D9808F05AFE7B
:10E6200004000DE00122019903A807F086FF041EF3
:10E6300006D103AA3100380008F040FA041EE4D0E5
:10E6400003A807F0B7FA200007B0F0BD01222900A7
:10E6500003A807F072FF041EF2D103AA31000C9840
:10E6600008F02CFA041ED3D0EAE7000070B50E4C77
:10E67000051E236805D05A1C2260002B09D02800F3
:10E6800070BD013B2360002BF9D1084816F02CFE29
:10E69000F5E7064816F074FD0028F0D02368002541
:10E6A000013B2360EBE7C046407B010800001040BF
:10E6B00000207047F0B557464E464546DE46E0B569
:10E6C0001D00436D8BB004000E001700002B00D11D
:10E6D000B1E0007801F034FD02AB5874012128004C
:10E6E00007F029FE002861DB210028004C3107F0EB
:10E6F000DBFD00285ADA05A80DF028FF02AB587C94
:10E7000003F0C4F944680734E4082000F1F7C6FFB9
:10E71000099000281AD001002200280007F04EFCC2
:10E72000051E15D005A80DF01BFF0998002805D07F
:10E730002100FAF7F7FC0998F1F7BAFF28000BB0AF
:10E740003CBC90469946A246AB46F0BD3F4DE9E73A
:10E75000099B21001800039316F0DCFD63001800EC
:10E760009A46F1F79BFF81460028EFD02000F1F791
:10E7700095FF804600281BD002AB597C179B0200F6
:10E7800000930598169B03F08FF900282FD0304D89
:10E7900005A80DF0E5FE0998002810D1484651461D
:10E7A000FAF7C0FC4846F1F783FF18E0294DC5E7AA
:10E7B00005A80DF0D5FE099800283ED0234D210074
:10E7C000FAF7B0FC0998F1F773FF51464846FAF79B
:10E7D000A9FC4846F1F76CFF4346002BAED04046FB
:10E7E0002100FAF79FFC4046F1F762FFA6E7434697
:10E7F000019306AB0093159A4B461499059803F0C4
:10E80000B7FB0028C3D1A34621004846CB4416F0ED
:10E8100081FD2100584616F07DFD2200494630005A
:10E8200007F05BFB051EB3D122005946380007F004
:10E8300054FB0500ACE7084D80E751464846FAF71F
:10E8400071FC4846F1F734FF004D77E780B2FFFFD7
:10E8500080B4FFFF80B3FFFF80B0FFFFF0B54546F7
:10E86000DE4657464E46E0B59846436D8FB00400ED
:10E8700003910492002B00D19AE0007801F060FC33
:10E8800004AB587600280BD109A80DF069FE4A4E5A
:10E8900030000FB03CBC90469946A246AB46F0BD56
:10E8A00009A80DF053FE04AB587E03F0EFF843685F
:10E8B0000733DB089A465B009B4601235B44180044
:10E8C0009946F1F7EBFE051E23D0431C0B935346EC
:10E8D0000133C31858460C93F1F7E0FE071E1DD014
:10E8E00001005246189807F069FB061E22D009A8BD
:10E8F0000DF036FE49462800FAF714FC2800F1F71F
:10E90000D7FE38005946FAF70DFC3800F1F7D0FE73
:10E91000BEE709A80DF024FE284EB9E709A80DF0BE
:10E920001FFE49462800FAF7FDFB2800F1F7C0FE5C
:10E93000224EADE75146380016F0ECFC3B00534444
:10E94000524619001998059307F038FB061ECED1E0
:10E950005146059816F0DEFC4B46009501930022C7
:10E9600008AB4146200000F0DBFD061EBFD10B9B2B
:10E9700051461800059316F0CDFC0C9B514618002B
:10E98000059316F0C7FC0AAB04AA944601930F2323
:10E9900063440093039A049B3900099803F0E2FC56
:10E9A000002807D104ABDB7B012BA0D0044E9EE7EF
:10E9B000014E6DE7034E9AE780B0FFFF80B2FFFF84
:10E9C00000B2FFFF80B4FFFF4B6E70B504000D0076
:10E9D000002B44D00368002B3ADB200007F01FFA1D
:10E9E000AB6D5B00984238D86B6E200098470435B9
:10E9F000061E0ED0300070BD0021200007F09BFCE9
:10EA0000002816D02A002100200007F03CFD002835
:10EA10001CD12368002BEFDB2900200007F044FC09
:10EA20000028E7DB2A002100200007F0EEFC002888
:10EA30000CD12900200007F037FC0028DADB2A007F
:10EA40002100200007F0E1FC0028F2D00600D1E709
:10EA5000002107F070FC0028BFD0044ECAE70A1D51
:10EA6000010008F02BF80600C4E7C04680B0FFFFA5
:10EA7000F0B5DE4657464E4645468046E0B59946D7
:10EA800085B0836D01A8DE1D8B46924607F08CF899
:10EA900043460C27F6081D1D4B465246310001A87F
:10EAA00008F020FB041E06D02FE0012101A807F08A
:10EAB00013FB041E29D1290001A807F0F5FB00284B
:10EAC000F3DA013F002F2BD0012101A807F033FC1E
:10EAD0000028E1DD01AA5946584607F040FD041E12
:10EAE00013D141465846FFF76FFF041E0DD15D4616
:10EAF000183501AA2900280007F031FD041E04D1B1
:10EB000041462800FFF760FF040001A807F052F813
:10EB1000200005B03CBC90469946A246AB46F0BDED
:10EB2000004CF5E700B3FFFFF0B5D6464F4646462A
:10EB3000C0B51E0037009EB0804603A889469246A5
:10EB400007F032F806A807F02FF809A807F02CF80C
:10EB50000CA807F029F80FA807F026F812A807F06C
:10EB600023F815A807F020F818A807F01DF81837A3
:10EB70001BA807F019F83A00310003A807F083FC3E
:10EB8000041E16D143461D1D06E003A92A000800F5
:10EB900007F03BFC041E0CD1290003A807F084FBFE
:10EBA0000028F2DA03AA110006A807F0D8FC041E18
:10EBB00021D003A806F0FEFF06A806F0FBFF09A877
:10EBC00006F0F8FF0CA806F0F5FF0FA806F0F2FF1C
:10EBD00012A806F0EFFF15A806F0ECFF18A806F043
:10EBE000E9FF1BA806F0E6FF20001EB01CBC904603
:10EBF0009946A246F0BD414606A8FFF7E5FE041E71
:10EC0000D7D13A00310009A807F061FC041E0DD0ED
:10EC1000CFE7002109A807F08EFB00280AD009A938
:10EC20002A00080007F02FFC041EC2D1099B0193A3
:10EC3000002BEEDB09AA11000CA807F090FC041EC3
:10EC4000B7D141460CA8FFF7BFFE041EB1D10CAAF4
:10EC500006A90FA807F03BFC041E0DD0A9E7002170
:10EC60000FA807F068FB00280AD00FA92A000800A7
:10EC700007F009FC041E9CD10F9B0193002BEEDBD7
:10EC8000269E26991836320012A807F0FCFB041EB7
:10EC900008D08EE712A92A00080007F0B6FB041E70
:10ECA00000D086E7290012A807F0FEFA0028F1DA62
:10ECB0003200269915A807F00AFC041E0ED078E74A
:10ECC000002115A807F037FB00280BD015A92A0052
:10ECD000080007F0D8FB041E00D06AE7159B0193DB
:10ECE000002BEDDB03AA15A918A807F038FC041EB9
:10ECF00000D05EE7414618A8FFF766FE041E00D06C
:10ED000057E709AA12A91BA807F029FC041E00D086
:10ED10004FE741461BA8FFF757FE041E00D048E707
:10ED20001BAA18A9504607F0AEFB041E00D040E70E
:10ED300041465046FFF748FE041E00D039E75246D0
:10ED40005146504607F00BFC041E00D031E7414607
:10ED50005046FFF739FE041E00D02AE75646183603
:10ED60001BAA18A9300007F0B2FB041E00D020E750
:10ED700053469B69002B0DDA0021300007F0DBFAC7
:10ED8000002807D02A003100300007F07CFB041E69
:10ED9000EED00EE732003100300007F0E0FB041E39
:10EDA00000D006E741463000FFF70EFE041E00D0FB
:10EDB000FFE632002799300007F0D1FB041E00D097
:10EDC000F7E641463000FFF7FFFD041E00D0F0E6F5
:10EDD0000CAA06A9484607F0C2FB041E00D0E8E6CC
:10EDE00041464846FFF7F0FD041E00D0E1E64E46DE
:10EDF000414618360FAA1031300007F0B0FB041E50
:10EE000000D0D6E641463000FFF7DEFD041E00D0FC
:10EE1000CFE632000CA9300007F035FB041E00D00D
:10EE2000C7E62900300007F03FFA002807DB2A0078
:10EE30003100300007F0E9FA041EF2D0B9E63200E2
:10EE40000FA9300007F08BFB041E00D0B1E641464D
:10EE50003000FFF7B9FD0400ABE6C04670B50C000A
:10EE6000183406000D00021D2100200008F032FABF
:10EE7000002800D070BD22002900280007F06FFB99
:10EE80000028F7D131002800FFF79EFD0028F1D1BE
:10EE90000121200006F053FFECE7C046F0B55746CD
:10EEA0004E464546DE46E0B59846036B97B00400F3
:10EEB0000F009146002B53D0C36B002B52D0A36D93
:10EEC00006932378013BDBB2042B49D8CE4AD35CAE
:10EED0000793002B44D0200000214C3006F049FF5E
:10EEE00001283DD10AAE09A80DF030FB300006F034
:10EEF0005BFE4946300006F099FE0DAB051E9B46B1
:10EF000057D010AB9A4613AB0593300006F052FE73
:10EF1000584606F04FFE504606F04CFE059806F0A7
:10EF200049FE002F11D018239C46BC44634606932B
:10EF30000C239C46BC44E046380006F03BFE4046AD
:10EF400006F038FE069806F035FE09A80DF008FB1D
:10EF5000280017B03CBC90469946A246AB46F0BD8F
:10EF6000AA4DF5E70DAB18009B4606F01DFE10AB51
:10EF700018009A4606F018FE13AB18000AAE059367
:10EF800006F012FE300006F00FFE4146300006F09B
:10EF90004DFE051E00D187E0584606F00BFE504698
:10EFA00006F008FE059806F005FE300006F002FEA9
:10EFB000CEE7180006F0F8FD10AB18009A4606F0F0
:10EFC000F3FD13AB1800059306F0EEFD41465846DD
:10EFD00006F02CFE051E98D1414650460C3106F035
:10EFE00025FE051E00D090E741460598183106F031
:10EFF0001DFE051E00D088E71F24069A300014402D
:10F0000023005C1EA34154091C19210006F0E6FDF3
:10F01000051E00D079E72100584606F0DFFD051EE9
:10F0200000D072E72100504606F0D8FD051E00D042
:10F030006BE72100380006F0D1FD051E00D064E723
:10F040000C239C46BC44634660462100984606F06B
:10F05000C5FD051E00D058E77B695A460293BB6880
:10F0600007990193B368099800935B4692685B69BE
:10F0700006F058F818239C46BC44634660460121BC
:10F08000069306F05CFE0500300006F093FD58463E
:10F0900006F090FD504606F08DFD059806F08AFDBD
:10F0A000002D00D151E747E74146584606F0BEFD26
:10F0B000051E00D070E7414650460C3106F0B6FD03
:10F0C000051E00D068E741460598183106F0AEFDF0
:10F0D000051E00D060E70121380006F030FE051E55
:10F0E00000D059E718239C46BC4463460021604683
:10F0F000069306F024FE051E00D04DE70C239C4627
:10F10000BC44604606F056FD231D5D46A3461C0028
:10F1100006E022002900280007F077F9002870D1C6
:10F120002100280007F0C0F80028F2DA209B5C4696
:10F13000AB46002B08D02900219B209A2000FFF726
:10F1400097FC051E00D027E7484606F068FE4246B9
:10F15000431E5D460792B346A0461E002CE03100D8
:10F16000484606F006FEC4B222002900380006F028
:10F17000A4FD002844D122000599069806F09DFDC3
:10F1800000283DD15B46009501932A003B003900E1
:10F190004046FFF7C9FC002832D122002900380080
:10F1A00006F08BFD00282BD122000599069806F069
:10F1B00084FD013E002823D1731CD0D14446079B17
:10F1C0003900200098465E46FFF748FEAB46050032
:10F1D000584606F0EFFC504606F0ECFC059806F0A9
:10F1E000E9FC300006F0E6FC002D00D0B0E6236B11
:10F1F000002B00D1ACE6E36B002B00D1A8E65EE665
:10F200005E46AB460500C7E65CE8011080B0FFFF34
:10F210000F4B10B51A680F48002A17D105210A2490
:10F22000017003314170043981700331C1700439B8
:10F23000017109314171063981710439C171093196
:10F2400001720A3941728472C272196010BDC046DF
:10F25000507B0108447B0108064B052802D106E0DB
:10F26000824204D00C331A78002AF9D10023180006
:10F270007047C04664E80110036B002B04D0C06BDC
:10F2800043425841013070470020FCE710B50400AC
:10F2900006F08AFC20000C3006F086FC20001830B6
:10F2A00006F082FC10BDC04670B500250400057054
:10F2B000043006F079FC2000103006F075FC2000C8
:10F2C0001C3006F071FC2000283006F06DFC200098
:10F2D000343006F069FC2000403006F065FC200068
:10F2E0004C3006F061FCA565E56525666566A5669A
:10F2F000E56625676567A56770BDC04670B50025E2
:10F3000004000570043006F04FFC2000103006F0B9
:10F310004BFC20001C3006F047FC2000283006F093
:10F3200043FC2000343006F03FFC2000403006F063
:10F330003BFC20004C3006F037FC2000A565E5655D
:10F3400025666566A566E56625676567A5677C3001
:10F3500006F02AFC2000883006F026FC20009430BD
:10F3600006F022FC2000A03006F01EFC70BDC04656
:10F3700010B5041E09D006F01DFC20000C3006F06C
:10F3800019FC2000183006F015FC10BD70B5061EE3
:10F3900025D0036E012B27D1706F00281BD0B36FCF
:10F3A0000025002B15D0EC006419A4000419002CD2
:10F3B00016D0200006F0FEFB20000C3006F0FAFB11
:10F3C0002000183006F0F6FBB36F0135706F9D42D8
:10F3D000E9D3F9F795FE7C213000F9F7A3FE70BD63
:10F3E00001359D42DFD3F4E7043006F0E3FB300043
:10F3F000103006F0DFFB30001C3006F0DBFB300085
:10F40000283006F0D7FB3000343006F0D3FB300054
:10F41000403006F0CFFB30004C3006F0CBFBBBE7B2
:10F4200070B5051E35D0036E012B33D1686F0028EF
:10F430001BD0AB6F0026002B15D0F400A419A4003C
:10F440000419002C42D0200006F0B4FB20000C3040
:10F4500006F0B0FB2000183006F0ACFBAB6F0136B5
:10F46000686F9E42E9D3F9F74BFE7C212800F9F73B
:10F4700059FE28007C3006F09DFB2800883006F0FD
:10F4800099FB2800943006F095FB2800A03006F088
:10F4900091FB70BD043006F08DFB2800103006F0A3
:10F4A00089FB28001C3006F085FB2800283006F078
:10F4B00081FB2800343006F07DFB2800403006F048
:10F4C00079FB28004C3006F075FBAFE701369E4211
:10F4D000B3D3C8E770B504000D0006F0A7FB002801
:10F4E00000D070BD290020000C310C3006F09EFBCE
:10F4F0000028F6D1290020001831183006F096FBBC
:10F50000EFE7C04610B5097801F0ACFF10BDC0466A
:10F5100010B51830002106F00EFF4342584110BDCF
:10F52000F0B5C646040000B504301F000E0090463A
:10F5300006F096FC236B0500002B33D0E36B002B09
:10F540001DD02E4C30000021183006F0F4FE0028AB
:10F550002AD04346002B2FD16B00079A01333B6022
:10F56000934249D80423069A30001370511C2A0094
:10F5700006F024FD002835D004BC9046F0BD079B62
:10F580003860984238D802000699300006F0DAFC5C
:10F590000028F1D1236B002BEED0E36B0024002B6D
:10F5A000EAD0CFE71548E7E7079B002B24D0069B5E
:10F5B000187001233B60DFE72000012BDCD1079AA4
:10F5C0006B1C3B60934217D8300000210C3006F0D2
:10F5D000D0FB069B02301870591C2A00300006F040
:10F5E000EDFCC9E7069B30009C46691C61442A007B
:10F5F0000C3006F0E3FCBFE70148BDE780B1FFFF38
:10F6000000B1FFFFF0B5C646040000B50E001700BC
:10F610001D1E61D0043006F023FC236B8046002BB6
:10F6200038D0E36B002B17D03B78002B36D1012D5F
:10F6300052D10121300006F082FB00282BD130008E
:10F6400001210C3006F07BFB002824D13000002182
:10F65000183006F074FB1EE085423DD12A003900C7
:10F66000300006F003FC002815D130000C3006F005
:10F67000A1FA2378092B31D030000121183006F08F
:10F680005EFB002807D1236B002B04D0E36B002B1B
:10F6900001D0C9E7164804BC9046F0BD042BF9D14F
:10F6A00043465B000133AB4216D1791C4246300021
:10F6B00006F013FC0028EED143463000591C79189F
:10F6C00042460C3006F009FC0028E4D1300001214C
:10F6D000183006F034FBDEE70648DCE7E9000139C4
:10F6E0000022300006F055FB0028C5D0D3E7C04605
:10F6F00080B1FFFF80B0FFFFF0B50600080089B0C1
:10F700000D001830012106F016FE041E00D09EE008
:10F71000336B002B00D18FE0F36B002B00D18DE019
:10F720000021280006F007FE002800DA8FE02C00F8
:10F730000C340021200006F0FEFD002800DA86E0EF
:10F74000371D3900280006F0AFFD002800DB7EE001
:10F750003900200006F0A8FD002800DB77E002A8B1
:10F7600006F022FA05A806F01FFA2200210002A8DE
:10F7700006F0F5FE041E08D002A806F01BFA05A844
:10F7800006F018FA200009B0F0BD310002A8FFF71A
:10F790001BF9041EF0D12A00290005A806F0DFFE9F
:10F7A000041EE9D1310005A8FFF70EF9041EE3D1CC
:10F7B000B369002B4DD0320005A91032080006F0C5
:10F7C00062FE041ED8D106E005A93A00080006F042
:10F7D0001CFE041ED0D1390005A806F065FD0028E6
:10F7E000F2DA05A92A00080006F0B9FE041EC3D10A
:10F7F000310005A8FFF7E8F8041EBDD1320005A9C5
:10F800001C32080006F03FFE041EB5D106E005A933
:10F810003A00080006F0F9FD041EADD1390005A834
:10F8200006F042FD0028F2DA05A902A806F03CFD28
:10F83000041EA1D0154C9FE7154CA3E7280006F045
:10F840000FFBF36D0733DB08984200D89AE70F4CA3
:10F8500098E705A90322080006F06FFE041E00D0F9
:10F860008AE70DE0002105A806F065FD0028B8D064
:10F8700005A93A00080006F006FE041E00D07BE74A
:10F88000059B0193002BEDDBABE7C04680B3FFFF88
:10F8900080B0FFFFF0B51E00036B83B004000F00C3
:10F8A0001500002B21D0C36B002B20D001211000AC
:10F8B00006F041FD002835DB210028004C3106F020
:10F8C000F3FC00282EDA31002000FFF715FF002896
:10F8D00009D1099B2A000193089B3900009320005D
:10F8E0003300FFF7DBFA03B0F0BD0F48FBE7002160
:10F8F000100006F03EFA002814D10121280006F07D
:10F9000038FA00280ED1280006F089FAE36D013894
:10F91000984207D1FE28D6D10221280006F029FA04
:10F920000028D0D00148DEE780B0FFFF80B3FFFFA2
:10F93000F0B557464E464546DE46E0B51F00036B20
:10F9400097B0040088461600002B00D16EE0C36B10
:10F95000002B6DD00121100006F0EDFC002800DA2C
:10F9600083E0210030004C3106F09EFC002800DBD3
:10F970007BE039002000FFF7BFFE051E4ED1236B50
:10F98000002B53D0E36B002B00D1E7E0A36D06936F
:10F990002378013BDBB2042B48D8AE4AD35C0793F3
:10F9A000002B43D0200000214C3006F0E2F9012862
:10F9B0003CD109A80CF0CAFD0AAB9946180006F024
:10F9C000F3F83100484606F031F90DAB051E9B46B1
:10F9D0004DD010AB9A4613AB0593484606F0EAF8B3
:10F9E000584606F0E7F8504606F0E4F8059806F0A9
:10F9F000E1F84346002B0ED01823434406930C2312
:10FA000043441E00404606F0D5F8300006F0D2F818
:10FA1000069806F0CFF809A80CF0A2FD280017B050
:10FA20003CBC90469946A246AB46F0BD8A4DF5E7F0
:10FA30000021100006F09DF9002816D101213000A8
:10FA400006F097F9002810D1300006F0E8F9E36DD0
:10FA50000138984209D1FE2800D08AE702213000FF
:10FA600006F087F9002800D183E77C4DD6E718001F
:10FA700006F09AF810AB18009A4606F095F813AB0A
:10FA80001800059306F090F83900584606F0CEF8B5
:10FA9000051EA2D1390050460C3106F0C7F8051EEC
:10FAA0009BD139000598183106F0C0F8051E94D195
:10FAB0001F24069A48461440631E9C415309E418CB
:10FAC000210006F08BF8051E00D086E7210058467D
:10FAD00006F084F8051E00D07FE72100504606F0AE
:10FAE0007DF8051E00D078E72100404606F076F844
:10FAF000051E00D071E70C234344210018001E00AE
:10FB000006F06CF8051E00D067E743465B695A466D
:10FB1000029343469B68079901934B469B6809985B
:10FB200000935B4692685B6905F0FCFA1823434436
:10FB300001211800069306F002F90500484606F078
:10FB400039F8584606F036F8504606F033F805986E
:10FB500006F030F8002D00D15DE753E70DAB18003B
:10FB60009B4606F021F810AB18009A4606F01CF8E8
:10FB700013AB1800059306F017F80AAB9946180066
:10FB800006F012F83900484606F050F8051E0CD071
:10FB9000584606F00FF8504606F00CF8059806F0A7
:10FBA00009F8484606F006F838E73900584606F0E6
:10FBB0003DF8051EECD1390050460C3106F036F800
:10FBC000051EE5D139000598183106F02FF8051EFD
:10FBD000DED10121404606F0B2F8051ED8D1182327
:10FBE000434400211800069306F0A9F8051ECFD162
:10FBF0000C234344180005F0DDFF231D1D005B4668
:10FC0000A3461C0006E02A002100200006F0FDFBB0
:10FC1000002878D12900200006F046FB0028F2DAFF
:10FC200023005C469B46209B002B07D0219B209AFB
:10FC300059462000FEF71CFF051EA9D1300006F032
:10FC4000EEF8431E07935B464546B346A0461E00AA
:10FC5000079B34E05CE8011080B0FFFF80B3FFFF3A
:10FC60000799584606F085F8C4B2220031002800F2
:10FC700006F023F8002849D122000599069806F0DD
:10FC80001CF8002842D14A46009601922B0032000F
:10FC900029004046FEF748FF002837D122003100F6
:10FCA000280006F00AF8002830D1220005990698AD
:10FCB00006F003F8079B013B0793002826D1013388
:10FCC000CED144463300290020005E469B46FFF714
:10FCD000C5F8A8460500584605F06CFF504605F0EB
:10FCE00069FF059805F066FF484605F063FF002DA3
:10FCF00000D093E6236B002B00D18FE6E36B002B43
:10FD000000D18BE642E60500A34641E70500B34675
:10FD10003EE7C046036B70B504000D00002B11D008
:10FD2000C36B002B10D00121280006F004FB002833
:10FD300025DB210028004C3106F0B6FA00281EDA37
:10FD4000002070BD0F48FCE70021280006F011F8E4
:10FD5000002814D10121280006F00BF800280ED14C
:10FD6000280006F05CF8E36D0138984207D1FE28C0
:10FD7000E6D10221280005F0FCFF0028E0D002486F
:10FD8000DFE7C04680B0FFFF80B3FFFFF0B5574606
:10FD90004E464546DE46E0B59A46036B83B0070003
:10FDA0000D009146002B47D0C36D07339846DB0802
:10FDB0009B46C36B002B36D0072342469A434533FC
:10FDC0009C46BC4463461F269046019353464A46D0
:10FDD0005946280007F086F9041E17D14346FA6DEC
:10FDE0002800991A06F078F9041E0FD1013E002E62
:10FDF00024D00121280006F09EFA0028E6DB0199B4
:10FE0000280006F051FA0028E0DA0024200003B0B0
:10FE10003CBC90469946A246AB46F0BD280005F092
:10FE2000FEFF00280CD153464A465946280007F0E9
:10FE300059F9041EF2D0E9E71C4CE7E71C4CE5E752
:10FE4000280005F0ECFFF96D013881421DD2411AFE
:10FE5000280006F041F9041ED8D100220021280014
:10FE600005F097FF041ED1D100220121280005F0E2
:10FE700090FF041ECAD1FB6DFE2B0DD03B6B002BF7
:10FE8000C3D0FB6B002BC1D096E70122280005F000
:10FE900080FF041EE1D0B9E700220221280005F00E
:10FEA00078FF0028EAD00400B0E7C04680B0FFFF2A
:10FEB00000B3FFFFF0B5C6460C0000B5010082B0EC
:10FEC000200015001E0001F0CDFA002803D002B07A
:10FED00004BC9046F0BD27007C3733002A0039006F
:10FEE0002000FFF753FF0028F1D139002000FFF771
:10FEF00011FF0028EBD128239846A044414620005A
:10FF0000FFF7FAFB0028E2D1210001968831009525
:10FF100043463A002000FEF7C1FFD8E7F0B5464659
:10FF2000D6464F46C0B50378AAB004000E00002B99
:10FF300000D1F6E00A789A4200D0F2E08823984691
:10FF400088444146883006F0AFF9002800D0E8E048
:10FF5000942399462000B1444946943006F0A4F910
:10FF6000002800D0DDE0A0239A462000B244A03053
:10FF7000514606F099F9041E00D0D2E002A805F01F
:10FF800013FE05A805F010FE08A80BAD05F00CFE49
:10FF90000CA82C7005F008FE0FA805F005FE12A8AD
:10FFA00005F002FE15A805F0FFFD18A805F0FCFD00
:10FFB0001BA805F0F9FD1EA805F0F6FDAC65EC6583
:10FFC0002C666C66AC66EC662C676C67AC673400BC
:10FFD0003178280001F046FA2B6B2834002B00D131
:10FFE0007EE0EB6B7C36002B00D17BE00121300002
:10FFF00006F0A1F9002800DA91E01EA9300006F011
:020000041001E9
:1000000053F9002800DB8AE021002800FFF774FB89
:10001000071E09D1019000902300320002A9280098
:10002000FEF73CFF071E4FD002A805F0C3FD05A850
:1000300005F0C0FD08A805F0BDFD2B6E012B2DD1EC
:10004000686F00281BD0AB6F0026002B15D0F40082
:10005000A419A4000419002C1CD0200005F0AAFD4E
:1000600020000C3005F0A6FD2000183005F0A2FDA0
:10007000AB6F0136686F9E42E9D3F9F741F87C21F6
:100080002800F9F74FF838002AB01CBC9046994672
:10009000A246F0BD01369E42D9D3EEE70CA805F08A
:1000A00089FD0FA805F086FD12A805F083FD15A8AF
:1000B00005F080FD18A805F07DFD1BA805F07AFD70
:1000C0001EA805F077FDBBE7414602A806F0ECF854
:1000D000002805D1494605A806F0E6F8002822D0F8
:1000E000154FA1E70021300005F043FE002816D18E
:1000F0000121300005F03DFE002810D1300005F050
:100100008EFEEB6D0138984209D1FE2800D07BE7C6
:100110000221300005F02DFE002800D174E7074FC2
:1001200082E7054FAFE7514608A806F0BDF8071E65
:1001300000D179E7004F77E780B0FFFF80B3FFFF82
:100140000138C3B20020042B01D8014AD05C7047AB
:100150005CE80110F0B5CE46474680B5446805001E
:10016000A5B000200E2C27D92600012301AF0E3E9A
:1001700001937E600E2E5CD815AB3C220021180046
:100180009846BB60F0F7DBFA38229446AB68B200C1
:100190006344994619004046F0F7B5FA264B002112
:1001A000E21892004846F0F7CAFA3A0029002800FF
:1001B00006F069F9002804D025B00CBC9046994699
:1001C000F0BD04AC23003A0043CA43C307A841462C
:1001D0003822A060F0F797FAE021200005F07CFFBC
:1001E0000028E9D122002900280006F04CF9002857
:1001F000E2D17A68072A07D9104B00219C46624455
:1002000092001CA8F0F79BFA22003900380006F093
:100210003AF90028D0D10F23E02138007B6005F0A7
:1002200007FF0028C8D13A002900280006F02BF962
:10023000C2E70348C0E7C046F2FFFF3FF9FFFF3FB8
:1002400080B0FFFF70B54468050090B00020072C17
:1002500018D90123073C03930494092C38D806AE1F
:100260002822002130000596F0F769FAA968A2005B
:100270001C313000F0F747FA1F2103A805F02CFFCE
:10028000002801D010B070BD049B00220193FF2113
:1002900001332800049305F07CFD0028F2D16A6840
:1002A000082A08D90B4BA8689C466244920020306B
:1002B0000021F0F744FA03A91322080006F0C2F95E
:1002C0000028DFD103AA2900280006F046F8D9E764
:1002D0000148D7E7F8FFFF3F80B0FFFF10B5426845
:1002E000040096B00020102A27D90123103A019368
:1002F000122A24D802929200A16804A840310390E7
:10030000F0F701FA092101A805F0E6FE002814D152
:10031000A0686268036CDB05DB0D0364112A07D952
:10032000094B44309C46624492000021F0F707FAE2
:1003300001AA2100200006F010F816B010BD12230B
:1003400048220293D8E7C046EFFFFF3FF0B5DE46F4
:1003500057464E464546E0B50C2187B0040005F0EF
:100360003DFC0190002800D0B8E0A368626898695D
:1003700019689E6A44188442894134191C60B44249
:10038000A4415D6892009A18494203924A19DD69B6
:100390006442A846A1469044C1448A428941A1458D
:1003A000A44149426442DD6A0919DC69AC46A045B2
:1003B0009241CC4452428918AC4592419C685242C9
:1003C00089180A198A428941DC6849426746A04671
:1003D0008C468218E0445F6082428041DF69444677
:1003E000BC4640421F6A059101198C44049464463E
:1003F000BC4662440294BA42A4416742029CBB4696
:10040000A246B2189A60B24292415C6ADA448142D2
:100410008941DA458041A04652429146AC4640426D
:100420004942D04409180298C144CC4491459241B4
:100430008146D86952428145804189184042081856
:10044000A0458941AC45924149424018524280182A
:10045000049A0599904688459241524282185869FB
:1004600067468446186A196980465118914292413C
:100470004144814280415242944440428246604419
:100480008919DF600719B846B142B641A045A441B9
:100490007642B044196141466442A146B045B64136
:1004A0005045A4414919A942AD41944592411800D3
:1004B00064427642A4194C446D4265195242AA180E
:1004C00059619A61039A1C30824207D9D21A1D3AA7
:1004D0009208013292000021F0F731F9019807B03B
:1004E0003CBC90469946A246AB46F0BDF0B5DE4610
:1004F00057464E46454601230400E0B59DB008909E
:100500000C930FA80C33342200210D930E90F0F7BA
:1005100016F91821200005F061FB0790002800D093
:1005200057E2A068036B416D98460368026D43442F
:100530001E00CC1815194645B6418C42A441C36D26
:1005400064427642A6199542A44101929D4292418D
:1005500064425242A419A41AED1A0091056042683F
:10056000611C00D13DE21219A242A4416442456BD4
:100570004746AC4629000295856D6244AB46AD18EE
:100580008A4292415E1952425D45AD4112199E4226
:10059000A4416D42AA186442A2184645A44164428F
:1005A000141B019AF71B9742AD41BF1A6D42826836
:1005B000641B47601519002C00DA56E2A542A441DD
:1005C0006442816B029E8C4665445A1903918D42A8
:1005D000AD4102999A42BF41961B8A4292417F42A5
:1005E0006D427D195242AD1A009A9642BF417F4238
:1005F000B61AED1BC2682D1986605419002D00DA59
:100600002EE2AC42AD416A429146C16B47468C46F0
:100610006444A2465C46019A5744D619009A47455D
:10062000BF419519039A0591AA1A141BA4468A453D
:10063000A44101997F428E42B641009964423C191F
:100640008D42BF41039976427F4234198D42AD41BC
:100650003C195A45BF416D42641B7F42E71B9C45D4
:10066000A441624664423F1BD21A4F44C2600269F1
:100670007FB2D419002F00DAEDE1BC42BF417A42CB
:100680000492009A47469446644421008A46140026
:10069000524492460A91016CA245A4410A00524478
:1006A000914664420B940A9C029AA246069189459F
:1006B00089419446009C4942A245A441CC448946C4
:1006C000029964428C4589415A460A940B9C019DCB
:1006D000A24667444942EE198C464745BF419519E9
:1006E0000199059A0A9CAA1A8E42B641544409926D
:1006F0004C4464447F4209993C195D45BF418C4696
:1007000076423419059E7F42B542AD413C199C4565
:10071000BF416D42D21A641B7F42E71B04999A4283
:10072000A4418C4664423F1BD21A6744026142696D
:100730007FB2D419002F00DA88E1BC42BF417A426F
:100740009246426C5C440399A04694460D00D844FE
:10075000C44465442F00029D0492EE19009D5C453F
:10076000A441AD195A199146D8459241524290463A
:10077000049A8F42BF419445924152429446029955
:10078000009A64428E42B64144447F429542AD4154
:1007900064443C199945BF41764234196D4206992B
:1007A0002C197F423F198945A4414A4664423F1BA8
:1007B000574486697FB2541A4461F519002F00DA54
:1007C0003FE1BD42BF417A4292465D195A199046B7
:1007D000846C0599A4460E0098459241C444664431
:1007E000524237009046A4459241039E9D42AD413E
:1007F000F6195242B14694468F42BF416D42039969
:100800004544D9447F428E42B64165447D19D9455D
:10081000BF417642049975197F427F198945AD41E0
:100820004A466D427E1B551A56448561C56976B2AB
:10083000AF19002E00DAFFE0B742B641724292468D
:100840000699059E88463200C56C9946EF19B84452
:10085000424494468845924152429046B445924162
:10086000E14452429446AF42BF41994592417F4292
:10087000524247449046A145924167445242474400
:10088000BF1A4A463E00171B026A5644C761944687
:100890009719002E00DACAE0B742B641724291467B
:1008A000019A049E94466744F1198C460699974232
:1008B000BF410E006644B046049E88459241B4454F
:1008C000B6417642B44652427F4267449446A845B8
:1008D000924167445242BF1A42463E00571B426A49
:1008E0004E44076290469719002E00DA9BE0B7420B
:1008F000B641764200998C466744E21994460499C1
:10090000A445924188465242E0449446009A974258
:10091000BF41884592417F42019952426744D719AD
:10092000884592415242BF1A4246BE19876A521AFE
:100930004262BA19002E00DA71E0B242BF417F4232
:100940005A441600AA189446AC4589415E45B64102
:1009500049428C46A21800997642A242A441B4446E
:100960008A42B6416442511A64447642A61B8162AF
:10097000C16AF6198A19002E4DDBB242B6417642A1
:10098000019F9A18BC1829199A429B41BC42A44164
:100990005B42A942AD416442E41859459B416D4216
:1009A0005B422D19ED1A5B46AE19C91AF343DB17EA
:1009B00033400363089BC1625A680D2A07D92D4B47
:1009C00034309C46624492000021EFF7B8FE002EBE
:1009D0000CDB07981DB03CBC90469946A246AB463E
:1009E000F0BD54425441013A6442C0E5224A0D9B95
:1009F0009446089C0E9A63449B00764200929E5057
:100A00000CA92200200005F000FD0028E1D10123FF
:100A10005B422360DDE77642B142B641B0E7764201
:100A2000B742BF418CE77642B045B64162E77642B5
:100A3000B4459241914633E77642B542924192469F
:100A4000FEE67F42BE4292419246BEE67F42BA42F5
:100A50009241924675E67F42BA429241049210E674
:100A60006D42AA4292419146CFE56442A242A4411E
:100A7000A7E5C046F3FFFF3FFFFFFF3FF0B5CE46BF
:100A8000474680B54468050095B00020072C2AD958
:100A9000012306930393093B98463C4AA0440892DD
:100AA0004346022209AF07920597082B20D92C2232
:100AB00000213800EFF743FEAE68202220363100D7
:100AC0003800EFF720FE0A230493314B0021E2188F
:100AD00092003000EFF733FE03A906AA080005F0E4
:100AE0003EFD002816D015B00CBC90469946F0BDCE
:100AF0002A3200213800EFF722FE4346AE689A0002
:100B0000203631003800EFF7FEFDA31F0493082CB8
:100B1000DBD1E1E703AA2900280005F01EFC00282C
:100B2000E1D108235B4298466C68A0444346082BF9
:100B300027D89B0099462C2200213800EFF7FFFDB3
:100B4000AE684A46203631003800EFF7DCFD079BDF
:100B5000019343440493082C06D90D4B0021E2185D
:100B600092003000EFF7EBFD03A906AA080005F09C
:100B7000F6FC0028B7D103AA2900280005F0EDFBF8
:100B8000B1E720239946183B9846D4E79CCD00084E
:100B9000F8FFFF3FF0B5DE4657464E464546012377
:100BA000E0B506008FB0039306A80733202200218A
:100BB00004930590EFF7C3FD0E21300005F00EF809
:100BC000071E00D0B4E0B068C26903689246C16AEB
:100BD0009A1A53459B418C468A4289415B42C91A05
:100BE0006346D21A026043680022002900D0ACE0BC
:100BF000016A056B8946591A4B459B415B42D21AE3
:100C0000A9429B415B42D21A8368491B52B29B4660
:100C100041600023002A00D09DE0426A446B904668
:100C20005A464146511AC345924152429B1AA1422B
:100C3000924152429B1A0022091B5BB281600092D2
:100C4000C168002B00D08CE05246836AD21A521839
:100C50009346994289415245924149425242521A21
:100C60000099E3448A469244E345924159465242F0
:100C70005244C160016952B201938B189B46002A0D
:100C80005EDB9345924153429A464B4662469A1A1E
:100C90005A44A918E3459B414A4592415B4252425E
:100CA000D31AA94292419B4652425A44016141697A
:100CB00052448B189946002A6EDB9145924151426D
:100CC00043465A1B4A44A318A945AD4142459241A7
:100CD0009C4652426D42531BA445AD419846634623
:100CE0006D4245446D18816943614A19002D57DBF7
:100CF000AA42AD416D42019B191B8918A242A44131
:100D000099429B4164425B421C1B6419E343726835
:100D1000DB1723408161C361082A07D9224B2030A9
:100D20009C46624492000021EFF709FD002C1FDB76
:100D300038000FB03CBC90469946A246AB46F0BD89
:100D4000524291429B419A469FE74A4293429241C6
:100D50005B18D2B24CE753429B459B419344DBB2B4
:100D60005BE75A4291429241D2B20092C9186BE7B6
:100D70000E4A049B9446059A63449B006442009289
:100D80009C5003A93200300005F03FFB0028CFD172
:100D900001235B423360CBE75242914289418FE7A6
:100DA0006D42A942AD41A6E7F8FFFF3FFFFFFF3FBD
:100DB000F0B5DE4657464E46454601230400E0B5F1
:100DC00095B0069008930BA80833242200210993BC
:100DD0000A90EFF7B4FC1021200004F0FFFE05900C
:100DE000002800D0EEE1A068036A02689C46456ACC
:100DF0006244914602932B00C46A4B44066B1F1B4E
:100E0000416BA346BC1B621A9446826B0395019208
:100E1000AB429241029D52429046A94592415B45A8
:100E20009B4152425B424244B742BF41D21A8C427C
:100E30009B417F42D21B019C5B42D31A6246A44570
:100E4000BF41121B7F4202604268DB1BD718002B98
:100E500000DABFE19F429B415B42039A856A944658
:100E60006744AC46BC446446A41B621AA046019C7D
:100E70000495141BA146C46B0094AC45A441039D8A
:100E80006442AF42BF41A246B445A4417F4264429E
:100E900057443F1B019D8845A441AA4292416442A8
:100EA0003F1B009C5242BF1AA14592415242BF1AB9
:100EB0004A46121B42608268FB18D718002B00DAE2
:100EC000B7E19F429B412C005B42049DAC466744C6
:100ED000BC46DC446246521A141BA046DC45A441C1
:100EE000AF42BF416442A1468C45A4417F42644267
:100EF0004F443F1B019CA2429241009C5242BF1AA8
:100F0000A04592415242BF1A4246FB18C768121BC5
:100F10008260FA18002B00DA86E19A429B415B421C
:100F200007935A449146B046B446D944C844C44491
:100F30006346029DCF183B1B5C1BA246D945A441CA
:100F40006442A146B045A4416442A046B445A441D0
:100F50006442A4465A4592418F42A441524264429F
:100F60004A44A146009CAB429B41A742BF41424438
:100F700062447F424A44D21B5B42D31A039A079CC5
:100F80009245BF41A44654467F42DB1BA21A6344EC
:100F9000C26002695BB2D718002B00DA40E19F42C1
:100FA0009B415B42F719F219914688468C46C8442A
:100FB000019DC444AA466246039D5244541BA24666
:100FC000B145A4416442A1468845A4416442A0467B
:100FD0008C45A4416442A446019CB742BF41A24251
:100FE000A4417F4264424F44AA429241A1464744F1
:100FF000049D674452424F44BF1AAA45924152424F
:10100000BF1A5246521BFB18026142695BB2D718E5
:10101000002B00DA00E19F429B415B42CF19CA19C5
:101020009146019A009D90469446C844C444AA46FD
:101030006246049D5244541BA2468945A441644221
:10104000A146019C8F42BF41A045A4416442A046F5
:10105000019C7F42A445A4416442A446009C4F44A5
:10106000A242A4416442A146AA4292414744674435
:1010700052424F44BF1ADA4592415242BF1A5C466F
:101080005246121BFB18426182695BB2D718002BD3
:1010900000DABDE09F4292415242019DAC46674456
:1010A000EB199A46009B2C0099469846D144C844B7
:1010B000C4446346029DCB185D1B01952500A245E3
:1010C000A4416442A246009CAF42BF41A145A44155
:1010D0006442A146009CAC45AD41A045A441644298
:1010E000A0467F4257444F446D424744EF198B421C
:1010F000AD416D42EF19029D039CAB42AD41019B96
:101100006D429C467D1BA445BF417F42EB1B9B1853
:101110006246C569121B5BB28261EA18002B00DAD5
:1011200071E09A429B415B420193009B029C9C466A
:101130006244A4469F18DD19AC446346049C1C1B02
:10114000A14623005C461B1B98469B1B9A46009BAE
:10115000029C9F42BF419A4292419D42AD417F42D3
:1011600052426D42BA18AA18A445AD41049C6D4282
:10117000A445A441AA186442141BD9459241B04524
:10118000B6415242A41A7642A41B019B8A45B6413D
:101190009C4653467642A41B644464B2591AE34306
:1011A000DB1723400362069BC1615A68092A07D9ED
:1011B000224B24309C46624492000021EFF7BFFA94
:1011C000002C0BDB059815B03CBC90469946A24616
:1011D000AB46F0BD5B429A429B413EE6184A099BF2
:1011E00094460A9A634464429B009C50069C009279
:1011F00008A92200200005F008F90028E2D1012307
:101200005B422360DEE75B429D429B4101938CE79A
:101210005B429A42924140E75B429A429B41FDE623
:101220005B429A429B41BDE65B429F429B410793D2
:1012300077E65B429A429B412C0046E6F7FFFF3F70
:10124000FFFFFF3FF0B5CE46474680B54468050036
:1012500095B00020052C28D93C4A0123089202228F
:101260000693039309AFA31F079205979846062B91
:1012700020D92C2200213800EFF761FAAE6818223D
:10128000183631003800EFF73EFA08230493304B4C
:101290000021E21892003000EFF751FA03A906AAE4
:1012A000080005F05CF9002816D015B00CBC90467B
:1012B0009946F0BD2A3200213800EFF740FA434644
:1012C000AE689A00183631003800EFF71CFA231F79
:1012D0000493062CDBD1E1E703AA2900280005F0DE
:1012E0003CF80028E1D16C68A31F9846062B27D84C
:1012F0009B0099462C2200213800EFF720FAAE68B7
:101300004A46183631003800EFF7FDF9079B019384
:1013100043440493062C06D90D4B0021E218920099
:101320003000EFF70CFA03A906AA080005F017F938
:101330000028BAD103AA2900280005F00EF8B4E766
:1013400018239946123B9846D4E7C0468CCD000836
:10135000FAFFFF3FF0B5CE46474680B5446805002A
:1013600095B00020062C28D93C4A0123089202227D
:101370000693039309AFE31F079205979846072B3F
:1013800020D92C2200213800EFF7D9F9AE681C22B1
:101390001C3631003800EFF7B6F909230493304BBF
:1013A0000021E21892003000EFF7C9F903A906AA5C
:1013B000080005F0D4F8002816D015B00CBC9046F3
:1013C0009946F0BD2A3200213800EFF7B8F94346BC
:1013D000AE689A001C3631003800EFF794F9631FAD
:1013E0000493072CDBD1E1E703AA2900280004F0CD
:1013F000B4FF0028E1D16C68E31F9846072B27D87B
:101400009B0099462C2200213800EFF798F9AE682E
:101410004A461C3631003800EFF775F9079B0193F7
:1014200043440493072C06D90D4B0021E218920087
:101430003000EFF784F903A906AA080005F08FF839
:101440000028BAD103AA2900280004F086FFB4E7D7
:101450001C239946153B9846D4E7C04694CD000816
:10146000F9FFFF3F70B504000D0084B0FDF78EFF5B
:1014700025700D2D00D994E1CC4BAD005B599F46F2
:10148000CB4B01A8636604F08FFB2000C94A1021F2
:10149000103005F0E3F8051E00D121E201A804F0A8
:1014A00089FB2000FDF772FF26E0C34B0125636630
:1014B0000623C24AA360E260C14A23626262C14A53
:1014C00023656265C04AE362A363C04B6560E56162
:1014D000E564A56222636563E363BD4B25646564CF
:1014E000A364201D04F09BFCA06520004C3004F098
:1014F00096FC25660025E065280004B070BDB54B5C
:10150000012563660823B44AA360E260B34A2362FC
:101510006262B34A23656265B24AE362A3636560AF
:10152000E561E564A56222636563AF4BD4E7AF4B29
:10153000012563660C23AE4AA360E260AD4A2362D4
:101540006262AD4A23656265AC4AE362A36365608B
:10155000E561E564A56222636563A94BBCE7A94B1D
:10156000012563660823A360A74BA84AE36007230D
:101570006262A74A23626265A64A2365E362A363A7
:101580006560E561E564A56222636563A24BA3E73C
:10159000A24B012563661123A14AA360E260A14A20
:1015A00023626262A04A23656265A04AE362A36384
:1015B0006560E561E564A562226365639C4B8BE72A
:1015C000082301259B4AA360E2609B4A6361A261F4
:1015D0009A4A236262629A4A23656265994AE36283
:1015E000A36365602561E561E564A56222636563C7
:1015F000954B71E70C230125944AA360E260944A5D
:101600006361A261934A23626262934A23656265C1
:10161000924AE362A36365602561E561E564A562C2
:10162000226365638E4B57E7102301258D4AA36023
:10163000E2608D4A6361A2618C4A236262628C4AD5
:10164000236562658B4AE362A36365602561E5619A
:10165000E564A56222636563874B3DE72000874B05
:10166000874A63661021103004F0F8FF051E00D091
:1016700017E7261D0121300004F061FB051E00D094
:101680000FE7FF21300004F0D3FC051E00D008E76F
:1016900013223100300004F050FF051E00D000E797
:1016A000300004F0BCFB4836A065764A10213000BB
:1016B00004F0D4FF051E00D0F3E60122FC21300027
:1016C00004F067FB051E00D0EBE62000092128305E
:1016D00004F035FB051E00D0E3E620000121403078
:1016E00004F02DFB051E00D0DBE62000343004F0B2
:1016F00061FAFE23E365FFE6634B0125636606237B
:10170000624AA360E260624A2365A261614AE362C1
:101710006262614AA3636265604A656025616561D2
:10172000E5612562E564A562226365635C4BD3E6EF
:101730005C4A5D4BE2605D4A0125A2615C4A6366DA
:1017400062620822072322655A4AA36062655A4AE8
:10175000E362A363656025616561E5612562E56417
:10176000A56222636563554BB6E6554B012563665A
:101770000823544AA360E260534A2365A261534A96
:10178000E3626262524AA3636265524A6560256100
:101790006561E5612562E564A562226365634E4B80
:1017A0009AE62000FDF7F2FD4C4DA5E684E9011014
:1017B0005501011048ED01104D03011054EE0110C8
:1017C000F4ED01103CEE01100CEE011024EE0110BE
:1017D000A4CD0008B10D011080F0011000F001103F
:1017E00060F0011020F0011040F00110ED04011034
:1017F00060F10110A0F0011030F10110D0F00110E3
:1018000000F10110950B011058EF0110E8EE0110E6
:101810003CEF011004EF011020EF0110DD02011078
:10182000A0F2011090F101105CF20110D4F101104E
:1018300018F201105CEA0110BCE90110DCE90110AA
:101840003CEA0110FCE901101CEA01106CEB0110EC
:101850007CEA0110ACEA01103CEB0110DCEA01105B
:101860000CEB0110DCEC01109CEB0110DCEB011027
:101870009CEC01101CEC01105CEC01104502011005
:101880001CED011024ED011045120110DCED0110DA
:101890008CED011090ED0110C4ED011094ED0110DC
:1018A000ACED0110CCEE0110551301106CEE0110DF
:1018B00070EE0110ACEE011074EE011090EE01100C
:1018C0007D0A0110E0EF011078EF01107CEF0110AC
:1018D000C0EF011080EF0110A0EF011080B1FFFFF9
:1018E000261D0121300004F02AFA051E00D0D5E59E
:1018F000E021300004F09CFB051E00D0CEE5012263
:101900003100300004F019FE051E00D0C6E5E021CC
:10191000300004F08DFB051E00D0BFE50122310030
:10192000300004F00AFE051E00D0B7E5300004F0D8
:1019300076FAA06520000521283004F000FA051E83
:1019400000D0ABE520000121403004F0F8F9051E7D
:1019500000D0A3E52000343004F02CF9DF21483614
:1019600001224900300004F014FA051E00D095E56C
:101970000B4A102101A804F071FE051E00D08DE570
:1019800001AA3100300004F0A2FD051E00D085E55B
:10199000C023FF33E36501A804F00CF9ACE5C046B1
:1019A00050ED011010B594210AF008FE10BDC0469C
:1019B00010B5002802D094210AF02EFE10BDC046BA
:1019C000020000B5343283B00092031D94220AF065
:1019D000B7FE03B000BDC0460A0053425A4103009F
:1019E00010B5011D013234330AF042FE10BDC0466D
:1019F00010B504000020002A06D0201D13000A00A4
:101A0000010020000AF060FE10BDC04610B50A00BB
:101A1000011D0AF077FE10BD10B5F4210AF0CEFDCD
:101A200010BDC04610B5002802D0F4210AF0F4FD24
:101A300010BDC046020000B5343283B00092031DD1
:101A4000F4220AF07DFE03B000BDC0460A005342F6
:101A50005A41030010B5011D033234330AF008FE69
:101A600010BDC04610B504000020002A06D0201D7D
:101A700013000A00010020000AF026FE10BDC04637
:101A800010B50A00011D0AF03DFE10BD421E030004
:101A9000042A05D88000C018024BC000C018704747
:101AA0000020FCE7E4F20110F0B54E46DE46454664
:101AB0005746E0B5040087B0080015000392994628
:101AC000FFF7E4FF061E00D1A0E0002D00D19DE04D
:101AD000A24B4568984629239B4643465A461B68B5
:101AE00000219B5C0A3A924696229A459B4112033A
:101AF0001340A022120294466A1E634413430492C8
:101B00002000122213F03CF843465A46EF1DFF080E
:101B1000F9001B6805919B5C87229A459B41120343
:101B200013409022120294464A1E6344134300213C
:101B30001222200013F024F8894B19689B468B6B06
:101B4000E3181A680B6924331B191B689B009B0C54
:101B50009B0099184B46002B14D03A001098C847A8
:101B6000002834D07F4DC0231322DB000021200049
:101B700013F006F8280007B03CBC90469946A246F0
:101B8000AB46F0BD2F1E22DD5346049AAA469A4367
:101B90002B00203B9B1AB1460D001E001F2F00DCBE
:101BA000D9E020234146292209688A5C00951F2A32
:101BB00000D8CAE06C4A6D49200013F0CBFC002825
:101BC000D0D1203F0435B742E8D14E4655460921D1
:101BD000200003F051FD059BAB4200D991E0644B1E
:101BE00030220021200012F0CBFF42462923126848
:101BF000D35C1F2B0CD85B4680211B681A68A21887
:101C000013681942FCD1E0231B020AE0594DB1E7E9
:101C10005B461B681A68A2181368002BFCD1E023EE
:101C20001B03049A002113432000122212F0A8FF84
:101C3000B2690E2120002B0003F0AAFB0E220A211C
:101C4000200003F0F1FC00280ED080231322DB01DA
:101C50000021200012F094FF2B000A22039920009B
:101C600003F022FC00257EE729239A46434652468C
:101C70001B6820009B5C0A3A9146C32299459B4110
:101C800012031340D0221202944663442B436F1C6C
:101C90001222002112F074FF3B00F26920000D2196
:101CA00003F076FB434652461B6820009B5CF02203
:101CB00099459B41D2021340802212029446049A15
:101CC00063441A4313000021122212F059FF2A4BD9
:101CD00030220021200012F053FF307B03F0F8F98E
:101CE000280003F0C9F92B00200008220A2100F087
:101CF0004BFE842313229B010021200012F040FFA1
:101D0000A3E729229146424649461F2712685B1BDA
:101D1000525C20009742924152420C3293401A008A
:101D200080239B0513430021802212F029FF4346A4
:101D30004A461B6800219B5C00229F4252412000C2
:101D400023320E4B12F01CFF49E7074A07492000D7
:101D500013F0C4FB33E73B0024E7C04614E8010856
:101D6000DCC2010801003200E146D2528D0B746CD6
:101D700009A000000B0032000A80000098900000CB
:101D8000F0B55746DE464E464546E0B5040085B000
:101D900008008A4615001F00FFF778FE061E00D1D6
:101DA000D9E00395002D00D1D5E0002F00D1D2E07D
:101DB0007968002900D1CEE0B968002900D1CAE0D5
:101DC0006949456889462921884649464046096847
:101DD000D2220B5C1F218B46E0219B459B410902CF
:101DE0008C46120313406344691E0B430291122276
:101DF0000021200012F0C4FE4846424600680299C5
:101E0000835C9020872200029B459B4184461203FD
:101E1000134063440B4312220021200012F0B0FE55
:101E20004A46404612680021135CC3229B459B41F1
:101E300012031340D0221202944663442B43122211
:101E4000200012F09DFE4A46404612680299135C3B
:101E5000A5229B459B4112031340B02212029446D7
:101E600063440B4312220021200012F089FE4A46EF
:101E7000404612680299135CB4229B459B411203B1
:101E80001340C0221202944663440B4312220021E5
:101E9000200012F075FE2B0032690E21200003F0A5
:101EA00077FA2B00B2690921200003F071FA6B1C4C
:101EB00072690D21200003F06BFA2B00326A0B21AE
:101EC000200003F065FA2B00726A0C21200003F059
:101ED0005FFA280003F0D0F8307B03F0F9F84846A9
:101EE000036840461B5CA020962200029B459B4154
:101EF000844612030299134063440B4312220021CB
:101F0000200012F03DFE2B00039A0A21200003F06E
:101F10003FFA09230C2200930B2101332000019585
:101F200003F0DCF82B000B227968200003F0BCFAE8
:101F30002B000C22B968200003F0B6FA00233B7096
:101F400053467B70FC232000DB011322002112F09A
:101F500017FE002000E0054805B03CBC90469946BD
:101F6000A246AB46F0BDC04614E801080B003200A3
:101F7000F0B557464E46DE464546E0B50400ABB0E8
:101F80000E0092461F00002900D19FE0002B00D1D7
:101F90009CE0349B002B00D198E0359B002B00D1B6
:101FA00094E0349B5878FFF771FD8046002800D1FB
:101FB00095E04368359A994608AB059319AB0693AB
:101FC000349B2000597804ABFFF7DAFE051E7ED162
:101FD000DC4B00219B461A682923D35C1F229446C0
:101FE000D2229C459B4112031340E02212029446E8
:101FF0004A466344013A134303922000122212F02E
